:100000000C94F91C0C942A1D0C942A1D0C942A1D86
:100010000C942A1D0C942A1D0C942A1D0C942A1D44
:100020000C942A1D0C942A1D0C942A1D0C942A1D34
:100030000C942A1D0C942A1D0C942A1D0C942A1D24
:100040000C942A1D0C94BAA10C942A1D0C942A1D00
:100050000C942A1D0C942A1D0C94E0DB0D942A119B
:100060000C942A1D0C9401FA0C94F7F90C942A1D97
:100070000C942A1D0C942A1D0C942A1D0C942A1DE4
:100080000C940CF80C942A1D0C942A1D0C942A1D17
:100090000C942A1D0C942A1D0C942A1D0C942A1DC4
:1000A0000C942A1D0C942A1D0C94DEF70C942A1D26
:1000B0000C942A1D0C942A1D0C942A1D0C94B0F744
:1000C0000C942A1D0C942A1D0C942A1D0C94D750B4
:1000D0000C94AD500C942A1D0C942A1D0C942A1DCE
:1000E0000C942A1DD91E1F1F251F4C1F591F621F4C
:1000F0006D1F312751282D296029BD34BD347B2A3D
:100100001E2B2D28BD34BD34BB2C542E8C2EBD345B
:100110008A30BD34BD34DB31BD34BD3465329832F4
:10012000BD341433D0339B2EA32EC72EEB2E1F2F9E
:10013000C22FD62FEF2FFC2F09301D30E1B503B6AB
:1001400023B648B66DB624B892B6B5B6D8B6FDB6E5
:1001500022B747B76CB791B724B8B6B7DBB700B8CA
:10016000B2B9B5B9B9B9BCB9BFB9E9B9C3B9C6B9BA
:10017000CAB9CDB9D0B9D4B9D7B9DAB9E9B9DEB904
:10018000E1B9E4B907E70AE7F9E6FDE603E741E785
:100190000EE712E718E71CE720E726E72AE72EE735
:1001A00041E734E738E73CE72CED31ED36ED40ED43
:1001B0004AEDC3ED54ED5CED64ED6EED78ED82ED4E
:1001C00091ED9BEDC3EDA5EDAFEDB9ED34FA3AFA43
:1001D0004CFA5CFA64FA91FA68FA91FA6CFA70FADD
:1001E00091FA74FA78FA7CFA84FA91FA8EFA084A4B
:1001F000D73B3BCE016E84BCBFFDC12F3D6C74313B
:100200009ABD56833DDA3D00C77F11BED9E4BB4C91
:100210003E916BAAAABE000000803F05A84CCDB25B
:10022000D44EB93836A9020C50B9918688083CA63C
:10023000AAAA2ABE000000803F000C9400B80C94CB
:100240003AFA0C94654F0C94B6B70C9474FA0C946B
:10025000251F0C94D0330C9484FA0C9403B60C94A0
:10026000E1B50C94FDB60C947CFA0C9424B80C9473
:100270001F1F0C941F2F0C94C3ED0C94C3B90C9446
:1002800026E70C941D300C944CFA0C94591F0C94D6
:10029000CAB90C9422B70C9440ED0C9447B70C9457
:1002A000564F0C9412E70C94DB310C9478FA0C94B2
:1002B0006D1F0C94C72E0C9491ED0C94D0B90C9436
:1002C0002D290C9468FA0C9407E70C94E9B90C9466
:1002D000B9ED0C946DB60C942D280C94FC2F0C9455
:1002E000DEB90C94C6B90C9434FA0C948A300C9490
:1002F000874F0C9403E70C942EE70C9448B60C94AB
:1003000098320C946CFA0C944C1F0C9492B60C948A
:1003100091FA0C9409300C942CED0D94361A0C942F
:1003200060290C94B5B90C94D8B60C94794F0C9400
:10033000542E0C9434E70C94A5ED0C9482ED0D949E
:10034000BF1A0C941CE70C94DBB70C9478ED0C945A
:10035000D91E0C940C500C94621F0C94E4B90C94AC
:10036000BD340C94DAB90C94CDB90C94D62F0C94FE
:100370006EED0C94F9E60C94B5B60C94BF4F0C944A
:10038000EF2F0C947B2A0C948EFA0C942AE70C9491
:100390005CFA0C94D4B90C94EB2E0C9470FA0C9477
:1003A00065320C94E1B90C946CB70C9423B60C94A0
:1003B000C22F0C94A32E0C9418E70C943CE70C94D9
:1003C0009B2E0C9464ED0C940AE70C9451280C9429
:1003D0005CED0C9436ED0C9431270C94284F0C9462
:1003E0001E2B0C94BCB90C9420E70C9431ED0C94AA
:1003F0008C2E0C9441E70C9464FA0C949BED0C94B5
:10040000B9B90C9491B70C940EE70C9414330C9476
:10041000BFB90C9438E70C94B2B90C94AFED0C94BE
:10042000BB2C0C944AED0C94D7B90C9454ED0C945D
:10043000FDE64E414E494E495459494E46CDCCCC2D
:100440003D0AD7233C17B7D13877CC2B329595E6A8
:10045000241FB14F0A000020410000C84200401C88
:100460004620BCBE4CCA1B0E5AAEC59D7400407AD5
:1004700010F35A00A0724E18090010A5D4E800002D
:10048000E87648170000E40B54020000CA9A3B00CB
:100490000000E1F505000080969800000040420F42
:1004A000000000A08601000000102700000000E806
:1004B00003000000006400000000000A00000000CB
:1004C000000100000000002C76D888DC674F08236C
:1004D000DFC1DFAE59E1B1B796E5E3E453C63AE6D2
:1004E00051997696E8E6C28426EB898C9B62ED40B2
:1004F0007C6FFCEFBC9C9F40F2BAA56FA5F4900501
:100500005A2AF75C936B6CF9676DC11BFCE0E40D34
:1005100047FEF520E6B500D0ED902E030094357728
:10052000050080841E080000204E0A000000C80C50
:10053000333333330F986E12831141EF8D211489B9
:100540003BE65516CFFEE6DB18D1844B381BF77C13
:100550001D901DA4BBE424203284725E228100C958
:10056000F124ECA1E53D274D323520500A4D3234BF
:10057000005072696E742050617573656400526535
:1005800073756D65005549205061757365004E6F38
:10059000204D61746368203A004D333033452D316E
:1005A000533635433455004D393939004D353032E5
:1005B0000A4D353030004D3330334530533231350C
:1005C000433855000A202A2A2A7265636461742E12
:1005D000646174615B305D203D004732380A473109
:1005E000204631303030205A313000556E737570EE
:1005F000706F72746564204F7074696F6E205365FC
:100600006C6563746564004D3139305335350A4784
:1006100032380A4732390A4D3430300A4D313034DD
:10062000533231350A4732380A4D3130395332317D
:10063000350A4D34323053310A4731583130305950
:1006400031303046353030300A47315A300A4D3576
:1006500030300A4D31313720536574205A204F66AF
:1006600066736574004731204631303030205A308F
:100670002E30004732380A473120463130303020A2
:100680005A302E30004D353030005A204F66667398
:100690006574203A202573004D353030005A204FC4
:1006A0006666736574203A202573004732385A0A0B
:1006B000473146313530305A302E30004732380A13
:1006C000473146313530305A302E30004D38340005
:1006D000473146313030305A302E30004732380AF8
:1006E000473146313030305A302E30005A204F6674
:1006F00066736574203A202573004D353030004D07
:10070000383400426567696E5377697463680072B4
:1007100065636461742E61646472203D3D0072659E
:10072000636461742E646174615B305D203D3D00E3
:1007300077616974776179203D3D000A202A2A2A71
:100740004E6F7A7A6C6554656D705374617475730D
:100750005B325D203D00434F4D4D554E4943415462
:10076000494F4E0044525952554E004552524F5235
:100770005300494E464F004543484F0047322F47EC
:10078000332062616420706172616D65746572739B
:100790000A00536C6565702E2E2E00486F6D652023
:1007A00058592046697273740A00486F6D65205865
:1007B00059204669727374004D3131372050726F81
:1007C0006265206661696C65642E0A4732380A00EA
:1007D00070726F62655F7265776970650047323964
:1007E000205265747279696E670050726F62696E2B
:1007F00067204661696C6564004D31313720426580
:1008000064206C6576656C696E67206661696C65ED
:10081000642E0A4730205A31300A4D333030205090
:10082000323520533838300A4D333030205035308F
:100830002053300A4D333030205032352053383871
:10084000300A4D333030205035302053300A4D338C
:1008500030302050323520533838300A4D33303064
:10086000205035302053300A473420533100707205
:100870006F62655F6661696C6564004D3131372078
:10088000426564206C6576656C696E6720646F6E86
:10089000652E00205A3A200020593A200042656413
:1008A00020583A20004D65736820706F696E74207F
:1008B00063616E6E6F74206265207265736F6C7613
:1008C00065640A004D302F3120427265616B204310
:1008D000616C6C656400436F6E74696E7565004D84
:1008E000302F3120427265616B2043616C6C65640E
:1008F000004E6F204D6F76652E00456E6420666950
:100900006C65206C6973740A00426567696E2066C5
:10091000696C65206C6973740A00526573756D6546
:1009200020534400286E6F2066696C65290043756A
:100930007272656E742066696C653A20002E0A003A
:1009400044656C6574696F6E206661696C65642CC2
:100950002046696C653A200046696C652064656CC8
:10096000657465643A005072696E742074696D65CF
:100970003A20000A53746174733A2046696C616DC1
:10098000656E7420757365643A20002C204C6F6E80
:1009900067657374206A6F623A2000546F74616CEB
:1009A0002074696D653A200053746174733A2000B5
:1009B0002C204661696C65643A20002C2046696EE3
:1009C00069736865643A20005072696E74733A20E6
:1009D0000053746174733A20004520436F6F6C6953
:1009E0006E672E2E2E00452048656174696E672E55
:1009F0002E2E006F666600770772076B0764075636
:100A00000744454255473A004D31313320530042A7
:100A1000656420436F6F6C696E672E2E2E004265F1
:100A2000642048656174696E672E2E2E006F6B001E
:100A30004348414D4245525F54454D504552415403
:100A4000555245004D4F54494F4E5F4D4F4445530D
:100A500000544845524D414C5F50524F5445435409
:100A6000494F4E004155544F5245504F52545F53D9
:100A7000445F5354415455530050524F4D50545FAE
:100A8000535550504F525400454D455247454E43E3
:100A9000595F50415253455200434153455F4C49C1
:100AA0004748545F4252494748544E4553530054B7
:100AB0004F47474C455F4C494748545300534F46B6
:100AC00054574152455F504F574552004255494C8B
:100AD000445F50455243454E54004C4556454C49A1
:100AE0004E475F44415441005A5F50524F424500C7
:100AF0004155544F4C4556454C005052494E545F59
:100B00004A4F420050524F475245535300415554AB
:100B10004F5245504F52545F54454D5000564F4C24
:100B2000554D455452494300454550524F4D0042A2
:100B3000494E4152595F46494C455F5452414E53CC
:100B40004645520053455249414C5F584F4E5F58FD
:100B50004F4646004649524D574152455F4E414D22
:100B6000453A4D61726C696E20322E305F445732C7
:100B700020544D334420453550534D444242205378
:100B80004F555243455F434F44455F55524C3A6879
:100B9000747470733A2F2F6769746875622E636F6F
:100BA0006D2F496E73616E6974794175746F6D61F3
:100BB00074696F6E2F4D61726C696E2F747265650A
:100BC0002F437265616C6974795F4D61726C696EF7
:100BD000322E302E782050524F544F434F4C5F5698
:100BE000455253494F4E3A312E30204D41434849EA
:100BF0004E455F545950453A544D334420453520B5
:100C0000506C75732045585452554445525F434FBC
:100C1000554E543A3120555549443A63656465321E
:100C20006132662D343161322D343734382D3962DA
:100C300031322D6335356336326633363766660AB0
:100C4000002F2F200020466C6F773A200050726FE3
:100C50007465637465642050696E0A00206F757452
:100C6000206F662072616E67650A00536572766F49
:100C700020003A200020536572766F200050726F7A
:100C80006265205A204F66667365743A2000496E8B
:100C900076616C69642065787472756465720A00A7
:100CA00020643A0020693A0020703A0020643A003B
:100CB00020693A0020703A0064697300656E004351
:100CC000290A0061626C656420286D696E20746574
:100CD0006D702000436F6C64206578747275646574
:100CE000732061726520004F4646004F4E004669F2
:100CF0006C616D656E742072756E6F7574206469B9
:100D00007374616E636520286D6D293A2000466911
:100D10006C616D656E742072756E6F757420004D18
:100D200065736820706F696E742063616E6E6F7496
:100D3000206265207265736F6C7665640A004D34BD
:100D4000323120696E636F727265637420706172F4
:100D5000616D657465722075736167650A004F6621
:100D60006673657473204170706C696564004572C8
:100D7000723A20546F6F206661722100546F6F20A9
:100D80006661722066726F6D207265666572656E4F
:100D9000636520706F696E740A00454550524F4D6F
:100DA000204F4B0A003F5A206F7574206F662072E7
:100DB000616E676520282D323020746F2032302913
:100DC0000A0050726F6265205A204F666673657420
:100DD0003A20003F4B2076616C7565206F7574205A
:100DE0006F662072616E67652028302D3130292EA4
:100DF0000A00416476616E6365204B3D00202050FF
:100E00006C616E6E65724275666665724279746574
:100E1000733A20002046726565204D656D6F7279CA
:100E20003A2000436F6D70696C65643A20536570B9
:100E300020203720323031390A00207C204175745F
:100E4000686F723A2054696E794D616368696E65A6
:100E50007333440A00323031392D30372D333000AE
:100E6000204C61737420557064617465643A20008D
:100E7000322E305F4457320A004D61726C696E0049
:100E800020536F6674776172652052657365740ACA
:100E900000205761746368646F67205265736574DE
:100EA0000A002042726F776E206F7574205265734E
:100EB00065740A002045787465726E616C20526515
:100EC0007365740A00506F77657255700A00737409
:100ED0006172740A006175746F25632E6700657214
:100EE000726F722077726974696E6720746F206602
:100EF000696C650A00446F6E6520736176696E6780
:100F00002066696C652E0A004D323900205A3A007D
:100F100020593A0020583A00656E6473746F7073FC
:100F2000206869743A200047323858590043616E8E
:100F30006E6F74206F70656E2073756264697220C5
:100F40000053442063617264206F6B0A006F706508
:100F50006E526F6F74206661696C65640A00766F0B
:100F60006C756D652E696E6974206661696C656467
:100F70000A00534420696E6974206661696C0A0036
:100F80004D3234004D323320257300577269746935
:100F90006E6720746F2066696C653A20002E0A0027
:100FA0006F70656E206661696C65642C2046696CA3
:100FB000653A20002E0A006F70656E206661696CCC
:100FC00065642C2046696C653A200046696C652092
:100FD00073656C65637465640A002053697A653AC9
:100FE000200046696C65206F70656E65643A20006C
:100FF000667265736800646F696E67002066696C6D
:10100000653A20004E6F772000454E4420535542EC
:10101000524F5554494E450A002220706F730022EA
:1010200020706172656E743A2200535542524F55DA
:1010300054494E452043414C4C207461726765749D
:101040003A2200747279696E6720746F2063616C54
:101050006C207375622D67636F64652066696C65CB
:1010600073207769746820746F6F206D616E7920CA
:101070006C6576656C732E204D4158206C657665E5
:101080006C2069733A310A005344207072696E749F
:10109000696E67206279746520004E6F7420534436
:1010A000207072696E74696E670A00627573793AAE
:1010B0002070617573656420666F7220696E70754B
:1010C000740A00627573793A2070617573656420E3
:1010D000666F7220757365720A00627573793A20C3
:1010E00070726F63657373696E670A007061757300
:1010F00065004D363030200A204D313137200A004E
:101100002066696C616D656E745F72756E6F757463
:10111000200066696C616D656E745F72756E6F75C7
:101120007420540046696C616D656E7452756E6F03
:1011300075742054004B494C4C2063617573656491
:1011400020627920746F6F206D75636820696E610D
:1011500063746976652074696D65202D20637572EE
:1011600072656E7420636F6D6D616E643A200070FD
:101170006F7765726F6666004B494C4C45442E2074
:10118000005072696E7465722068616C7465642EBB
:10119000206B696C6C28292063616C6C6564210A82
:1011A0000053544F505045442E20005072696E74C5
:1011B00065722073746F7070656420647565207447
:1011C0006F206572726F72732E2046697820746882
:1011D00065206572726F7220616E64207573652080
:1011E0004D39393920746F20726573746172742EB1
:1011F000202854656D70657261747572652069731D
:101200002072657365742E205365742069742061A3
:10121000667465722072657374617274696E672991
:101220000A006563686F3A004572726F723A004255
:10123000696C696E656172204C6576656C696E6774
:1012400020477269643A0A0057616974696E6720C1
:10125000666F72206865617475702E0A004C656156
:1012600076696E6720473236003F53706563696662
:1012700069656420582C5920636F6F7264696E61D0
:101280007465206F7574206F6620626F756E64736D
:101290002E0A003F28522965706561742076616CC2
:1012A0007565206E6F7420706C61757369626C6512
:1012B0003B206D757374206265206174206C6561DC
:1012C000737420312E0A003F2852296570656174BD
:1012D000206D75737420626520737065636966693B
:1012E0006564207768656E206E6F74207573696E13
:1012F0006720616E204C43442E0A003F53706563A3
:101300006966696564206E6F7A7A6C652074656DB4
:101310007065726174757265206E6F7420706C6197
:10132000757369626C652E0A003F53706563696668
:101330006965642066696C616D656E742073697A95
:1013400065206E6F7420706C61757369626C652EB8
:101350000A003F537065636966696564207072694D
:101360006D65206C656E677468206E6F7420706C9C
:1013700061757369626C652E0A003F5072696D6514
:10138000206C656E677468206D75737420626520CB
:10139000737065636966696564207768656E206E41
:1013A0006F74207573696E6720616E204C43442E04
:1013B0000A003F537065636966696564206E6F7AE1
:1013C0007A6C652073697A65206E6F7420706C6129
:1013D000757369626C652E0A003F526574726163B1
:1013E00074696F6E204D756C7469706C69657220DC
:1013F0006D757374206265207370656369666965D5
:10140000642E0A003F537065636966696564205203
:10141000657472616374696F6E204D756C74697068
:101420006C696572206E6F7420706C61757369628F
:101430006C652E0A003F53706563696669656420B8
:101440006C6179657220686569676874206E6F7475
:1014500020706C61757369626C652E0A0043292ED9
:101460000A003F537065636966696564206265645C
:101470002074656D7065726174757265206E6F742D
:1014800020706C61757369626C65202834302D00A2
:10149000473236207374617274696E672E2E2E0A7D
:1014A000004F46460A0046616465204865696768E2
:1014B000742000426564204C6576656C696E672017
:1014C000004661696C656420746F20656E61626CB2
:1014D0006520426564204C6576656C696E670A001C
:1014E000496E76616C6964206D6573682E0A002907
:1014F0000A002062797465733B2063726320005395
:10150000657474696E67732053746F726564202804
:1015100000454550524F4D206461746173697A658E
:10152000206572726F722E0A00290A002062797497
:1015300065733B2063726320002073746F7265646F
:101540002073657474696E6773207265747269655F
:10155000766564202800202863616C63756C617473
:10156000656429210A0020213D2000454550524F45
:101570004D20435243206D69736D61746368202D63
:10158000202873746F7265642920002053697A657E
:101590003A2000496E6465783A2000204D61726CF3
:1015A000696E3D563638290A00454550524F4D2048
:1015B00076657273696F6E206D69736D61746368AF
:1015C0002028454550524F4D3D00496E76616C696B
:1015D000642065787472756465720A007C3C3E5EB6
:1015E0002B3D3F2F5B5D3B2C2A225C004D31313778
:1015F000004D33310053442072656164206572727E
:101600006F720A00446F6E65207072696E74696E45
:10161000672066696C650A0043616E6E6F74206FA7
:1016200070656E20737562646972200025697300AD
:1016300025696D20256973002569682025696D205D
:1016400025697300256964202569682025696D2056
:10165000256973002569792025696420256968203A
:1016600025696D202569730023646566696E6520B0
:1016700044454641554C545F0000626564004B642C
:1016800020004B6920004B702000504944204175D8
:10169000746F74756E652066696E69736865642120
:1016A0002050757420746865206C617374204B70D1
:1016B0002C204B6920616E64204B6420636F6E7335
:1016C00074616E74732066726F6D2062656C6F77E3
:1016D00020696E746F20436F6E66696775726174FE
:1016E000696F6E2E680A00504944204175746F740A
:1016F000756E65206661696C6564212074696D652D
:101700006F75740A00453120544845524D414C20B4
:1017100052554E4157415900424544205448455284
:101720004D414C2052554E41574159005468657205
:101730006D616C2052756E6177617900453120488A
:10174000656174696E67204661696C656400426515
:10175000642048656174696E67204661696C6564E0
:101760000048656174696E67206661696C65640034
:10177000504944204175746F74756E6520666169C7
:101780006C6564212054656D706572617475726555
:1017900020746F6F20686967680A00204B643A20E4
:1017A00000204B693A2000204B703A20000A204369
:1017B0006C617373696320504944200A00204B64B4
:1017C0003A2000204B693A2000204B703A20000A52
:1017D000204E6F206F76657273686F6F740A0020F9
:1017E00054753A2000204B753A2000206D61783AFC
:1017F0002000206D696E3A200020643A20002062AB
:101800006961733A2000504944204175746F7475C2
:101810006E652073746172740A00504944204175EA
:10182000746F74756E65206661696C6564212054FF
:10183000656D706572617475726520746F6F206874
:101840006967680A00504944204175746F74756E69
:1018500065206661696C6564212042616420657859
:10186000747275646572206E756D6265720A00220D
:101870000A00556E6B6E6F776E20636F6D6D616ED3
:10188000643A20220020746F6F206C6F6E672065B1
:101890007874727573696F6E2070726576656E7498
:1018A00065640A0020636F6C6420657874727573D8
:1018B000696F6E2070726576656E7465640A0024C7
:1018C000F4D43050C38E20C2A24017828B70111204
:1018D0007A910D816CD90AA861E108C75866076141
:1018E0005143061E4B5D05C145A7041A4111040969
:1018F0003D9803713931034036DB0265339102D4E0
:10190000305402802E1D02632CEE01752AC501B0F1
:1019100028A001102781018F2564012B244B01E0B1
:10192000223401AC211F018D200D01801FFC008499
:101930001EED00971DDF00B81CD200E61BC600207C
:101940001BBC00641AB200B219A8000A19A0006AF0
:10195000189900D117910040178B00B516840031FB
:10196000167E00B31579003A157300C7146F00583E
:10197000146A00EE1366008813630025135E00C727
:10198000125B006C12570015125400C11151007007
:10199000114F0021114B00D61049008D1047004611
:1019A00010440002104200C00F4000800F3E004271
:1019B0000F3C00060F3B00CB0E3800930E37005C47
:1019C0000E3500270E3400F30D3200C10D310090AA
:1019D0000D3000600D2E00320D2D00050D2C00D9AC
:1019E0000C2B00AE0C2900850C29005C0C2700355F
:1019F0000C27000E0C2600E80B2400C40B2400A0CA
:101A00000B23007D0B23005A0B2100390B210018FA
:101A10000B2000F80A1F00D90A1E00BB0A1E009DF9
:101A20000A1D00800A1D00630A1C00470A1B002CC7
:101A30000A1B00110A1A00F7091A00DD091900C46F
:101A4000091900AB091900920917007B09180063F6
:101A50000917004C09160036091600200916000A5D
:101A6000091500F5081500E0081400CC081400B8AA
:101A7000081400A4081400900813007D0812006BDD
:101A800008130058081200460812003408110023F9
:101A90000811001208110001081100F0071000E001
:101AA000071000D0071000C0071000B0070F00A1FA
:101AB00007100091070E0083070F0074070F0065E1
:101AC000070E0057070E0049070E003B070D002EBA
:101AD000070E0020070D0013070D0006070D00F983
:101AE000060C00ED060D00E0060C00D4060C00C844
:101AF000060C00BC060C00B0060C00A4060B0099F6
:101B0000060C008D060B0082060B0077060B006C9E
:101B1000060B0061060A0057060B004C060A00423D
:101B2000060A0038060A002E060A0024060A001AD1
:101B3000060A001006090007060A00FD050900F460
:101B4000050900EB050900E2050900D9050900D0E7
:101B5000050900C7050900BE050900B5050800AD67
:101B6000050800A50509009C050800940508008CDF
:101B7000050800840508007C050800740508006C51
:101B8000050700650508005D050700560508004EBD
:101B90000507004705070040050800380507003124
:101BA0000507002A050700230507001C0506001687
:101BB0000507000F0507000805060002050700FBE2
:101BC000040600F5040700EE040600E8040600E23F
:101BD000040700DB040600D5040600CF040600C994
:101BE000040600C3040600BD040600B7040600B1E5
:101BF000040500AC040600A6040600A00405009B32
:101C000004060095040500900406008A040500857A
:101C1000040500800406007A0405007504050070C0
:101C20000405006B04050066040500610405005C02
:101C300004050057040500520405004D0405004842
:101C4000040500430405003E0404003A0405003581
:101C5000040500300404002C0405002704040023BC
:101C60000405001E0404001A0404001604050011F3
:101C70000404000D04040009040500040404000029
:101C8000040400FC030400F8030400F4030400F05F
:101C9000030400EC030400E8030400E4030400E090
:101CA000030400DC030400D8030400D4030400D0C0
:101CB000030400CC030400C8030300C5030300248D
:101CC000F404D9201BC40C5C0E9804C4095F02659F
:101CD000077101F405F900FB04B30048048700C153
:101CE0000369005803550003034500BE023A00840F
:101CF00002310053022A002902250004022000E4D8
:101D0000011C00C8011900AF0117009801140084DC
:101D1000011300710110006101100051010E004318
:101D2000010D0036010B002B010B0020010B0015EB
:101D30000109000C01090003010800FB000800F381
:101D4000000800EB000700E4000600DE000600D8F3
:101D5000000600D2000600CC000500C7000500C246
:101D6000000500BD000400B9000400B5000400B186
:101D7000000400AD000400A9000400A5000300A2B7
:101D80000003009F0004009B0003009800030095DF
:101D900000020093000300900003008D0002008BFE
:101DA0000003008800020086000200840003008116
:101DB0000002007F0002007D0002007B000200792B
:101DC0000002007700010076000200740002007239
:101DD000000100710002006F0002006D0001006C44
:101DE0000002006A0001006900020067000100664D
:101DF0000001006500010064000200620001006152
:101E0000000100600001005F0002005D0001005C55
:101E10000001005B0001005A000100590001005858
:101E20000001005700010056000100550001005458
:101E30000001005300000053000100520001005156
:101E4000000100500001004F0001004E0000004E54
:101E50000001004D0001004C0001004B0000004B50
:101E60000001004A0001004900010048000000484C
:101E70000001004700010046000000460001004547
:101E80000000004500010044000100430000004341
:101E9000000100420000004200010041000000413A
:101EA000000100400001003F0000003F0001003E33
:101EB0000000003E0001003D0000003D0001003C2C
:101EC0000000003C0000003C0001003B0000003B23
:101ED0000001003A0000003A00010039000000391A
:101EE0000001003800000038000000380001003711
:101EF0000000003700010036000000360000003608
:101F000000010035000000350000003500010034FC
:101F100000000034000000340001003300000033F2
:101F200000000033000100320000003200000032E7
:101F300000010031000000310000003100010030DC
:101F400000000030000000300001002F0000002FD2
:101F50000000002F0000002F0001002E0000002EC6
:101F60000000002E0001002D0000002D0000002DBB
:101F70000000002D0001002C0000002C0000002CAF
:101F80000000002C0001002B0000002B0000002BA3
:101F90000000002B0001002A0000002A0000002A97
:101FA0000000002A0001002900000029000000298B
:101FB000000000290000002900010028000000287E
:101FC0000000002800000028000000280001002771
:101FD0000000002700000027000000270000002765
:101FE0000001002600000026000000260000002658
:101FF000000000260001002500000025000000254B
:10200000000000250000002500000025000100243C
:102010000000002400000024000000240000002430
:102020000001002300000023000000230000002323
:102030000000002300000023000000230001002214
:102040000000002200000022000000220000002208
:1020500000000022000100210000002100000021FA
:1020600000000021000000210000002100000021EC
:1020700000010020000000200000002000000020DF
:1020800000000020000000200000002000000020D0
:102090000001001F0000001F0000001F0000001FC3
:1020A0000000001F0000001F0000001F0001001EB4
:1020B0000000001E0000001E0000001E000000C204
:1020C0003100001C260000F4190000D80F0000EBBE
:1020D000080000C004000075020000400100004D2F
:1020E000323830205030205339300050726F6269DE
:1020F0006E6720506F696E742025692F2569002E48
:102100000A002F0050726F62696E67206D657368F8
:1021100020706F696E742000202844525952554E29
:102120002900473239204175746F20426564204C84
:102130006576656C696E67003F20284C2C522C46F2
:102140002C4229206F7574206F6620626F756E6453
:10215000732E0A003F2856296572626F7365206CE2
:102160006576656C20697320696D706C6175736943
:10217000626C652028302D34292E0A0042616420CB
:102180005A2076616C75650A004E6F2062696C6931
:102190006E65617220677269640A0046696E6973D0
:1021A000686564210A00206F662000205A002059CB
:1021B00000476F696E6720746F3A20580043570AD2
:1021C00000206469723A0020616E676C653A0053C2
:1021D00074617274207261646975733A00506F7330
:1021E0006974696F6E696E67207468652070726FBC
:1021F00062652E2E2E0A003F4E756D626572206F4D
:1022000066206C65677320696E206D6F76656D65FD
:102210006E74206E6F7420706C61757369626C658A
:102220002028302D3135292E0A003F2028582C59DE
:1022300029206F7574206F6620626F756E64732E2F
:102240000A003F53616D706C652073697A65206E7A
:102250006F7420706C61757369626C652028342D11
:102260003530292E0A004D3438205A2D50726F62B5
:1022700065205265706561746162696C697479206A
:10228000546573740A003F2856296572626F73653E
:10229000206C6576656C20697320696D706C617562
:1022A0007369626C652028302D34292E0A005A5F2C
:1022B00053544F505F50494E005A5F535445505F3E
:1022C00050494E005A5F4D494E5F50494E005A5F8B
:1022D000454E41424C455F50494E005A5F44495279
:1022E0005F50494E005A5F43535F50494E00595F5B
:1022F00053544F505F50494E00595F535445505FFF
:1023000050494E00595F4D41585F50494E00595F4A
:10231000454E41424C455F50494E00595F44495239
:102320005F50494E00595F43535F50494E00585F1C
:1023300053544F505F50494E00585F535445505FBF
:1023400050494E00585F4D41585F50494E00585F0C
:10235000454E41424C455F50494E00585F444952FA
:102360005F50494E00585F43535F50494E005353EE
:102370005F50494E00534552564F335F50494E000F
:10238000534552564F325F50494E00534552564FB7
:10239000315F50494E00534552564F305F50494EC1
:1023A00000534453530053445F4445544543545FE2
:1023B00050494E0053434B5F50494E0052414D50DF
:1023C000535F44395F50494E0052414D50535F4472
:1023D000385F50494E0052414D50535F4431305F99
:1023E00050494E004D4F53495F50494E004D4F5399
:1023F0004645545F445F50494E004D49534F5F502E
:10240000494E004D4158363637355F53535F50497A
:102410004E004C45445F50494E004845415445529A
:102420005F4245445F50494E004845415445525F24
:10243000305F50494E0046494C5F52554E4F5554FF
:102440005F50494E0046414E315F50494E00464173
:102450004E5F50494E0045315F535445505F5049DF
:102460004E0045315F454E41424C455F50494E005C
:1024700045315F4449525F50494E0045315F4353F7
:102480005F50494E0045305F535445505F50494EB0
:102490000045305F454E41424C455F50494E004536
:1024A000305F4449525F50494E0045305F43535FAF
:1024B00050494E00455F4D5558325F50494E0045DA
:1024C0005F4D5558315F50494E00455F4D5558306E
:1024D0005F50494E004156525F53535F50494E0082
:1024E0004156525F53434B5F50494E004156525F35
:1024F0004D4F53495F50494E004156525F4D49532D
:102500004F5F50494E0054454D505F4245445F5027
:10251000494E0054454D505F315F50494E0054457F
:102520004D505F305F50494E0046494C5749445426
:10253000485F50494E0054584400525844002054BB
:1025400000205200416363656C65726174696F6E4F
:102550003A2050003F4A206F7574206F66207261E8
:102560006E67652028302E303120746F20302E3376
:10257000290A0050574D3A20202534640050574D09
:102580003A20202534640050574D3A2020253464E9
:102590000050574D3A20202534640050574D3A20C2
:1025A000202534640050574D3A20202534640050D3
:1025B000574D3A20202534640050574D3A202025AD
:1025C00034640050574D3A20202534640050574D54
:1025D0003A20202534640050574D3A202025346499
:1025E0000050574D3A20202534640050574D3A2072
:1025F000202534640050574D3A2020253464005083
:10260000574D3A20202534640050574D3A2020255C
:10261000346400433A2000423A2000413A2000202E
:10262000202020434F4D002020206E6F6E2D7374AC
:10263000616E646172642050574D206D6F64650057
:10264000202020636F6D7061726520696E74657201
:102650007275707420656E61626C65640020202064
:102660006F766572666C6F7720696E7465727275CD
:10267000707420656E61626C6564003A20002020F1
:10268000202054494D534B00423A20002020202066
:102690005443435200413A20002020202054434319
:1026A00052002020202043533A2000202020205791
:1026B000474D3A200050574D3A20202534640050B1
:1026C000574D3A2020253464004700480000008818
:1026D000008A008C00B300B400000098009A009CAF
:1026E00000A800AA00AC0028012A012C012020200B
:1026F0002054494D455200440045006E0080008141
:10270000006F00B000B1007000900091007100A057
:1027100000A1007200200121017300206973206173
:102720006C736F207469656420746F2074686973BA
:102730002070696E0054494D45523143000A202EE5
:10274000002020002020506F72743A2000202020AA
:1027500000202020416E616C6F6720696E203D2053
:1027600025356C64003C756E757365642F756E6BF2
:102770006E6F776E3E0020284125326429202000AC
:102780002533642000257350494E3A20004F75745C
:10279000707574203D2000496E70757420203D20B6
:1027A00000416E616C6F6720696E203D2025356C9D
:1027B000640070726F746563746564200020284142
:1027C00025326429202000253364200025735049D8
:1027D0004E3A20003A2500013625010129253B000B
:1027E0001E2543001325450006254400F924320127
:1027F000EC243301E0243401D5243501CA24280116
:10280000BF242A01B4242C01AA242A019F241C01DC
:102810009124180185241A017B242C0170242201A3
:1028200062241E01562424014E2409014524070177
:102830003624020129240A011A24080112240D0158
:1028400003244201FA233201ED230701E42333017B
:10285000D6230A01C9230801BC230901B42334018A
:10286000A6233101A123350196230B018B230601F9
:1028700080230501752304016E233501652335018D
:102880005B2337014E2326014423030139233601FC
:102890002E230301252331011B233D010E23380183
:1028A00004230E01F9223C01EE220E01E52228014B
:1028B000DB223001CE223E01C4221201B9222E01B8
:1028C000AE2212014361703A00220A00656E7175F2
:1028D000657565696E672022002042002050006FF8
:1028E0006B00526573656E643A200053544F50502C
:1028F00045442E20005072696E7465722073746FA7
:10290000707065642064756520746F206572726FE5
:1029100072732E2046697820746865206572726F24
:102920007220616E6420757365204D3939392074C9
:102930006F20726573746172742E202854656D70F7
:102940006572617475726520697320726573657450
:102950002E2053657420697420616674657220723C
:10296000657374617274696E67290A004E6F204343
:102970006865636B73756D2077697468206C696E28
:1029800065206E756D6265722C204C617374204CED
:10299000696E653A20004E6F20436865636B7375FE
:1029A0006D2077697468206C696E65206E756D6244
:1029B00065722C204C617374204C696E653A20005E
:1029C000636865636B73756D206D69736D617463A6
:1029D000682C204C617374204C696E653A20004C61
:1029E000696E65204E756D626572206973206E6F29
:1029F00074204C617374204C696E65204E756D6255
:102A000065722B312C204C617374204C696E653AD1
:102A100020004D31313000776169740A000000B444
:102A2000430000B44300000000000048420000489A
:102A300042000080405761726E696E673A20486FAD
:102A40006D696E672042756D702044697669736F99
:102A500072203C20310A000202040000A040000065
:102A6000A040000000400000B4430000B443000058
:102A7000C8430101FF53544F502063616C6C65647F
:102A80002062656361757365206F6620424C546FE8
:102A9000756368206572726F72202D207265737481
:102AA0006172742077697468204D3939390A00538E
:102AB000544F502063616C6C65642062656361757E
:102AC0007365206F6620424C546F75636820657291
:102AD000726F72202D207265737461727420776931
:102AE0007468204D3939390A002F2F616374696F7A
:102AF0006E3A00627574746F6E00656E6400707279
:102B00006F6D70745F0073686F77004D38373620D3
:102B1000526573706F6E64696E672050524F4D50EE
:102B2000545F00554E4B4E4F574E20535441544521
:102B30000047434F44455F494E464F004C43445F76
:102B400050415553455F524553554D450046494CFC
:102B5000414D454E545F52554E4F55545F434F4E75
:102B600054494E55450046494C414D454E545F52DF
:102B7000554E4F5554004D323400436F6E74696E9C
:102B800075650044697361626C6552756E6F75742A
:102B9000005075726765204D6F72650050617573E6
:102BA00065640070617573656400486F74656E6478
:102BB00020746F6F20636F6C640A005061757365D9
:102BC00000507265737320627574746F6E20286F85
:102BD00072204D3130382920746F20726573756D05
:102BE000650A00496E736572742066696C616D6573
:102BF0006E7420616E6420707265737320627574E8
:102C0000746F6E20286F72204D313038290A0043CE
:102C10006F6E74696E7565005265686561742044F5
:102C20006F6E6500526568656174696E672E2E2E41
:102C300000526568656174696E6700486561746516
:102C40007254696D656F75740052656865617400D2
:102C500048656174657254696D656F757400507272
:102C600065737320627574746F6E20286F72204DC7
:102C70003130382920746F2068656174206E6F7A56
:102C80007A6C650A004E6F7A7A6C65205061726BBF
:102C9000656400436F6E74696E7565004E6F7A7A75
:102CA0006C65205061726B656400486F74656E647A
:102CB00020746F6F20636F6C640A00726573756DAA
:102CC000656400626567696E00436F6E74696E7556
:102CD000650044697361626C6552756E6F7574004E
:102CE00050757267654D6F726500506175736564EC
:102CF000004C6F61642046696C616D656E740043C1
:102D00006F6E74696E7565004C6F61642046696C06
:102D1000616D656E74205400496E7365727420662F
:102D2000696C616D656E7420616E6420707265738C
:102D30007320627574746F6E20286F72204D31306D
:102D400038290A00526573756D650070012C019079
:102D5000012701B0012201C0011D01F0011801107D
:102D600002130130020E016002090190020401C049
:102D700002FF000003FA004003F5008003F000D0DA
:102D800003EB002004E6007004E100E004DC0040F6
:102D900005D700C005D2004006CD00D006C800808F
:102DA00007C3003008BE00F008B900C009B400B085
:102DB0000AAF00B00BAA00D00CA500000EA0005076
:102DC0000F9B00C01096005012910000148C00C0A0
:102DD000158700B0178200B0197D00D01B78000065
:102DE0001E730040206E0090226900F024640040B1
:102DF000275F0090295A00E02B5500102E5000202C
:102E0000304B0010324600E033410090353C00105A
:102E100037370070383200A0392D00B03A2800A0B2
:102E20003B2300603C1E00103D1900903D14001033
:102E30003E0F00703E0A00C03E0500003F0000400B
:102E40003FFBFF803FF6FFC03FF1FF202D20496E82
:102E500076616C6964206578747275646572206E41
:102E6000756D62657220210A001000C90210012CE4
:102E7000014001220170011801B0010E01F00104AE
:102E8000015002FA00B002F0003003E600D003DC8B
:102E9000009004D2007005C800A006BE000008B46F
:102EA00000B009AA00D00BA000600E960060118C43
:102EB000000015820020197800C01D6E00A0226459
:102EC00000B0275A00902C500000314600E0343CFE
:102ED0000010383200903A2800603C1E00A03D14DB
:102EE00000803E0A00203F000045312054484552F2
:102EF0004D414C2052554E415741590042454420C6
:102F0000544845524D414C2052554E41574159006D
:102F1000546865726D616C2052756E6177617900DD
:102F20004531204572723A204D415854454D50006C
:102F30004572723A204D415854454D502042454407
:102F4000004D415854454D50207472696767657251
:102F50006564004531204572723A204D494E544512
:102F60004D50004572723A204D494E54454D502007
:102F7000424544004D494E54454D50207472696796
:102F80006765726564000A0A0020205A5F4D494E49
:102F90003A002020595F4D41583A002020585F4D9B
:102FA00041583A004D383420582059205A204500C5
:102FB000202F002042403A0020403A0020573A009B
:102FC00020573A00446F6E652E0A0066616C736587
:102FD000004641494C3A204E6F207472696767651C
:102FE000722064657465637465640A004641494CE7
:102FF0003A204E6F69736520646574656374656417
:10300000202D20706C656173652072652D72756E60
:1030100020746573740A0020646574656374656464
:103020002E0A003D20424C546F7563682070726513
:103030002056332E3120286F7220636F6D706174BB
:1030400069626C6529003D205A20536572766F20B5
:1030500050726F6265003D20424C546F756368206A
:1030600056332E310020282B2F2D20346D73293A12
:1030700020003A2033306D73206F72206D6F7265BF
:103080000A002E2050756C7365207769647468009F
:103090002A2A20506C6561736520747269676765C0
:1030A000722070726F62652077697468696E203370
:1030B0003020736563202A2A0A004641494C3A2091
:1030C000424C544F55434820656E61626C656420E4
:1030D0002D205365742075702074686973206465B1
:1030E00076696365206173206120536572766F2075
:1030F00050726F6265207769746820494E56455258
:1031000054494E472073657420746F20277472757C
:1031100065272E0A0020204445504C4F5945442035
:1031200073746174653A204C4F5720286C6F67693F
:10313000632030290020204445504C4F59454420FD
:1031400073746174653A204849474820286C6F675A
:103150006963203129003D204D656368616E6963B4
:10316000616C205377697463682064657465637467
:1031700065640A005741524E494E473A20494E561F
:10318000455254494E472073657474696E672070C8
:10319000726F6261626C79206261636B77617264E5
:1031A000732E0A002E204465706C6F7920262073E0
:1031B000746F7720342074696D65730A003D204276
:1031C0004C546F75636820436C617373696320317D
:1031D0002E322C20312E332C20536D61727420310D
:1031E0002E302C20322E302C20322E322C20332E1A
:1031F000302C20332E312064657465637465642E31
:103200000A002E20436865636B20666F7220424C73
:10321000544F5543480A002E205A5F4D494E5F4592
:103220004E4453544F505F494E56455254494E47B1
:103230003A20002E2050726F6265205A5F4D494E31
:103240005F50494E3A20002C2073746F7720616ED6
:10325000676C653A202020002C206465706C6F79C3
:1032600020616E676C653A2000536572766F20703E
:10327000726F626520746573740A2E207573696EAF
:103280006720696E6465783A2020004D34332057FA
:103290006169742043616C6C656400436F6E74698E
:1032A0006E7565004D343320576169742043616C3D
:1032B0006C6564005761746368696E672070696E3D
:1032C000730A0064697300656E0061626C65640A6C
:1032D00000656E6473746F70206D6F6E69746F72C9
:1032E0002000204500205A00205900204D3932206E
:1032F0005800205A00205900580020204D61783A8B
:103300002000205A00205900580020204D696E3AB4
:103310002000536F667420656E6473746F70733A27
:1033200020004732380020496E76616C6964206560
:1033300078747275646572200000002100240027F3
:10334000002A002D003000330001010000040107B5
:10335000010A0100002200250028002B002E003168
:1033600000340002010000050108010B01000020EB
:10337000002300260029002C002F0032000001004D
:1033800000030106010901050505050705080808F0
:1033900008020202020A0A080804040404010101E6
:1033A00001010101010303030303030303040707EE
:1033B000070C0C0C0C0C0C0C0C020202020606068C
:1033C00006060606060B0B0B0B0B0B0B0B01021074
:1033D000202008081020401020408002010201082F
:1033E00004020101020408102040808040201008DF
:1033F0000402018004020180402010080402010838
:103400000402010102040810204080010204081097
:1034100020408000000A0B02090C0D0E080703046F
:10342000010000000000000000000000000000009B
:10343000000000000000000000000000000000127A
:10344000111000000000000000000000000000005B
:1034500000000000000000000050726F62696E679B
:10346000204661696C65640A0050726F62696E671C
:10347000204661696C656400486F6D652025732581
:1034800073257320466972737400204669727374E1
:103490000A00486F6D6520006F70656E00545249D8
:1034A000474745524544003A200066696C616D65A6
:1034B0006E74007A5F6D696E00795F6D6178007877
:1034C0005F6D6178005265706F7274696E67206518
:1034D0006E6473746F70207374617475730A002066
:1034E0005A3A0020593A0020436F756E7420583ABA
:1034F0000020453A00205A3A0020593A00583A0034
:1035000020746F6F206C6F6E6720657874727573AE
:10351000696F6E2070726576656E7465640A00204E
:10352000636F6C6420657874727573696F6E207058
:10353000726576656E7465640A004572726F7220FA
:1035400077726974696E6720746F20454550524FD9
:103550004D210A00363726033C3D380E2E303E12F0
:103560001A1C1808440AFF4308090700010A2069C9
:103570006E6974207A70726F62655F7A6F666673C7
:103580006574203D2000454550524F4D20496E69DD
:103590007469616C697A65640A0048617264636F7A
:1035A0006465642044656661756C74205365747449
:1035B000696E6773204C6F616465640A00D0070010
:1035C00000D0070000640000004B00000000803BBA
:1035D0004400803B4400002041000096420000A0CF
:1035E000420000A042000048440000BE423A0A00E7
:1035F00020204D363033200020440020204D34312F
:103600003220530046696C616D656E742072756E70
:103610006F75742073656E736F723A0A00205500DF
:103620004C0046696C616D656E74206C6F61642F2F
:10363000756E6C6F6164206C656E677468733A0AAE
:103640000020204D393030204B004C696E6561728E
:1036500020416476616E63653A0A0020204D38355A
:1036600031205A005A2D50726F6265204F66667382
:1036700065740020440020490020204D3330342060
:10368000500020440020490020204D33303120508C
:10369000005049442073657474696E67733A0A0078
:1036A000204A0020204732392057204900205A0064
:1036B00020204D3432302053004175746F20426514
:1036C00064204C6576656C696E673A0A00205A0082
:1036D00020590020204D323036205800486F6D654B
:1036E000206F66667365743A0A00204A0020540011
:1036F00020530020204D323035204200204A3C6AC1
:10370000756E635F6465763E00416476616E6365E5
:10371000643A20423C6D696E5F7365676D656E74D7
:103720005F74696D655F75733E20533C6D696E5FB4
:1037300066656564726174653E20543C6D696E5FB8
:1037400074726176656C5F66656564726174653E0E
:103750000020540020520020204D323034205000F0
:10376000416363656C65726174696F6E2028756E64
:103770006974732F7332293A20503C7072696E74E9
:103780005F616363656C3E20523C72657472616375
:10379000745F616363656C3E20543C74726176654E
:1037A0006C5F616363656C3E0A00204500205A002F
:1037B00020590020204D3230312058004D61786969
:1037C0006D756D20416363656C65726174696F6EC0
:1037D0002028756E6974732F7332293A0A002045C8
:1037E00000205A0020590020204D3230332058004C
:1037F0004D6178696D756D2066656564726174658B
:10380000732028756E6974732F73293A0A005374F4
:103810006570732070657220756E69743A0A0020B5
:10382000204D3230302044300A0020204D323030DC
:103830002044002044697361626C65640A00466933
:103840006C616D656E742073657474696E67733A2C
:103850000020286D6D2900202047323120202020B3
:103860003B20556E69747320696E206D6D00486F42
:103870006D696E67204661696C6564002E0A006F91
:1038800070656E206661696C65642C2046696C65A4
:103890003A2000626564002C2073797374656D2092
:1038A00073746F7070656421204865617465725F20
:1038B00049443A20004265642048656174696E6736
:1038C000204661696C65640048656174696E6720B3
:1038D0006661696C65640042454420544845524D18
:1038E000414C2052554E4157415900546865726D04
:1038F000616C2052756E61776179004531204865B1
:103900006174696E67204661696C65640048656131
:1039100074696E67206661696C6564004531205486
:103920004845524D414C2052554E41574159005443
:103930006865726D616C2052756E617761790054B3
:103940004D334420453520506C75732052656164B9
:10395000792E005072696E74696E672E2E2E00509B
:1039600072696E74205061757365640063616E6383
:10397000656C005072696E742041626F7274656488
:103980000055492041626F727400726573756D65F0
:10399000004D3234000000B4430000B4430000C8BE
:1039A00043000000000000000000000000446966C1
:1039B0006665723A200046726F6D5374703A005318
:1039C0007465707065723A00556E4C6576656C3A38
:1039D000004C6576656C65643A005261773A202048
:1039E0002020000A4C6F676963616C3A00009F01F8
:1039F0008D0111241FBECFEFD1E2DEBFCDBF00E0AD
:103A00000CBF18E0A0E0B2E0E6E5F7E502E00BBF8E
:103A100002C007900D92AC3BB107D9F72EE1ACEB99
:103A2000B8E001C01D92AB38B207E1F71CE1C8EF66
:103A3000DCE100E006C021970109802FFE010F9410
:103A4000D427C73FD10780E00807A9F70F94741166
:103A50000D94992B0C9400002F923F924F925F92FD
:103A60006F927F928F929F92AF92BF92CF92DF928E
:103A7000EF92FF920F931F93CF93DF93CDB7DEB7F3
:103A8000E3970FB6F894DEBF0FBECDBF809109015A
:103A9000817091E098272091E208921781F190932C
:103AA000E208811116C00E94AF5180915B1883FF1C
:103AB00009C08FEB93E00E94D6F961E080E00F949B
:103AC0002E031DC060E081E00F942E0388ED93E08B
:103AD00014C000915B1803FB002700F90E943E51BF
:103AE00080915B18877F80935B18002341F060E032
:103AF00081E00F942E0381EF93E00E94D6F980912C
:103B0000BC0881FF11C180914D1690914E16891B02
:103B10008F70843008F008C18CE0E9EBF3E1DE013E
:103B2000119601900D928A95E1F78091770290911C
:103B30007802A0917902B0917A0288A799A7AAA7E2
:103B4000BBA79C01AD016091B9137091BA1380912C
:103B5000BB139091BC130F94DC276B017C01609325
:103B6000B9137093BA138093BB139093BC138091D5
:103B70007B0290917C02A0917D02B0917E028CA785
:103B80009DA7AEA7BFA79C01AD016091BD13709129
:103B9000BE138091BF139091C0130F94DC2768A3CC
:103BA00079A38AA39BA36093BD137093BE138093E4
:103BB000BF139093C01380917F0290918002A091D7
:103BC0008102B091820288AB99ABAAABBBAB9C01DE
:103BD000AD016091C1137091C2138091C313909194
:103BE000C4130F94DC274B015C016093C1137093E5
:103BF000C2138093C3139093C413A7019601C70106
:103C0000B6010F944D212B013C0128A139A14AA1F5
:103C10005BA1CA01B9010F944D219B01AC01C30105
:103C2000B2010F94DD272B013C01A5019401C501D0
:103C3000B4010F944D219B01AC01C301B2010F945B
:103C4000DD270F948B2A9B01AC0160E070E080E8D7
:103C50009FE30F94D72820916C0230916D02409120
:103C60006E0250916F020F944D212DEC3CEC4CEC08
:103C70005DE30F944D2120E030E040E85EE30F94D7
:103C80004D212B013C0120E030E040E85FE30F9440
:103C9000E72087FFF1C3A3019201C701B6010F948A
:103CA0004D2128A539A54AA55BA50F94DD27609372
:103CB000B9137093BA138093BB139093BC13A301F1
:103CC000920168A179A18AA19BA10F944D212CA5F5
:103CD0003DA54EA55FA50F94DD276093BD1370939E
:103CE000BE138093BF139093C013A3019201C5012B
:103CF000B4010F944D2128A939A94AA95BA90F94B1
:103D0000DD276093C1137093C2138093C313909304
:103D1000C4130E943AEF8CE0FE013196A9EBB3E1A7
:103D200001900D928A95E1F78091E10881110C9440
:103D30000F398091DF089091E0089C012F5F3F4F81
:103D40003093E0082093DF08883E934010F40C94F1
:103D50000F3981E08093E1081092E0081092DF08AB
:103D60008091C608882309F498C30E942483811196
:103D700094C38091DE088F5F8093DE088091DE0817
:103D8000853620F01092DE081092C608E091C60831
:103D90008E2FEE0F990BAA0BBB0BFC013197E7306E
:103DA000F10508F0A0C08827EE58FF4F8F4F0D9403
:103DB000D4270E941C83882309F495C081E0809356
:103DC000000284E094E00E94D6F980E190E09093B4
:103DD000E0168093DF1685E08093D31602E8009307
:103DE000D61684E190E1A0E0B0E08093D7169093DE
:103DF000D816A093D916B093DA160F94B60081E0C6
:103E00009AE59093E0168093DF1686E390E0909316
:103E1000E2168093E11687E08093D3160093D616BE
:103E200084E890E0A0E0B0E08093D7169093D81695
:103E3000A093D916B093DA160F94B60052C00E9420
:103E40001C83882309F44FC048C082E194E00E949B
:103E5000D6F981E09AE59093E0168093DF1680E42E
:103E600090E09093E2168093E11607E00093D3165A
:103E700082E88093D61684E890E0A0E0B0E08093DA
:103E8000D7169093D816A093D916B093DA160F943C
:103E9000B6000093C60827C08091DD08882319F179
:103EA0000E941C838823F9F00E94248381111BC087
:103EB000F7C20E941C838823B1F00E9424838111E1
:103EC00012C01CC30E94248381110DC042E060E037
:103ED00070E0CB010E943A8304C00E9424838111C8
:103EE00002C01092C60880910002882309F4ACC277
:103EF0008091C4089091C508892B09F08FC18091E9
:103F0000DA089091DB08892B09F01EC184E096E065
:103F10009093E0168093DF1680EA90E89093E21683
:103F20008093E11617E01093D31602E80093D6169B
:103F300080EA90E0A0E0B0E08093D7169093D81686
:103F4000A093D916B093DA160F94B60080910302AD
:103F500090910402A0910502B09106020097A1057C
:103F6000B10511F51092E0161092DF1615E01093CE
:103F7000D3160093D6168AE890E1A0E0B0E08093D3
:103F8000D7169093D816A093D916B093DA160F943B
:103F9000B60089E090E09093E0168093DF161093CE
:103FA000D3160093D61640C00196A11DB11DF5E0B1
:103FB000B695A79597958795FA95D1F70197A10999
:103FC000B109009731E0A307B10558F0B093E016AE
:103FD000A093DF169093E2168093E1161093D31608
:103FE00007C09093E0168093DF1685E08093D31688
:103FF00012E81093D6168AE890E1A0E0B0E0809332
:10400000D7169093D816A093D916B093DA160F94BA
:10401000B60088E090E09093E0168093DF1685E08C
:104020008093D3161093D6168CE890E1A0E0B0E010
:104030008093D7169093D816A093D916B093DA161A
:104040000F94B6008091030290910402A0910502A2
:10405000B09106020097E1E0AE07B10550F0B093D1
:10406000E016A093DF169093E2168093E11687E0A6
:1040700005C09093E0168093DF1685E08093D316F9
:1040800082E88093D61688E890E1A0E0B0E08093C3
:10409000D7169093D816A093D916B093DA160F942A
:1040A000B6008091030290910402A0910502B091A4
:1040B0000602BA2FA92F982F88270097F1E0AF07A3
:1040C000B10550F0B093E016A093DF169093E2167E
:1040D0008093E11687E005C09093E0168093DF1689
:1040E00085E08093D31612E81093D61681EA90E00B
:1040F000A0E0B0E08093D7169093D816A093D9167D
:10410000B093DA160F94B6008091AC18882319F09A
:1041100082E090E002C083E090E09093E01680930C
:10412000DF1685E08093D3161093D61685E490E1D0
:10413000A0E0B0E08093D7169093D816A093D9163C
:10414000B093DA160F94B6000091DA081091DB08EC
:10415000053611057CF41093E0160093DF1685E018
:104160008093D31682E88093D61680E090E1A0E099
:10417000B0E011C0C801845691099093E016809375
:10418000DF1685E08093D31682E88093D61681E00F
:1041900090E1A0E0B0E08093D7169093D816A0935A
:1041A000D916B093DA160F94B6000F5F1F4F109315
:1041B000DB080093DA08093C110564F180E294E021
:1041C0000E94D6F981E090E09093C5088093C408DE
:1041D0008093000281E09AE59093E0168093DF16C9
:1041E0008DE290E09093E2168093E11687E0809351
:1041F000D31682E88093D61684E890E0A0E0B0E081
:104200008093D7169093D816A093D916B093DA1648
:104210000F94B6001092E1080C940F3980914D165E
:1042200090914E16891B8F7009F092C10E94608D8B
:1042300081118EC180915B1882FD8AC112C384E610
:1042400090E09093E0168093DF161093D3160093BE
:10425000D6168EE090E1A0E0B0E08093D716909360
:10426000D816A093D916B093DA160F94B600C601EB
:1042700082539048880F991F9093E0168093DF1621
:104280001093D3160093D6168FE090E1A0E0B0E033
:104290008093D7169093D816A093D916B093DA16B8
:1042A0000F94B6000F94FC0D90E09093E01680936D
:1042B000DF1685E08093D31682E88093D61686E1D8
:1042C00090E1A0E0B0E08093D7169093D816A09329
:1042D000D916B093DA160F94B60020E030E048EC1F
:1042E00052E46091D5137091D6138091D7139091B9
:1042F000D8130F944D210F9449297093E0166093C1
:10430000DF1615E01093D31602E80093D61686E266
:1043100090E1A0E0B0E08093D7169093D816A093D8
:10432000D916B093DA160F94B6006091390C7091DB
:104330003A0C80913B0C90913C0C0F94492970935E
:10434000E0166093DF161093D3160093D61686E31B
:1043500090E1A0E0B0E08093D7169093D816A09398
:10436000D916B093DA160F94B6006091FE087091DA
:10437000FF0880910009909101090F9449297093D9
:10438000E0166093DF161093D3160093D6168CE3D5
:1043900090E1A0E0B0E08093D7169093D816A09358
:1043A000D916B093DA160F94B60080913D0C909117
:1043B0003E0C9093E0168093DF161093D316009373
:1043C000D61684E390E1A0E0B0E08093D7169093F6
:1043D000D816A093D916B093DA160F94B600809130
:1043E0000209909103099093E0168093DF161093D1
:1043F000D3160093D6168AE390E1A0E0B0E0809354
:10440000D7169093D816A093D916B093DA160F94B6
:10441000B6000091D60801113CC18091D8088111E5
:1044200038C18091DD0881118BC1809187169091F0
:104430008816A0918916B0918A168C3420E19207D3
:10444000A105B10509F0A1C133E2C32E37E1D32E96
:104450000AE189EC94E10E94874FE090CB08F0904C
:10446000CC08181619060CF085C38AE1E816F10489
:1044700014F40C94D0347EC38CE0FE013196A9EB89
:10448000B3E101900D928A95E1F70E943AEF809195
:10449000BC088D7F8093BC0847CC1092DE086ECCA0
:1044A00082ED95E00E94D6F98091DC0890E0A0E0D2
:1044B000B0E0895B9F4FAE4FB54A21E03AE53093BB
:1044C000E0162093DF169093E2168093E11687E0C2
:1044D0008093D31682E88093D61684E890E0A0E01B
:1044E000B0E08093D7169093D816A093D916B093C6
:1044F000DA160F94B6001092DD08F3CC81E08093B9
:1045000000021092C60880EE95E00E94D6F981E084
:104510009AE59093E0168093DF168EE490E09093F6
:10452000E2168093E11687E08093D31682E88093A9
:10453000D61684E890E0A0E0B0E08093D716909380
:10454000D816A093D916B093DA160F94B600CBCC38
:104550008CE090E09093E0168093DF1605E00093E6
:10456000D31682E88093D61684E190E1A0E0B0E013
:104570008093D7169093D816A093D916B093DA16D5
:104580000F94B6000F94DE0C20E13EE040E050E0D6
:104590000F943D272115310591E04907510560F041
:1045A0005093E0164093DF163093E2162093E11605
:1045B00087E08093D31606C03093E0162093DF1671
:1045C0000093D31602E80093D61680E190E1A0E0B4
:1045D000B0E08093D7169093D816A093D916B093D5
:1045E000DA160F94B6000F94DE0C20E13EE040E0B6
:1045F00050E00F943D272CE330E040E050E00F9472
:104600003D273093E0162093DF1615E01093D31664
:104610000093D61682E190E1A0E0B0E08093D71637
:104620009093D816A093D916B093DA160F94B600CB
:104630000F94FC0D882391F00F94FC0D8F5F8093F5
:10464000D908C82ED12C833308F0F9CDC601880FC4
:10465000991F9093E0168093DF1604C01092E01625
:104660001092DF161093D3160093D6168EE090E1C9
:10467000A0E0B0E08093D7169093D816A093D916F7
:10468000B093DA160F94B6001092E0161092DF166F
:10469000F7CD20E030E048EC52E46091390C7091A5
:1046A0003A0C80913B0C90913C0C0F944D216B0186
:1046B0007C0160913D0C70913E0C072E000C880B24
:1046C000990B0F94EE209B01AC01C701B6010F942A
:1046D000D7280F9450296436710510F064E670E015
:1046E0007093E0166093DF1645E0A42EA092D316D7
:1046F00052E8B52EB092D61684E290E1A0E0B0E088
:104700008093D7169093D816A093D916B093DA1643
:104710000F94B600C090390CD0903A0CE0903B0C4E
:10472000F0903C0C20E030E040E253E4C701B601D9
:104730000F943D2A18160CF03AC1011188C137C1F7
:104740008091CD0801E0080F0093CD0890E0909390
:10475000E0168093DF1685E08093D31682E880937D
:10476000D61682E490E1A0E0B0E08093D716909353
:10477000D816A093D916B093DA160F94B6000A3063
:1047800008F453CE1092CD0850CE8A349041A10542
:10479000B10509F459CE80E00E94188420E030E091
:1047A00040E251E40F944D210F9449297093E01693
:1047B0006093DF1615E01093D31602E80093D61627
:1047C00088E490E1A0E0B0E08093D7169093D816EB
:1047D000A093D916B093DA160F94B60081E00E9428
:1047E000188420E030E040E251E40F944D210F9412
:1047F00049297093E0166093DF161093D316009347
:10480000D6168AE490E1A0E0B0E08093D7169093AA
:10481000D816A093D916B093DA160F94B60082E09A
:104820000E94188420E030E040E251E40F944D21D2
:104830000F9449297093E0166093DF161093D316F6
:104840000093D6168CE490E1A0E0B0E08093D716F8
:104850009093D816A093D916B093DA160F94B60099
:10486000F3CD8091FE089091FF08A0910009B091CE
:10487000010988A399A3AAA3BBA36091020970911F
:104880000309072E000C880B990B0F94EE206B0187
:104890007C0120E030E040E050E40F94DC2728A1C8
:1048A00039A14AA15BA10F943D2A181604F140904A
:1048B000390C50903A0C60903B0C70903C0C60911D
:1048C0003D0C70913E0C072E000C880B990B0F9439
:1048D000EE204B015C0120E030E040E251E40F9417
:1048E000DC27A30192010F943D2A181604F58DE0F0
:1048F00090E09093E0168093DF1685E08093D316C6
:1049000082E88093D61684E190E1A0E0B0E0809345
:10491000D7169093D816A093D916B093DA160F94A1
:10492000B6008091C20881113FC081E03DC020E007
:1049300030E040E050E4C701B6010F94DD2728A124
:1049400039A14AA15BA10F94E72087FD0EC020E0AA
:1049500030E040E251E4C501B4010F94DD27A3012A
:1049600092010F94E72087FFB8CC84E190E0909308
:10497000E0168093DF1685E08093D31682E880935B
:10498000D61684E190E1A0E0B0E08093D716909332
:10499000D816A093D916B093DA160F94B60080916A
:1049A000C208811101C082E08093C20896CC609158
:1049B0003D0C70913E0C072E000C880B990B0F9448
:1049C000EE209B01AC01C701B6010F943D2A609116
:1049D000D80887FDAEC0662309F423CD062E000C4F
:1049E000770B8BE397E00E94C75C1092D808109277
:1049F000DB081092DA0884E090E09093E016809350
:104A0000DF1685E08093D31602E80093D6168EE871
:104A100090E1A0E0B0E08093D7169093D816A093D1
:104A2000D916B093DA160F94B60081E09AE5909308
:104A3000E0168093DF1683E590E09093E216809372
:104A4000E11687E08093D3160093D61663C01092C8
:104A5000D60820E030E040E251E46091CE08709149
:104A6000CF088091D0089091D1080F944D210F94D8
:104A700049297093E0166093DF16A092D316B09286
:104A8000D61684E590E1A0E0B0E08093D71690932D
:104A9000D816A093D916B093DA160F94B60020E07A
:104AA00030E040E251E46091D2087091D3088091E7
:104AB000D4089091D5080F944D210F9449297093F3
:104AC000E0166093DF16A092D316B092D61688E552
:104AD00090E1A0E0B0E08093D7169093D816A09311
:104AE000D916B093DA160F94B6008EEE95E00E94B8
:104AF000D6F981E09AE59093E0168093DF1681E481
:104B000090E09093E2168093E11687E08093D316AD
:104B1000B092D61684E890E0A0E0B0E08093D7167B
:104B20009093D816A093D916B093DA160F94B600C6
:104B300078CC662309F475CC8091DA089091DB0873
:104B40009C012F5F3F4F3093DB082093DA0865E02C
:104B500070E00F94C0279093E0168093DF1685E0F5
:104B60008093D31682E88093D6168EE890E1A0E079
:104B7000B0E0D4CF1E141F040CF04CCB90918416DF
:104B800080912317981322C0909185168091241745
:104B900098131CC023E0E216F104C4F0909125178D
:104BA0009093831680912617809386169330D1F4C4
:104BB000982F9D7F9038B1F4909127179F3409F07A
:104BC00059C0909128179B3409F054C08AE1E3E260
:104BD000F7E1DF011D928A95E9F71092CC08109257
:104BE000CB0818CB833809F045C0809127179091E6
:104BF0002817982789279827A0E0B0E08093871688
:104C000090938816A0938916B0938A16C09029179E
:104C1000D12CE12CF12CC0928B16D0928C16E09204
:104C20008D16F0928E16AAE2B7E140E050E0BA018C
:104C30004C155D056E057F0508F04AC04A015B0111
:104C4000B694A79497948794F4013696EE0FFF1FBD
:104C5000ED57F94E8C9190E0982F882711962C9162
:104C60001197822B918380834E5F5F4F6F4F7F4FF1
:104C70001296DECF813861F58091271790E0A0E091
:104C8000B0E08093871690938816A0938916B0930E
:104C90008A1680912817482F50E060E070E040931A
:104CA0008B1650938C1660938D1670938E16A9E216
:104CB000B7E1EFE8F6E190E020E030E028173907AF
:104CC00039F04D9150E0419351932F5F3F4FF6CF14
:104CD0008AE1E3E2F7E1DF011D928A95E9F710929C
:104CE000CC081092CB0881E394E00E94D6F9609141
:104CF000C608161664F4062E000C770B80E397E0C6
:104D00000E94C75C8AE00E94CBF80C94C134609189
:104D10008F16709190168EE197E00E94A95C8AE050
:104D20000E94CBF8409187165091881660918916A1
:104D300070918A168FE097E00E94985C8AE00E944A
:104D4000CBF88091871690918816A0918916B09122
:104D50008A16EDE8F2E000E010E041915191619196
:104D600071914115510561057105D1F14817590738
:104D70006A077B0791F5AC01BD01485050416109BC
:104D80007109453051056105710568F1AC01BD013E
:104D9000477F423350416105710541F18433F0E1B1
:104DA0009F07A105B10511F1AC01BD014654504169
:104DB000610971094730510561057105D0F0AC01F9
:104DC000BD014455504161097109453051056105E6
:104DD000710588F402E110E00EC00F5F1F4FBDCFD8
:104DE0000FEF1FEF08C003E010E005C008E010E07F
:104DF00002C00FE010E08A509042A109B109833D42
:104E00009105A105B10530F00F3F2FEF120721F4F6
:104E10000C94C13409E110E0F2E5CF2EF4E0DF2E6E
:104E2000F60181916F01882319F00E94CBF8F8CF29
:104E3000B801012E000C880B990B0E943FF90E94CB
:104E4000D0F983E097E00E94D6F90A31110510F0FD
:104E50000C94BD34F8018827E758FF4F8F4F0D940D
:104E6000D42780918F169091901681309105E1F4AE
:104E7000109200028FEF80930B1B60E080E00F9494
:104E80002E0300E614E0D8018D918D01882319F0DE
:104E90000E94CBF8F8CF81E09AE59093E0168093DA
:104EA000DF168EE290E0AFC08230910509F0C5C0F8
:104EB00081E0809300020F946D0E8FEF96E0909347
:104EC0003709809336098BE090E09093E016809349
:104ED000DF1605E00093D31612E81093D61680E093
:104EE00092E1A0E0B0E08093D7169093D816A093FB
:104EF000D916B093DA160F94B6001092E0161092FD
:104F0000DF160093D3161093D6168EE090E1A0E042
:104F1000B0E08093D7169093D816A093D916B0938B
:104F2000DA160F94B6001092E0161092DF16009376
:104F3000D3161093D6168FE090E1A0E0B0E08093F6
:104F4000D7169093D816A093D916B093DA160F946B
:104F5000B6001092E0161092DF160093D31610934D
:104F6000D61686E190E1A0E0B0E08093D71690934A
:104F7000D816A093D916B093DA160F94B60062E053
:104F800070E080E090E00E942C841092E016109275
:104F9000DF160093D3161093D61680E190E1A0E0BF
:104FA000B0E08093D7169093D816A093D916B093FB
:104FB000DA160F94B6001092E0161092DF160093E6
:104FC000D3161093D61682E190E1A0E0B0E0809372
:104FD000D7169093D816A093D916B093DA160F94DB
:104FE000B6000AE814E0F80181918F01882319F0D6
:104FF0000E94CBF8F8CF81E09AE59093E016809379
:10500000DF168DE290E09093E2168093E11687E040
:105010008093D31682E88093D61684E890E0A0E0CF
:10502000B0E08093D7169093D816A093D916B0937A
:10503000DA160F94B6000C94C1348330910549F50B
:1050400081E08093000204EB14E0D8018D918D0182
:105050008823C9F00E94CBF8F8CF809187169091F1
:105060008816A0918916B0918A168233F0E19F07C5
:10507000A105B10509F05BC480918F16909190163F
:10508000009709F023C480910202882309F40DC31C
:105090001DC3049711F00C94C134109200020C94BB
:1050A000C13480918F169091901681309105D1F482
:1050B0001092000280910202882319F082E090E0B1
:1050C00002C083E090E09093E0168093DF1685E0C5
:1050D0008093D31682E88093D6168EE190E1A0E00B
:1050E000B0E09FCF8230910519F50EED14E0F80184
:1050F00081918F01882319F00E94CBF8F8CF81E0CD
:10510000809300028091C208843049F081E09AE5E2
:105110009093E0168093DF1685E390E074CF81E0F2
:105120009AE59093E0168093DF1686E390E06BCFCC
:105130008330910509F04CC020910202222319F11D
:105140009093E0168093DF1685E08093D31682E873
:105150008093D6168EE190E1A0E0B0E08093D71660
:105160009093D816A093D916B093DA160F94B60080
:1051700040E060E070E088EC92E40F94D40E10926E
:1051800002020C94C13482E090E09093E016809388
:10519000DF1685E08093D31682E88093D6168EE1E1
:1051A00090E1A0E0B0E08093D7169093D816A0933A
:1051B000D916B093DA160F94B60040E060E070E0C4
:1051C000CB010F94D40E81E0809302020C94C13481
:1051D000049711F00C94C134809111098823F1F0E7
:1051E00082E090E09093E0168093DF1685E0809354
:1051F000D31682E88093D6168FE190E1A0E0B0E06C
:105200008093D7169093D816A093D916B093DA1638
:105210000F94B600109211090C94C13483E090E011
:105220009093E0168093DF1685E08093D31682E892
:105230008093D6168FE190E1A0E0B0E08093D7167E
:105240009093D816A093D916B093DA160F94B6009F
:1052500081E0809311090C94C13460918F16709194
:10526000901680E090E00F94EC206B017C0120E030
:1052700030E04AEF53E40F94E72087FF11C020E0AD
:1052800030E040E251E4C701B6010F943D2A181600
:105290006CF0C12CD12C70E2E72E71E4F72E06C021
:1052A000C12CD12CEAEFEE2EE3E4FE2EC701B601AD
:1052B0000F94492970937202609371020C94C13467
:1052C0008091871690918816A0918916B0918A16C0
:1052D0008830F0E19F07A105B10509F050C081E0D9
:1052E0009AE59093E0168093DF168DE290E090931C
:1052F000E2168093E11687E08093D31612E81093AC
:10530000D61684E890E0A0E0B0E08093D7169093A2
:10531000D816A093D916B093DA160F94B60010924F
:10532000E0161092DF1605E00093D3161093D61600
:1053300080E190E1A0E0B0E08093D7169093D8167A
:10534000A093D916B093DA160F94B6001092E01617
:105350001092DF160093D3161093D61682E190E1D7
:10536000A0E0B0E08093D7169093D816A093D916FA
:10537000B093DA160F94B6000F946D0E8FC08A307A
:1053800020E19207A105B105E1F580918F1690917A
:105390009016813F910511F00C94C13481E09AE59B
:1053A0009093E0168093DF1686E390E09093E216E8
:1053B0008093E11687E08093D31682E88093D61617
:1053C00084E890E0A0E0B0E08093D7169093D816E0
:1053D000A093D916B093DA160F94B6004EE755E0B5
:1053E00065E875E084E00E94B2D160E081E795E075
:1053F0000F942E0E87E695E0909337098093360937
:105400004DC08C309041A105B10509F047C0809195
:105410008F1690919016019709F040C00F94A31B2E
:105420001092C20881E0809300028CE090E090939B
:10543000E0168093DF1685E08093D31612E8109370
:10544000D61684E190E1A0E0B0E08093D716909367
:10545000D816A093D916B093DA160F94B60081E04F
:105460009AE59093E0168093DF1685E390E09093A1
:10547000E2168093E11687E08093D3161093D61638
:1054800084E890E0A0E0B0E08093D7169093D8161F
:10549000A093D916B093DA160F94B60080918716B0
:1054A00090918816A0918916B0918A168C309041FF
:1054B000A105B10511F00C94C13480918F16909123
:1054C0009016029711F00C94C1340F94A31B81E045
:1054D0008093D8081092C208809300021092DB08D3
:1054E0001092DA0881E09AE59093E0168093DF1637
:1054F00082E590E088CD20918F1630919016B90109
:1055000080E090E037FF09C00F94EC2020E030E00D
:1055100040E857E40F94DC2702C00F94EC2020E011
:1055200030E048EC52E40F94D7286B017C0120E076
:1055300030E040EA51EC0F943D2A87FD31C020E075
:1055400030E040EA51E4C701B6010F94E720181695
:105550003CF1A70196016091D5137091D61380910B
:10556000D7139091D8130F94DC2720E030E048EC5B
:1055700053E40F944D2190580F944929CB010F9477
:10558000FA02C092D513D092D613E092D713F092BC
:10559000D8138AEF96E0909337098093360928C094
:1055A00020E030E048EC52E46091D5137091D613BE
:1055B0008091D7139091D8130F944D210F944929BE
:1055C0007093E0166093DF1685E08093D31682E82F
:1055D0008093D61686E290E1A0E0B0E08093D716E3
:1055E0009093D816A093D916B093DA160F94B600FC
:1055F0006091D5137091D6138091D7139091D813E1
:105600008E010B5E1F4F23E041E00F94BF1B9F9361
:105610008F938CEE96E09F938F93045111091F9303
:105620000F930F947F20C8010E9406850F900F9062
:105630000F900F900F900F900C94C13480918F16A3
:1056400090919016009729F481E0809300020C94C9
:10565000C13481309105B1F480910202882349F070
:1056600081E09AE59093E0168093DF168CE390E05A
:10567000CACC81E09AE59093E0168093DF168BE325
:1056800090E0C1CC82309105F9F28330910539F573
:105690008091020240E0882389F060E070E088ECAD
:1056A00092E40F94D40E1092020281E09AE5909356
:1056B000E0168093DF1689E390E0A5CC60E070E00F
:1056C000CB010F94D40E81E08093020281E09AE531
:1056D0009093E0168093DF168AE390E094CC8530B7
:1056E000910559F540E060E070E084E393E40E94A6
:1056F000AF8246E060E070E08CE892E40E94AF8206
:1057000084EB90E09093E0168093DF1605E0009321
:10571000D31612E81093D61684E390E1A0E0B0E02F
:105720008093D7169093D816A093D916B093DA1613
:105730000F94B60086E490E02DC08630910599F56F
:1057400040E060E070E080E793E40E94AF8246E0D2
:1057500060E070E08CED92E40E94AF8280EF90E018
:105760009093E0168093DF1605E00093D31612E8BD
:105770001093D61684E390E1A0E0B0E08093D716B2
:105780009093D816A093D916B093DA160F94B6005A
:105790008EE690E09093E0168093DF160093D31688
:1057A0001093D616BFC0813F910511F00C94C134FF
:1057B00040E060E070E0CB010F94D40E41E060E087
:1057C00070E0CB010F94D40E1092020240E060E032
:1057D00070E0CB010E94AF8246E060E070E0CB0158
:1057E0000E94AF821092E0161092DF1605E000933F
:1057F000D31612E81093D61684E390E1A0E0B0E04F
:105800008093D7169093D816A093D916B093DA1632
:105810000F94B60061E070E080E090E00E942C847C
:105820001092E0161092DF160093D3161093D6163E
:105830008AE390E1A0E0B0E08093D7169093D81669
:10584000A093D916B093DA160F94B60061E070E019
:1058500080E090E00E942C8484E190E09093E01638
:105860008093DF160093D3161093D61684E190E14F
:10587000A0E0B0E08093D7169093D816A093D916E5
:10588000B093DA160F94B60081E09AE59093E01693
:105890008093DF1689E390E09093E2168093E116FF
:1058A00087E08093D3161093D61684E890E0A0E0AA
:1058B000B0E08093D7169093D816A093D916B093E2
:1058C000DA160F94B60082E00C94BA348130910558
:1058D000A9F440E060E070E0CB010E94AF8210923A
:1058E000E0161092DF1685E08093D31682E880934D
:1058F000D61684E390E1A0E0B0E093CB029711F0DC
:105900000C94C13446E060E070E0CB010E94AF82AD
:105910001092E0161092DF1685E08093D31682E88D
:105920008093D6168AE390E1A0E0B0E07ACB84338E
:1059300020E19207A105B10551F460918F16709195
:10594000901680E090E00F94EC2040E010C08A3385
:105950009041A105B10511F00C94C13460918F16EE
:105960007091901680E090E00F94EC2046E00E9449
:10597000AF820C94C13480918F169091901600974D
:1059800009F462CE8130910509F04CC08091AC18C9
:10599000882319F083E090E002C082E090E09093C9
:1059A000E0168093DF1685E08093D31682E880931B
:1059B000D61685E490E1A0E0B0E08093D7169093EE
:1059C000D816A093D916B093DA160F94B6008AE0D1
:1059D00090E09093E0168093DF1685E08093D316D5
:1059E00082E88093D61680E092E1A0E0B0E0809358
:1059F000D7169093D816A093D916B093DA160F94B1
:105A0000B6000E941C83811103C08CED96E002C099
:105A100080ED96E0909337098093360982E0809379
:105A2000C60871C18230910509F0A8C081E0809359
:105A3000000288E0EEECF8E0DF011D928A95E9F7BC
:105A400080E090E0A0E2B1E48093CE089093CF088C
:105A5000A093D008B093D1088093D2089093D30834
:105A6000A093D408B093D50884E690E09093E01614
:105A70008093DF1605E00093D31612E81093D61634
:105A800084E590E1A0E0B0E08093D7169093D8161B
:105A9000A093D916B093DA160F94B60020E030E048
:105AA00040E251E46091D2087091D3088091D4080B
:105AB0009091D5080F944D210F9449297093E016C9
:105AC0006093DF160093D3161093D61688E590E105
:105AD000A0E0B0E08093D7169093D816A093D91683
:105AE000B093DA160F94B6006091390C70913A0CAD
:105AF00080913B0C90913C0C0F9449297093E016D7
:105B00006093DF160093D3161093D61686E390E1C8
:105B1000A0E0B0E08093D7169093D816A093D91642
:105B2000B093DA160F94B60080913D0C90913E0C24
:105B30009093E0168093DF160093D3161093D61639
:105B400084E390E1A0E0B0E08093D7169093D8165C
:105B5000A093D916B093DA160F94B60062E070E005
:105B600080E090E00E942C8481E09AE59093E0161A
:105B70008093DF1681E490E00C94FD35833091052D
:105B800009F076C01092DC0880E00E94188420E0C2
:105B900030E040E251E40F944D210F944929709375
:105BA000E0166093DF1605E00093D31612E8109319
:105BB000D61688E490E1A0E0B0E08093D7169093E9
:105BC000D816A093D916B093DA160F94B60081E0D8
:105BD0000E94188420E030E040E251E40F944D210F
:105BE0000F9449297093E0166093DF160093D31643
:105BF0001093D6168AE490E1A0E0B0E08093D71627
:105C00009093D816A093D916B093DA160F94B600D5
:105C100082E00E94188420E030E040E251E40F94DA
:105C20004D210F9449297093E0166093DF1600937D
:105C3000D3161093D6168CE490E1A0E0B0E08093E8
:105C4000D7169093D816A093D916B093DA160F945E
:105C5000B60062E070E080E090E00E942C8481E079
:105C60009AE59093E0168093DF1687E490E0C5C72D
:105C70008430910509F485C68530910549F44EE7D5
:105C800050E160E070E085E095E00F94650079C632
:105C9000069709F076C68CEC96E0909337098093CE
:105CA00036098BE090E02BC280918F169091901670
:105CB000019711F51092000281E09AE59093E016A9
:105CC0008093DF168FE390E09093E2168093E116C5
:105CD00087E08093D31682E88093D61684E890E01C
:105CE000A0E0B0E08093D7169093D816A093D91671
:105CF000B093DA160F94B60080918F16909190169B
:105D0000029709F03EC681E09AE59093E0168093F1
:105D1000DF1680E490E077C9E0918F16F09190163D
:105D20003197EB30F10508F0E4C18827ED56FF4FBD
:105D30008F4F0D94D4278091C81480FF5CC6869540
:105D400080FD5CC658C62DEC3CEC4CEC5DE36091EC
:105D5000D5137091D6138091D7139091D8130F94C7
:105D6000DD276B017C0120E030E040EA51EC0F942C
:105D70003D2A87FDC2C120E030E040EA51E4C7017E
:105D8000B6010F94E72018160CF03FC6B6C12DECF3
:105D90003CEC4CEC5DE36091D5137091D61380918F
:105DA000D7139091D8130F94DC276B017C0120E06E
:105DB00030E040EA51EC0F943D2A87FD9EC120E07F
:105DC00030E040EA51E4C701B6010F94E72018160D
:105DD0000CF092C692C180E00E94D0D50E941C8334
:105DE000811103C083E796E002C085E696E09093B8
:105DF00037098093360982E08093C60881E09AE5EE
:105E00009093E0168093DF1684E590E09093E2167D
:105E10008093E11687E08093D31682E88093D616AC
:105E200084E890E0A0E0B0E08093D7169093D81675
:105E3000A093D916B093DA160F94B6005EC183E032
:105E40008093C60883E090E09093E0168093DF167D
:105E500085E08093D31682E88093D6168DE890E192
:105E6000A0E0B0E08093D7169093D816A093D916EF
:105E7000B093DA160F94B600E12CF12C00E0DD248B
:105E8000D394AA24A39445E0942E55E0852E62E88D
:105E9000762EDD2031F0CC24C39435E0B32E10E013
:105EA00005C0CC24CA94BB24BA9414E0DA24B116F9
:105EB000D1F1802F90E04897A4F50F5FF701919EF4
:105EC000E00DF11D1124EE0FFF1FEE0FFF1FE45A2E
:105ED000FB4E20E030E04AE754E46081718182812A
:105EE00093810F944D210F9449297093E01660938C
:105EF000DF168092D3167092D616802F90E08158CC
:105F0000974F880F991F092E000CAA0BBB0B80938B
:105F1000D7169093D816A093D916B093DA160F948B
:105F2000B6001C0DC4CFBFEFEB1AFB0AE5E0EE167E
:105F3000F10409F0AECF81E09AE59093E0168093EA
:105F4000DF1685E590E09093E2168093E11687E0F6
:105F50008093D31682E88093D61684E890E0A0E080
:105F6000B0E08093D7169093D816A093D916B0932B
:105F7000DA160F94B60087E096E090933709809385
:105F80003609BBC042E060E070E080E890E40E9427
:105F90003A8340E060E070E084E393E40E943A8357
:105FA00041E060E070E084E393E413C042E060E02D
:105FB00070E080E890E40E943A8340E060E070E0A6
:105FC00080E292E40E943A8341E060E070E080E287
:105FD00092E40E943A8386E08093C6088EC042E035
:105FE00060E070E080E890E40E943A8340E060E086
:105FF00070E080EA93E4E6CF42E060E070E080E8A1
:1060000090E40E943A8340E060E070E080EA93E42C
:106010000CC042E060E070E080E890E40E943A83C7
:1060200040E060E070E080E292E40E943A8341E068
:1060300060E070E080EA93E4CCCF8091AC188111ED
:106040001CC083E090E09093E0168093DF1685E01B
:106050008093D31682E88093D61685E490E1A0E081
:10606000B0E08093D7169093D816A093D916B0932A
:10607000DA160F94B60081E01BC082E090E09093A6
:10608000E0168093DF1685E08093D31682E8809334
:10609000D61685E490E1A0E0B0E08093D716909307
:1060A000D816A093D916B093DA160F94B60080E0F4
:1060B0000E94D0D520E030E048EC52E46091D51346
:1060C0007091D6138091D7139091D8130F944D21CE
:1060D0000F9449297093E0166093DF1685E0809352
:1060E000D31682E88093D61686E290E1A0E0B0E075
:1060F0009BCE8BEE95E00E94D6F98AE090E09093DB
:10610000E0168093DF1685E08093D31682E88093B3
:10611000D6164BC184E08093C60880918716909173
:106120008816A0918916B0918A1660918F16709189
:1061300090168834F0E19F07A105B10509F453C01A
:106140008A3420E19207A105B10509F456C08C34C8
:1061500030E19307A105B10509F45AC08634904196
:10616000A105B10509F05EC063307105B9F58AED8E
:1061700095E0909337098093360981E08093DD089C
:10618000809300021092CD0881E09AE59093E0168A
:106190008093DF168AE490E09093E2168093E116F4
:1061A00087E08093D31612E81093D61684E890E027
:1061B000A0E0B0E08093D7169093D816A093D9169C
:1061C000B093DA160F94B6008AE090E09093E01650
:1061D0008093DF1685E08093D316E5C06093DC08DA
:1061E0001092C608CEC380E090E0A4EBB3E48CA389
:1061F0009DA3AEA3BFA3312C15C080E090E0A4EB1B
:10620000B3E48CA39DA3AEA3BFA3332433940AC0ED
:1062100080E090E0A8ECB3E48CA39DA3AEA3BFA361
:1062200082E0382E80E090E00F94EC2020E030E017
:1062300040E251E40F94D7286B017C0120E030E06C
:10624000A9010F94E72087FF09C01092C708109298
:10625000C8081092C9081092CA081FC02CA13DA1FD
:106260004EA15FA1C701B6010F943D2A18164CF04C
:10627000C092C708D092C808E092C908F092CA0834
:106280000CC08CA19DA1AEA1BFA18093C708909323
:10629000C808A093C908B093CA086091C708709154
:1062A000C8088091C9089091CA08432D0E943A837A
:1062B00061E070E080E090E00E942C8480E00E9429
:1062C000188420E030E040E251E40F944D210F9417
:1062D00049297093E0166093DF1605E00093D3160A
:1062E00012E81093D61688E490E1A0E0B0E0809325
:1062F000D7169093D816A093D916B093DA160F94A8
:10630000B60081E00E94188420E030E040E251E4D1
:106310000F944D210F9449297093E0166093DF1676
:106320000093D3161093D6168AE490E1A0E0B0E073
:106330008093D7169093D816A093D916B093DA16F7
:106340000F94B60082E00E94188420E030E040E222
:1063500051E40F944D210F9449297093E0166093F6
:10636000DF160093D3161093D6168CE490E1A0E0CC
:10637000B0E08093D7169093D816A093D916B09317
:10638000DA160F94B60061E070E080E090E00E94C1
:106390002C841092C6088AE090E09093E0168093D7
:1063A000DF160093D3161093D61680E092E1A0E09A
:1063B000B0E00C9411288091871690918816A091D6
:1063C0008916B0918A168635E0E19E07A105B105D0
:1063D00009F041C020E030E040E253E46091390C24
:1063E00070913A0C80913B0C90913C0C0F94E720FB
:1063F00020918F163091901687FF0AC42530310501
:1064000008F006C480EA90E09093E0168093DF16CF
:1064100085E08093D31612E81093D61680E290E1BF
:10642000A0E0B0E08093D7169093D816A093D91629
:10643000B093DA160F94B60065E070E080E090E06B
:106440000E942C8481E09AE59093E0168093DF16F9
:1064500082E490E0D2C38435F0E19F07A105B10545
:10646000B9F460918F167091901680E090E00F94CF
:10647000EC2020E030E040E251E40F94D728609314
:10648000CE087093CF088093D0089093D10879C23A
:1064900088359041A105B10509F073C260918F164E
:1064A0007091901680E090E00F94EC2020E030E0B6
:1064B00040E251E40F94D7286093D2087093D30838
:1064C0008093D4089093D5085CC260918F16709128
:1064D000901684EC95E00E94A95C80918F169091B3
:1064E000901682309105A1F038F4009771F0019771
:1064F000E1F48EE295E043C28430910579F058F0E2
:10650000059799F489E995E00BC088E195E037C2D9
:1065100086EB95E005C08CEA95E002C087EA95E03D
:1065200090933709809336092CC282E495E027C204
:1065300081E595E00E94D6F980918F169091901692
:106540008130910519F46499C3C41BC2892B09F0E9
:1065500018C28FE595E00E94D6F98091BD08813080
:1065600039F585E795E00E94D6F981E09AE59093A8
:10657000E0168093DF168EE290E09093E21680930F
:10658000E11687E08093D31682E88093D61684E8DC
:1065900090E0A0E0B0E08093D7169093D816A09337
:1065A000D916B093DA160F94B6001092C10835C010
:1065B000823069F489E895E00E94D6F981E09AE595
:1065C0009093E0168093DF1686E390E00EC0833050
:1065D00031F58DE995E00E94D6F981E09AE5909336
:1065E000E0168093DF1681E490E09093E2168093AA
:1065F000E11687E08093D31682E88093D61684E86C
:1066000090E0A0E0B0E08093D7169093D816A093C6
:10661000D916B093DA160F94B6001092821E10921B
:10662000BD080F946D0EADC180918F16909190169C
:106630008F3F910531F028F08FEF90E0A0E0B0E0BF
:1066400002C0A0E0B0E08093030290930402A09304
:106650000502B09306028091030290910402A0917A
:106660000502B09106020097A105B10509F5109247
:10667000E0161092DF1605E00093D31612E810938F
:10668000D6168AE890E1A0E0B0E08093D716909308
:10669000D816A093D916B093DA160F94B60089E0F5
:1066A00090E09093E0168093DF160093D3163DC0E0
:1066B0000196A11DB11D05E0B695A7959795879503
:1066C0000A95D1F70197A109B109009731E0A30715
:1066D000B10550F0B093E016A093DF169093E21648
:1066E0008093E11687E005C09093E0168093DF1653
:1066F00085E08093D31612E81093D6168AE890E1CD
:10670000A0E0B0E08093D7169093D816A093D91646
:10671000B093DA160F94B60088E090E09093E016FC
:106720008093DF1685E08093D3161093D6168CE8FD
:1067300090E1A0E0B0E08093D7169093D816A09394
:10674000D916B093DA160F94B60080910302909197
:106750000402A0910502B0910602BA2FA92F982F2A
:1067600088270097E1E0AE07B10550F0B093E0163E
:10677000A093DF169093E2168093E11687E005C0A0
:106780009093E0168093DF1685E08093D31682E81D
:106790008093D61681EA90E0A0E0B0E00C94112836
:1067A00081EB95E00E94D6F90E94A3824091871662
:1067B000509188166091891670918A16882339F055
:1067C000433DF0E25F076105710509F4C7C3423D2F
:1067D00050426105710509F0D4C080918F169091E7
:1067E0009016019709F00CC50E94A382882309F432
:1067F00007C580910B1B87FDC4C0A2E18A02C001BE
:1068000011248A53934E0E945751C12C90E2D92EE5
:10681000E12CF12C05E012E81092E0161092DF1640
:106820000093D3161093D616C092D716D092D816CE
:10683000E092D916F092DA160F94B600BFEFCB1A99
:10684000DB0AEB0AFB0AEAE0CE16E0E2DE06E10430
:10685000F10411F700910B1BF2E10F0280011124EA
:10686000025A144EF80101900020E9F7C8018E1B6E
:106870009F0B439697FD01967C01F594E7941E14B7
:106880001F040CF0C6C49E012F5F3F4F690184E1D5
:10689000D9011D928A95E9F7A70162EC75E0C9015B
:1068A0000F94502BB801C6018E0D9F1D0F943B2BEA
:1068B00040E050E260E070E0C6010F94650062E0E5
:1068C00070E080E090E00E942C8440E060E070E0A6
:1068D0008FE793E40F94D40E41E060E070E08FE71F
:1068E00093E40F94D40E109202028DE090E0909306
:1068F000E0168093DF1685E08093D31612E810939C
:10690000D61684E190E1A0E0B0E08093D716909392
:10691000D816A093D916B093DA160F94B60062E099
:1069200070E080E090E00E942C8481E09AE59093F2
:10693000E0168093DF1685E390E09093E216809353
:10694000E11687E08093D3161093D61684E890E082
:10695000A0E0B0E08093D7169093D816A093D916F4
:10696000B093DA160F94B60081E080930002809312
:10697000C10883E08093C20804C08EE895E00E94BD
:10698000D6F980E5E3E8F6E1DF011D928A95E9F7A3
:106990008AE58093841685EA809385160C940A21F3
:1069A00089EC94E10E94654FF701ED5DF84E80831C
:1069B000809123178A3581F01E141F0414F00C9463
:1069C0002922D601E02F1D92EA95E9F71092CC0812
:1069D0001092CB080C94292262E070E080E090E0F5
:1069E0000E942C84FFEFEF1AFF0AF092CC08E0928D
:1069F000CB080C9429228CEB96E002C08BEA96E03F
:106A0000909337098093360955CB88E290E00F9434
:106A1000FA022DEC3CEC4CEC5DE36091D5137091E7
:106A2000D6138091D7139091D8130F94DD276B0163
:106A30007C0120E030E040EA51EC0F943D2A87FDD4
:106A400012C020E030E040EA51E4C701B6010F94E3
:106A5000E720181644F0C092D513D092D613E092D6
:106A6000D713F092D81320E030E048EC52E4609164
:106A7000D5137091D6138091D7139091D8130F949A
:106A80004D210F9449297093E0166093DF1685E03D
:106A90008093D31682E88093D61686E290E1A0E038
:106AA000B0E08093D7169093D816A093D916B093E0
:106AB000DA160F94B6006091D5137091D6138091B9
:106AC000D7139091D8138E010B5E1F4F23E041E046
:106AD0000F94BF1B9F938F938DE996E09F938F93A5
:106AE000045111091F930F930F947F20C8010E9436
:106AF000068588E996E076C088ED9FEF0F94FA024C
:106B00002DEC3CEC4CEC5DE36091D5137091D61309
:106B10008091D7139091D8130F94DC276B017C01DF
:106B200020E030E040EA51EC0F943D2A87FD12C08E
:106B300020E030E040EA51E4C701B6010F94E720BD
:106B4000181644F0C092D513D092D613E092D71302
:106B5000F092D81320E030E048EC52E46091D51375
:106B60007091D6138091D7139091D8130F944D2123
:106B70000F9449297093E0166093DF1685E08093A7
:106B8000D31682E88093D61686E290E1A0E0B0E0CA
:106B90008093D7169093D816A093D916B093DA168F
:106BA0000F94B6006091D5137091D6138091D713CE
:106BB0009091D8138E010B5E1F4F23E041E00F949C
:106BC000BF1B9F938F938AE896E09F938F93045106
:106BD00011091F930F930F947F20C8010E9406850F
:106BE00085E896E090933709809336090F900F90CF
:106BF0000F900F900F900F9080CA9093E2168093A1
:106C0000E11687E08093D3161093D6160C940D28C6
:106C10002430310589F481E00F94791A2091D2084B
:106C20003091D3084091D4085091D5080F94DD27B6
:106C300041E00F94501AB2C02530310508F4F4C079
:106C40002630310509F431C108F023C181E0809379
:106C5000D60840E060E070E08EE393E40E94AF82EB
:106C600020E030E048EC52E46091390C70913A0C2D
:106C700080913B0C90913C0C0F944D216B017C0159
:106C800060913D0C70913E0C072E000C880B990B07
:106C90000F94EE209B01AC01C701B6010F94D728D9
:106CA0000F9450296436710510F064E670E070931B
:106CB000E0166093DF1605E00093D31612E81093F8
:106CC000D61684E290E1A0E0B0E08093D7169093CE
:106CD000D816A093D916B093DA160F94B600609127
:106CE000390C70913A0C80913B0C90913C0C0F94B4
:106CF00049297093E0166093DF160093D316109322
:106D0000D61686E390E1A0E0B0E08093D71690938A
:106D1000D816A093D916B093DA160F94B6008091C6
:106D20003D0C90913E0C9093E0168093DF160093FB
:106D3000D3161093D61684E390E1A0E0B0E08093E0
:106D4000D7169093D816A093D916B093DA160F944D
:106D5000B60065E070E080E090E00E942C8481E065
:106D60009AE59093E0168093DF1684E490E0909388
:106D7000E2168093E11687E08093D3161093D6161F
:106D800084E890E0A0E0B0E08093D7169093D81606
:106D9000A093D916B093DA160F94B60020E030E035
:106DA00040E251E46091CE087091CF088091D00804
:106DB0009091D1080F944D210F9449297093E016BA
:106DC0006093DF1605E00093D31612E81093D616F1
:106DD00084E590E1A0E0B0E08093D7169093D816B8
:106DE000A093D916B093DA160F94B60020E030E0E5
:106DF00040E251E46091D2087091D3088091D408A8
:106E00009091D5080F944D210F9449297093E01665
:106E10006093DF160093D3161093D61688E590E1A1
:106E2000A0E0B0E00C9411282230310579F480E024
:106E30000F94791A2091CE083091CF084091D00854
:106E40005091D1080F94DD2740E0F3CE2330310577
:106E500070F081E00F94791A2091D2083091D30814
:106E60004091D4085091D5080F94DC27E1CE213011
:106E7000310509F093CF80E00F94791A2091CE0864
:106E80003091CF084091D0085091D1080F94DC2761
:106E9000DBCF213F310509F081CF1092D60861E0A8
:106EA00070E080E090E00E942C8481E09AE590936D
:106EB000E0168093DF1681E490E09093E2168093D1
:106EC000E11687E08093D31682E88093D61658CFD8
:106ED0008FE096E00E94D6F981E00E949BD08DE081
:106EE00090E09093E0168093DF1685E08093D316B0
:106EF00012E81093D61684E190E1A0E0B0E0809310
:106F0000D7169093D816A093D916B093DA160F948B
:106F1000B60083E08093C20881E09AE59093E01682
:106F20008093DF1685E390E09093E2168093E1165C
:106F300087E08093D3161093D61684E890E0A0E003
:106F4000B0E08093D7169093D816A093D916B0933B
:106F5000DA160F94B6001092BD0813CD87E296E0C2
:106F60000E94D6F980910C1B90910D1B99272091BE
:106F70008F16309190168217930708F402CD8AEB92
:106F800095E00E94D6F980918F16815080930B1B5B
:106F9000A4ED8A2EA0E29A2EA12CB12C05E012E8D5
:106FA0001092E0161092DF160093D3161093D616A7
:106FB0008092D7169092D816A092D916B092DA166F
:106FC0000F94B6002FEF821A920AA20AB20A3EED7F
:106FD000831630E29306A104B10411F780910B1BD4
:106FE000A2E18A02C0011124FC01E25AF44E7F01A1
:106FF00001900020E9F7C7018E1B9F0B439697FD78
:1070000001968C011595079510161106FCF49E014A
:107010002F5F3F4F690184E1D9011D928A95E9F7FD
:10702000A80162EC75E0C9010F94502BB701C601AD
:10703000800F911F0F943B2B44ED50E260E070E015
:10704000C6010F94650005E012E806C044ED50E269
:1070500060E070E0C701F5CF1092E0161092DF16E5
:107060000093D3161093D6168092D7169092D81606
:10707000A092D916B092DA160F94B600BFEF8B1A11
:107080009B0AAB0ABB0AE6EE8E16E0E29E06A1045E
:10709000B10411F78E010F5F1F4F84E1D8011D92DB
:1070A0008A95E9F780910D1B8F9380910C1B8F932C
:1070B000809190168F9380918F168F938CEC95E032
:1070C0009F938F931F930F930F946A2B4EED50E273
:1070D00060E070E0C8010F94650062E070E080E05D
:1070E00090E00E942C840FB6F894DEBF0FBECDBF97
:1070F00031E2C32E32E1D32EE12CF12C43E1442EB8
:1071000040E6542E612C712C88248394912CAA245F
:10711000AA94BA2C75E0272EE2E83E2E0AE010E091
:1071200080910C1B90910D1B8815990594F1B092DC
:10713000E016A092DF162092D3163092D616409217
:10714000D7165092D8166092D9167092DA160F940C
:10715000B6001093E0160093DF162092D3163092FB
:10716000D616C092D716D092D816E092D916F092C1
:10717000DA160F94B600FFEF8F1A9F0A20E1420E35
:10718000511C611C711C3FEFC31AD30AE30AF30AB6
:10719000C7CF80918F169091901624E0880F991F89
:1071A0002A95E1F78D5F9F49A0E0B0E020EF37E836
:1071B0003093E0162093DF1605E00093D31612E813
:1071C0001093D6168093D7169093D816A093D916FD
:1071D000B093DA160F94B60080918F1690919016A6
:1071E000805E9D4EA0E0B0E026E030E03093E016F7
:1071F0002093DF160093D3161093D6160C94112803
:1072000080918F1690919016892B11F40C94242B59
:10721000B8CB40E050E260E070E0C8014ECBE396AE
:107220000FB6F894DEBF0FBECDBFDF91CF911F9197
:107230000F91FF90EF90DF90CF90BF90AF909F9015
:107240008F907F906F905F904F903F902F90089518
:107250002F923F924F925F926F927F928F929F9266
:10726000AF92BF92CF92DF92EF92FF920F931F9354
:10727000CF93DF93CDB7DEB7C154D1090FB6F894E1
:10728000DEBF0FBECDBF22968FAF22972091F708A9
:107290002CAF21E02093F708809154128D3409F42B
:1072A000A4C4843511F40C94DC4B873411F00C9495
:1072B000E34B80915212909153128B31910509F456
:1072C00020C2B4F48430910534F482309105E4F5A1
:1072D00097FF2EC086C48531910511F40C94E54BBF
:1072E0008A31910509F409C2049709F07AC4C6C12C
:1072F0008A32910509F4AEC34CF48D319105B1F099
:107300000CF429C24E9709F465C26BC48B35910504
:1073100009F41EC38C35910509F41EC38A35910505
:1073200009F05FC41092F6080C94E54B14E03FC2DC
:1073300080918702882311F40C94E54B0E9408E0A9
:107340000E943AEF0C94E54B20918702222311F41E
:107350000C94E54B11E0029709F010E00E9408E060
:1073600019821A821B821C821D821E821F8218862D
:1073700082E50E9432D0882309F438C10E94B2CF3E
:107380004B015C0120E030E0A9010F94E720882345
:1073900009F442C18091770290917802A09179021C
:1073A000B0917A028CA39DA3AEA3BFA380917B0270
:1073B00090917C02A0917D02B0917E0288A799A74E
:1073C000AAA7BBA78091B9139091BA13A091BB1340
:1073D000B091BC138CA79DA7AEA7BFA78091BD138A
:1073E0009091BE13A091BF13B091C01388AB99AB1D
:1073F000AAABBBAB2CA53DA54EA55FA56CA17DA1FD
:107400008EA19FA10F94E72081110DC028A939A951
:107410004AA95BA968A579A58AA59BA50F94E72031
:10742000882309F4F9C020E030E0A901C501B401C6
:107430000F94E720881F8827881F181729F080E0FD
:1074400090E0A0E8BFEB04C080E090E0A0E8BFE3DC
:1074500088AF99AFAAAFBBAF2CA13DA14EA15FA150
:107460006CA57DA58EA59FA50F94DC276CAB7DAB8D
:107470008EAB9FAB28A539A54AA55BA568A979A9BC
:107480008AA99BA90F94DC276B017C012CA93DA93B
:107490004EA95FA9CA01B9010F944D212B013C01EE
:1074A000A7019601C701B6010F944D219B01AC01C4
:1074B000C301B2010F94DD270F948B2A2B013C01ED
:1074C0009B01AC0160E070E080E89FE30F94D72857
:1074D00021966CAF7DAF8EAF9FAF219720E030E05B
:1074E00040E05FE3C301B2010F944D212B013C0149
:1074F000A5019401C501B4010F944D214B015C011C
:10750000A3019201C301B2010F944D219B01AC0173
:10751000C501B4010F94DC270F948B2A28AD39AD37
:107520004AAD5BAD0F944D214B015C01C701B60123
:10753000905821962CAD3DAD4EAD5FAD21970F9487
:107540004D21A50194010F944D216B017C012CA5C7
:107550003DA54EA55FA56CA17DA18EA19FA10F9415
:10756000DD2720E030E040E05FE30F944D219B01F8
:10757000AC01C701B6010F94DD272CA13DA14EA19E
:107580005FA10F94DC2769837A838B839C8328A96E
:1075900039A94AA95BA968A579A58AA59BA50F94D5
:1075A000DD2720E030E040E05FE30F944D216B01E8
:1075B0007C0121962CAD3DAD4EAD5FAD21976CA900
:1075C0007DA98EA99FA90F944D21A50194010F9427
:1075D0004D219B01AC01C701B6010F94DD2728A501
:1075E00039A54AA55BA50F94DC2712C089E40E9447
:1075F00032D0882331F00E94B2CF69837A838B83A3
:107600009C838AE40E9432D0882331F00E94B2CF5A
:107610006D837E838F83988720E030E0A9016981A4
:107620007A818B819C810F94E72081110BC020E02F
:1076300030E0A9016D817E818F8198850F94E720CC
:107640008823A1F0412FBE016F5F7F4F89EB93E14B
:107650000E94E7C10E9425EE6093C0147093C1148C
:107660008093C2149093C3140C94E54B0E94E75C82
:107670008CE797E00E94025C0C94E54B80E50E9449
:1076800032D0882329F00E9450AC6B017C0103C0EA
:10769000C12CD12C760183E50E9432D0882361F081
:1076A0000E94B2CF20E030E04AE754E40F944D212D
:1076B0000F9450296B017C010E9443C88091DA131A
:1076C000811105C060E082E997E00F942E0E0E94C0
:1076D00025EEC60ED71EE81EF91E0E9425EEDC011F
:1076E000CB018C199D09AE09BF09B7FD02C00C94EE
:1076F000E54B80E00E94C15DF0CF0E94FE660C94D5
:10770000E54B0E949FE781110C94E54B80E090E0EF
:10771000A8E4B2E489839A83AB83BC8380E090E0E1
:10772000A0E2B1E48D839E83AF83B88789879A876F
:10773000AB87BC8780E50E9432D0882321F00E946D
:107740008ACF862F01C080E0BE016F5F7F4F0F940C
:10775000660D0C94E54B8091D9138770873011F03A
:107760000C94F04B60E08FE40E94E96681110C9468
:10777000E54B0C94F04B8091AC1881111DC00E9418
:1077800006B18823F9F0115011F40C94924D40E0A9
:1077900050E06DED77E085E00E94F9D061E080ED8A
:1077A00097E00E943FD088EB97E00F949C100E94D6
:1077B0009FE7882301F306C060E08FE40E94E9663A
:1077C0008823E9F20E9463D08BE798E00F949C1025
:1077D0000C94E54B20E030E044E252E46091770203
:1077E000709178028091790290917A020F94DC274F
:1077F000AB01BC0188E50E9414866C8F7D8F8E8F53
:107800009F8F20E030E040E051E460917B02709176
:107810007C0280917D0290917E020F94DC27AB0167
:10782000BC0189E50E9414869B01AC0169837A83BF
:107830008B839C836C8D7D8D8E8D9F8D0E94FCBF74
:10784000882311F40C94E54B80E00E94D0D50E946F
:1078500022F261E085E40E94E966182F21E0482FBA
:10786000BE016F5F7F4FCE014C960E944EE86B01C8
:107870007C019B01AC010F94CF2A81115FC08C8CDD
:107880009D8CAE8CBF8C20E030E0A901C501B40115
:107890000F94E72087FF05C027E137EB41E558EB60
:1078A00004C027E137EB41E558E3C501B4010F946B
:1078B000DD27AB01BC018DE998E00E94B65C8980B0
:1078C0009A80AB80BC8020E030E0A901C501B40102
:1078D0000F94E72087FF05C027E137EB41E558EB20
:1078E00004C027E137EB41E558E3C501B4010F942B
:1078F000DD27AB01BC0188E998E00E94B65C20E07E
:1079000030E0A901C701B6010F94E72087FF05C049
:1079100027E137EB41E558EB04C027E137EB41E5C0
:1079200058E3C701B6010F94DD27AB01BC0183E921
:1079300098E00E94B65C8AE00E94CBF80E9409F2AF
:10794000113011F40E9467AB0E94CFF30C94E54B09
:107950002093F6080C94E54B85EA282E83E0382E18
:1079600096E4E92E93E1F92E27E732E03DA32CA31C
:1079700029ECC22E23E1D22E00E010E0D1018D913E
:107980001D010E9432D0882309F44BC00E94B2CF5F
:107990002B013C01133049F0F601208131814281F5
:1079A00053810F94DC272B013C01ACA1BDA12D918B
:1079B0003D914D915C91C301B2010F94DC274B01C5
:1079C0005C012DEB37E346E855EB0F943D2A87FD2C
:1079D0000AC02DEB37E346E855E3C501B4010F9427
:1079E000E7201816F4F4133051F4409283025092B9
:1079F0008402609285027092860201E012C0A501A5
:107A00009401F70160817181828193810F94DD2758
:107A1000D7016D937D938D939C931397812F0E9433
:107A2000CFCD1F5FB4E0EB0EF11CECA1FDA13496AD
:107A3000FDA3ECA3F4E0CF0ED11C143009F09ECFCF
:107A4000002321F083E892E00E9454C80E94CFF303
:107A50000C94E54B80918702882311F40C94E54B3C
:107A600089E40E9432D0082F882321F00E94AECFF3
:107A7000E82E01C0E12C8AE40E9432D0182F88231E
:107A800021F00E94AECFF82E01C0F12C002319F096
:107A900024E02E1528F0112349F034E03F1530F48E
:107AA00085EA98E00E94025C0C94E54B0E94106409
:107AB0000023F1F020915014309151144E2D4203C7
:107AC000B001439F700D11248091EE0B9091EF0B4C
:107AD000680F791F072E000C880B990B0F94EE206E
:107AE0006093B9137093BA138093BB139093BC1334
:107AF0001123F1F020915214309153144F2D420371
:107B0000B001439F700D11248091F00B9091F10B07
:107B1000680F791F072E000C880B990B0F94EE202D
:107B20006093BD137093BE138093BF139093C013E3
:107B300060E080E50E94E966882381F10023B1F0CE
:107B400020E030E044E252E46091B9137091BA133E
:107B50008091BB139091BC130F94DD276093B913F0
:107B60007093BA138093BB139093BC131123B1F09D
:107B700020E030E040E051E46091BD137091BE130D
:107B80008091BF139091C0130F94DD276093BD13B4
:107B90007093BE138093BF139093C01340E050E0E6
:107BA000BA0186E40E9414866B017C0120E030E07B
:107BB000A9010F943D2A181684F420E030E040E734
:107BC00052E4C701B6010F94D72860936C027093FA
:107BD0006D0280936E0290936F020E943AEF0C94B4
:107BE000E54B0E9477A10C94E54B80915212909145
:107BF00053128537910511F40C9412460CF050C1C4
:107C00008934910509F417C50CF069C08A319105D2
:107C100009F49CC39CF58431910509F411C37CF4EB
:107C20008131910509F4EBC22CF4029708F460C28B
:107C30000C94D94B429709F44CC70C94D94B87311B
:107C4000910509F427C38CF48531910509F41EC30D
:107C5000469711F00C94D94B0E943E5180915B18CD
:107C6000877F80935B180C94E54B8831910509F46C
:107C700029C3499709F45FC30C94D94B8F319105FF
:107C800009F492C47CF48C31910509F4D7C30CF447
:107C90006BC38D31910509F4DBC34E9709F4DFC343
:107CA0000C94D94B8A32910509F49EC464F4803255
:107CB000910509F433C4819711F00C94D94B0E94BB
:107CC000838C0C94E54B8B32910509F4B0C4C097BA
:107CD00011F00C94D94B0E947BAC0C94E54B883688
:107CE000910509F451C5D4F58135910509F4D9C63A
:107CF000C4F48C34910509F4ADC44CF48B34910573
:107D000011F00C94D94B0E94A0C60C94E54B8D3415
:107D1000910509F4A3C48E34910509F4A3C40C940D
:107D2000D94B8435910509F4D4C674F48235910594
:107D300009F4CCC68335910511F00C94D94B81E040
:107D40008093F0080C94E54B8535910509F4C4C681
:107D50008C35910509F4D9C60C94D94B8E36910512
:107D600009F491C5D4F48B36910509F48AC654F40C
:107D70008936910509F423C68A36910509F459C656
:107D80000C94D94B8C36910511F40C94E54B8D363F
:107D9000910509F41DC50C94D94B8137910509F45F
:107DA000C8C55CF48F36910509F47EC5803791050E
:107DB00011F40C94E54B0C94D94B8237910509F4DE
:107DC0002EC78337910511F00C94D94B84E59BE0C5
:107DD0000E94025C60E084E49BE00E94ADC560E02C
:107DE0008FE29BE00E94ADC561E088E29BE00E94CB
:107DF000ADC561E08DE19BE00E94ADC561E08DE025
:107E00009BE00E94ADC560E084E09BE00E94ADC5B0
:107E100061E08AEF9AE00E94ADC561E080EF9AE0F0
:107E20000E94ADC561E088EE9AE00E94ADC561E0B8
:107E30008AED9AE00E94ADC561E08CEC9AE00E9468
:107E4000ADC560E08DEB9AE00E94ADC560E08FEAC1
:107E50009AE00E94ADC560E089E99AE00E94ADC554
:107E600061E088E89AE00E94ADC561E089E79AE0A8
:107E70000E94ADC561E084E69AE00E94ADC561E074
:107E800081E59AE00E94ADC560E084E49AE00E943A
:107E9000ADC560E080E39AE00E94ADC50C94E54B6F
:107EA0008F32A1E09A0711F40C94A3490CF07AC028
:107EB0008B3C910509F475C7ACF58D37910509F434
:107EC000EDC5BCF48737910509F4EFC60CF4BBC6C9
:107ED0008837910509F4ECC68937910511F00C94A7
:107EE000D94B10922609109225090E945CF50C943A
:107EF000E54B8E3B910509F450C554F48C3891053F
:107F000009F439C58B39910509F46DC50C94D94B29
:107F1000883C910509F4D4C6893C910509F41DC734
:107F20000C94D94B8D3D910509F492C7E4F48E3C35
:107F3000910509F45AC76CF48C3C910509F452C7B9
:107F40008D3C910511F00C94D94B0E940EBC0C9401
:107F5000E54B833D910509F46BC78C3D910509F410
:107F60006AC70C94D94B8232E1E09E0711F40C945D
:107F700061485CF4823E910509F4C0C788319140A4
:107F800011F40C94CA470C94D94B8D3231E093070D
:107F900011F40C946C488E32914011F40C945F49AA
:107FA0000C94D94B853FA1E09A0711F40C94BA4A7E
:107FB0000CF04EC08A39E1E09E0711F40C94E54BB9
:107FC00014F5803921E0920711F40C94A6493CF491
:107FD0008033914011F40C94EC480C94D94B8139C6
:107FE000A1E09A0711F40C94A9498239914011F04B
:107FF0000C94D94B80E00E94AFAB0E9467AB0E940B
:10800000CFF30C94E54B853AE1E09E0711F40C9414
:10801000BA497CF48C3921E0920711F40C94AF49F1
:10802000843A914011F00C94D94B0E943E650C9417
:10803000E54B8C3A41E0940711F40C942A4A843FB2
:10804000914011F00C94D94B0E943E760C94E54B74
:108050008B35B2E09B0711F40C94164B4CF5883F1E
:10806000F1E09F0711F40C94C04A9CF4863F31E084
:10807000930711F40C94BD4A873F914011F00C9482
:10808000D94B61E083E50E94E9660E9437FC0C94BD
:10809000E54B8C30A2E09A0711F40C94D14A883554
:1080A000924011F00C94D94B0E94E0E00C94E54B07
:1080B0008438E3E09E0711F40C948F4B6CF4833505
:1080C00023E0920711F40C94D94A8C36934011F4B2
:1080D0000C94E54B0C94D94B803A43E0940709F497
:1080E00053C2873E934011F40C94CB4B0C94D94B64
:1080F0000091FF0B1091000C80E50E9432D0882384
:1081000061F00E9450AC6B017C01BB24B394672BDF
:10811000682B692B31F4B12C04C0B12CC12CD12CAB
:10812000760183E50E9432D0882311F40C94A44D8B
:108130000E94B2CF20E030E04AE754E40F944D2192
:108140000F9450296B017C01B1100BC0672B682B79
:10815000692B39F40115110521F0F8018081811195
:1081600002C0B12C02C0BB24B3940E9443C8B1101A
:1081700003C086E396E001C0C8010E944B851091C0
:10818000F70883E08093F70881E08093821E46ED34
:1081900058E06FED78E082E00E94F9D084EC98E03E
:1081A0000E944B85C114D104E104F104B1F00E9496
:1081B00025EEC60ED71EE81EF91E0E9425EEDC0134
:1081C000CB018C199D09AE09BF09B7FF0EC0809184
:1081D000821E81110C94A94D08C08091821E8823B3
:1081E00021F080E00E94C15DF8CF80E090E00E9425
:1081F0004B851092821E1093F7080C94E54B8091EA
:108200004E1284FF02C00C94AE4D8091501287FF35
:1082100002C00C94AE4D80915112837011F00C94F9
:10822000AE4D60E081EF98E00F942E0E5F988A9833
:108230008091080181708093060112980C94E54B9F
:1082400089E099E00E94025C10922A0B8FEB95E185
:108250000E94847C8BE1EFEBF5E1DE011196019049
:108260000D928A95E1F740E050E0BE016F5F7F4FCD
:1082700080E090E00E94C452CE0101960E94BA7D37
:108280008AEF98E00E94025C0C94E54B0E94AF518B
:108290000C94E54BE091FF0BF091000C808188235A
:1082A00029F0803209F410823196F8CF40E061E085
:1082B0008091FF0B9091000C0E949A541092831EA3
:1082C0000C94E54B8091BC0A8823E9F080E090E0B3
:1082D000A0EAB1E488A399A3AAA3BBA31C8E1D8E18
:1082E0001E8E1F8E19821A821B821C8220E0AE0114
:1082F000405E5F4FBE01645E7F4FCE0101960E94DB
:10830000B9D10C94E54B0E94608D882321F00E9426
:108310004F510E94A0C640E050E06AE179E085E05C
:108320000E94B2D161E08AE899E30E943FD00F94A5
:10833000B20E0C94E54B80915B1882FF03C08B7FDB
:1083400080935B180E94E7E10C94E54B80915B18E9
:1083500083FD02C00C94E54B83E50E9432D081116D
:108360000C94CA4D0C94E54B83E40E94E9CF88231A
:10837000D9F18EE299E00E94025C80916915882310
:1083800051F1BE016F5F7F4F86E695E10E944B7B06
:108390008E010F5F1F4FD8018D918D01882319F039
:1083A0000E94CBF8F8CFBE016F5F7F4F80E090E076
:1083B0000E9462548091BC1A882389F080E20E9456
:1083C000CBF80CEB1AE1F80181918F01882339F089
:1083D0000E94CBF8F8CF84E299E00E94025C8AE028
:1083E0000E94CBF80C94E54B83E50E9432D08823A1
:1083F00009F10E949ACF182F90E0CD970CF01CE362
:108400001093E7080E9425EE6B017C01212F30E0DC
:10841000A8EEB3E00F949127C60ED71EE81EF91EF2
:10842000C092E308D092E408E092E508F092E608F2
:108430000C94E54B0E9417510C94E54B40E060E032
:108440008091FF0B9091000C0E949A540C94E54B84
:1084500080915B188E7F80935B180C94E54B809124
:108460005B1883FD02C00C94E54B0E945FEA80918B
:108470005B1883FD02C00C94E54B6091FF0B70917B
:10848000000CCE014C960F9412028C01009711F44F
:108490000C94E54B6C8D7D8D19821C8222E0AC0121
:1084A000CE0101960E949D81811102C0F12C14C061
:1084B000CE0101960F9480018823C1F361E0CE01C3
:1084C00001960E942F7B009789F325EEDC012C9307
:1084D0001C820E943E7DF82ECE0101960E94BA7D3C
:1084E000B801FF2089F088E599E00E94D45C8AE019
:1084F0000E94CBF8109257181092581810925918E1
:1085000010925A180C94E54B80E499E00E94D45CD8
:108510008DE399E00E94025C0C94E54B80915B181E
:1085200082FD0E9443C880915B1883FD02C00C94B9
:10853000E54B60E080E50E94E966182F482F61E076
:108540008091FF0B9091000C0E949A5483E50E9449
:1085500032D0882381F00E948ACFAB01BC014093C6
:108560005718509358186093591870935A1886E604
:1085700095E10E94457A0E944F5111110C94E54BF0
:108580000E94A0C60C94E54B2091FF0B3091000C8B
:1085900090915B18926090935B1840E060E0C90195
:1085A0000E949A540C94E54B0F94DE0C6C8F7D8FD7
:1085B0008E8F9F8FBE016F5F7F4FCE014C960E94C2
:1085C000A78B60E0CE0101960F94890E0E94EB5CB0
:1085D000BE016F5F7F4F86E699E00E94D45C8AE01F
:1085E0000E94CBF80C94E54B83E50E9432D088239F
:1085F00011F40C94E54B0E949ACFF82E6DE070E0D8
:1086000080E50E9460AC8C0197FF02C00C94E54BA2
:10861000E82E60E089E40E94E96681110C94DB4D4C
:10862000802F0E943CF6811186C40C94DB4D0E9481
:10863000FBE30C94E54B80E50E94E9CF882311F41D
:108640000C94E54B80915B1882FF02C00C94E54BC3
:108650000C94F44D0F942D0D0C94E54B0E9404C71F
:108660000C94E54B60E070E083E50E9460AC8E34D2
:10867000910531F40E9479C70F94B20E0C94E54B2A
:1086800081ED99E00E94025C6091150970911609D4
:1086900088EC99E00E94A95C609117097091180913
:1086A0008BEB99E00E94A95C609115097091160905
:1086B0008091170990911809681B790B80916713B5
:1086C000815021E030E0823010F020E030E0621B89
:1086D000730B80EB99E00E94A95C8AE00E94CBF8C2
:1086E00088EA99E00E94025C8091190990911A0928
:1086F000A0911B09B0911C098C8F9D8FAE8FBF8FED
:10870000BE016F5F7F4FCE014C960E94A78BBE01CA
:108710006F5F7F4F8BE999E00E94D45C80911D09C7
:1087200090911E09A0911F09B09120098C8F9D8FF7
:10873000AE8FBF8FBE016F5F7F4FCE014C960E9400
:10874000A78BBE016F5F7F4F8BE899E00E94D45CDE
:1087500020E030E04AE754E4609121097091220959
:1087600080912309909124090F94D728AB01BC0173
:1087700083E799E00E94B65C8DE60E94CBF88AE020
:108780000E94CBF80C94E54B8091821183FF02C0CC
:108790000C94E54B0E94B7E087FF02C00C94E54BB8
:1087A00083E50E9432D0882379F00E94B2CF0F94E3
:1087B00049298B01CB010E9475DE0135110524F496
:1087C0000E9404C70F94B20E0F948F1A0C94E54BBD
:1087D0008091821183FF02C00C94E54B0E94B7E0A8
:1087E000F82E87FF02C00C94E54B83E50E9432D03F
:1087F000082F811106C082E50E9432D0182F8823ED
:10880000C1F10E94B2CF0F944929CB010E9475DEBD
:108810000E94B2CF20E030E040EA52E40F94E7201B
:10882000181614F40C94FF4D0E9404C70F94B20E56
:1088300060913D0C70913E0C072E000C880B990B3B
:108840000F94EE204B015C014090390C50903A0C93
:1088500060903B0C70903C0CA30192010F943D2A58
:10886000181614F40C94124E002311F40C94034EB9
:1088700011E00F948F1A112309F4A7C7602F8F2DD1
:108880000E9484D8A2C78EE40E9432D0882309F4C3
:108890009CC70E948ACF6093D7127093D81280939E
:1088A000D9129093DA1291C783E50E94E9CF882309
:1088B00031F060E083E50E946FAC809382110E94EA
:1088C000EB5C81E09AE00E94025C80918211882337
:1088D00069F107EFE02E09E0F02E00E010E020E063
:1088E0008091821190E0A0E0B0E0002E04C0B69527
:1088F000A795979587950A94D2F780FF0EC0DD243F
:10890000D394D20E222319F08CE20E94CBF8F70107
:10891000859194910E94025C2D2D0F5F1F4FB2E054
:10892000EB0EF11C05301105D9F659CD83EF99E016
:1089300054CD83E50E9432D0882371F00E949ACFF3
:10894000282F30E02D3331051CF4809301023DC700
:108950008CE38093010239C70E94EB5C40910102D5
:1089600050E060E070E088E09AE00E94985C8AE065
:108970000E94CBF82AC78091821183FD26C783E528
:108980000E9432D0882309F420C70E94B2CF0F94EE
:108990004929CB010E94026418C78091821183FD8E
:1089A00014C783E50E9432D0182F81110C94154E04
:1089B00082E50E9432D081110C94154E06C70E94A8
:1089C000B7E0182F87FD0AC08DE29AE00E94025C92
:1089D000812F0E9494D68AE00E94CBF8ECADE09300
:1089E000F7080C940E4F83E50E9432D0882309F4D7
:1089F000ECC60E949ACF182F90E0CD970CF01CE3A4
:108A00001093EC080E9425EE6B017C01212F30E0D1
:108A1000A8EEB3E00F949127C60ED71EE81EF91EEC
:108A2000C092E808D092E908E092EA08F092EB08D8
:108A3000CCC660E080E50E946FACF82EF1E0F8173C
:108A400008F4C3C681E40E94E9CF882321F0609135
:108A5000220C062F02C00FEF10E083E50E9432D0F7
:108A6000882349F00E948ACF8B016F3F710519F06E
:108A700010F00FEF10E0EF2DF0E0EE5DF34F00830C
:108A8000A4C660E080E50E946FAC823008F09DC60D
:108A9000E82FF0E0EE5DF34F108297C60E94E7E109
:108AA00094C60E9486DE0E9404C70E94D7C90E9415
:108AB0007EF610921E1410921D1410921C1468EE73
:108AC00073E080E090E00E94D35B7FC61092F008D4
:108AD0007CC60E946AE379C683E50E94E9CF8823B9
:108AE00009F473C60E94B2CF20E030E04AE754E4B4
:108AF0000F944D210F9450296093F1087093F20860
:108B00008093F3089093F40860C60E94B7E087FD55
:108B10005CC690914E1294FD04C09091501297FF44
:108B20000AC0B5EACB2EB3E0DB2E13E8E12E11E14B
:108B3000F12E10E009C090915112937091F7682FB7
:108B400081E00E94C0E341C6D6018D916D010E9473
:108B500032D0882309F459C0133009F04FC00E9465
:108B6000B2CF4B015C0120E030E040EA51E40F94C9
:108B7000E72087FF3AC0A50194016091A31170918D
:108B8000A4118091A5119091A6110F94D7282B01C3
:108B90003C019B01AC016091B3117091B4118091C3
:108BA000B5119091B6110F944D216093B31170934C
:108BB000B4118093B5119093B6116091160C709119
:108BC000170C8091180C9091190C0F94EC20A301B4
:108BD00092010F944D210F9450296093160C7093BD
:108BE000170C8093180C9093190C8092A3119092FB
:108BF000A411A092A511B092A61107C00E94B2CFF5
:108C0000F701648B758B868B978B1F5FF4E0EF0EFB
:108C1000F11C143009F098CF0E941FC8D6C50F94DC
:108C20002A0FD3C58091FF0B9091000C009741F063
:108C3000DC012C91222321F060E00F94890EC5C540
:108C40000F94B20EC2C50091FF0B1091000C83E08F
:108C5000F12C40E08150E1F0F8019081292F2B7F29
:108C60002134C1F721812133A9F7913421F09534C2
:108C700021F441E002C0FF24F39498012E5F3F4F9E
:108C800089012F5F3F4FD8019C919032C9F3E2CF09
:108C900041110E94EB5CFF2021F081E49CE00E94E6
:108CA000025CC8010E94D6F990C50E9405F58DC5E9
:108CB00081E080932609809325090E945CF585C593
:108CC0000E94B7E0182F87FD80C584E40E94E9CF99
:108CD000882309F43FC00E94B2CF6B017C0101E000
:108CE00020E030E0A9010F94E720811101C000E0ED
:108CF0000093521320E030E0A901C701B6010F94A0
:108D0000E720882339F10E94B2CFB4E01B02F001C2
:108D10001124E95AFC4E608371838283938320E09F
:108D200030E0A90160915713709158138091591345
:108D300090915A130F94E72081110CC080E090E0CD
:108D4000A0EEBFE38093571390935813A093591349
:108D5000B0935A130E9401CB38C50E94B7E087FD3B
:108D600034C5A5EAEA2EA3E0FA2E03E811E1F701E3
:108D700081917F010E94E9CF882351F00E94B2CFF8
:108D80000F945029D8016D937D938D939C931397E5
:108D90000C5F1F4FB1E103391B0749F70E94A8C7B9
:108DA00014C50E94B7E087FD10C5F5EAEF2EF3E089
:108DB000FF2E03E811E1F70181917F010E94E9CFC5
:108DC000882349F00E94B2CFD80194966D937D9389
:108DD0008D939C9397970C5F1F4FB1E103391B074D
:108DE00051F7F3C40E94B6BCF0C475EAC72E73E015
:108DF000D72EE9E2EE2EE9E0FE2E10E0F601819199
:108E00006F010E94E9CF882359F00E94B2CFD701A9
:108E10006D937D938D939C931397812F0E94CFCD5B
:108E20001F5FB4E0EB0EF11C133041F70C94263DAC
:108E30000E94B5E2CAC483E50E9432D0882309F4B7
:108E4000C4C40E94AECF9093720280937102BDC4DD
:108E50000E94B7E0F82E87FDB8C483E50E9432D0A7
:108E60000F2D0F2C000C110B882369F10E94AECF3F
:108E7000F801EE0FFF1FE15BFD4F91838083000F30
:108E8000111F000F111FF801E05EFD4F7F01BC01B3
:108E9000990F880B990B0F94EE202AE037ED43E2EF
:108EA0005CE30F944D21F801ED5AFC4E2081318195
:108EB000428153810F944D21D7016D937D938D9302
:108EC0009C93139782C40E94EB5C85E40E94CBF8CC
:108ED00080E38F0D0E94CBF8F801EE0FFF1FE15BDE
:108EE000FD4F6081718185E49CE00E94C75C85E252
:108EF0000E94CBF88AE00E94CBF867C480E50E940C
:108F0000E9CF882309F461C460E070E080E50E9445
:108F100060ACF82E6FEF7FEF83E50E9460AC8C01B0
:108F20000196039708F051C4F7FC4FC48F2D0E949F
:108F30003CF6882339F00E94E75C8DE49CE00E94B7
:108F4000025C43C40E9443C860E08F2D0E94C7ECBE
:108F50000F3FBFEF1B0731F00130110571F000E04A
:108F600010E00DC08F2D0E946FEC31E020E0892BC6
:108F700009F030E0032F122F02C001E010E08F2D26
:108F80000E946FEC8017910709F41FC480E00E94D3
:108F9000C15DF5CF80E50E94E9CF882309F415C4AF
:108FA0000E94AECF8C01892B09F07FC083E50E941F
:108FB000E9CF882389F00E94AECF8F3FEFEF9E0765
:108FC00029F487E496E10E9483F6FFC3BC0187E49D
:108FD00096E10E94C2F6F9C30E94EB5C60E070E08B
:108FE00085E79CE00E94C75C8091491628E532E045
:108FF0006901C81AD10887FDD394CC0CDD1CCC0CB8
:10900000DD1C0D2C000CEE08FF088091481628E8A6
:1090100030E04901881A910887FD9394880C991CC7
:10902000880C991C092C000CAA08BB0880914716D3
:109030008F3FC1F090E0FC01EE0FFF1F8E0F9F1FCE
:10904000FC01E652FA4E2181328183E0220F331F68
:109050008A95E1F794E0369527959A95E1F72E5F8A
:109060003F4F02C020E030E02F5F3F4FC901330F78
:10907000AA0BBB0B9C01AD01281939094A095B09F0
:10908000A4EBB0E00F947E27A701960128193909B7
:109090004A095B090F945F27B90182E79CE00E94AF
:1090A000C75C8AE00E94CBF890C30E94E75CB801DD
:1090B0008BE69CE00E94C75C8CE59CE00E94025C11
:1090C00084C38AE50E9432D08111E4C583E50E9401
:1090D00032D08111DFC579C360E085E40E946FACB6
:1090E000811173C080E50E94E9CF882351F00E946E
:1090F000B2CF6093400C7093410C8093420C9093DC
:10910000430C89E40E94E9CF882381F00E94B2CF0A
:109110002CEA35EC47E25EE30F944D216093440C5A
:109120007093450C8093460C9093470C84E40E9406
:10913000E9CF882381F00E94B2CF2CEA35EC47E2D8
:109140005EE30F94D7286093480C7093490C80938A
:109150004A0C90934B0C0E94EB5C4091400C509158
:10916000410C6091420C7091430C88EA9CE00E9493
:10917000B65C2CEA35EC47E25EE36091440C7091FA
:10918000450C8091460C9091470C0F94D728AB0169
:10919000BC0184EA9CE00E94B65C2CEA35EC47E214
:1091A0005EE36091480C7091490C80914A0C90915B
:1091B0004B0C0F944D21AB01BC0180EA9CE00E9456
:1091C000B65C8AE00E94CBF800C30E94E75C8EE8A0
:1091D0009CE00E94025CF9C280E50E94E9CF8823EE
:1091E00051F00E94B2CF60930509709306098093F5
:1091F00007099093080989E40E94E9CF882381F048
:109200000E94B2CF2CEA35EC47E25EE30F944D2189
:109210006093090970930A0980930B0990930C09D4
:1092200084E40E94E9CF882381F00E94B2CF2CEA27
:1092300035EC47E25EE30F94D72860930D097093F5
:109240000E0980930F09909310090E94EB5C4091E6
:10925000050950910609609107097091080984EB8E
:109260009CE00E94B65C2CEA35EC47E25EE360913C
:10927000090970910A0980910B0990910C090F94CA
:10928000D728AB01BC0180EB9CE00E94B65C2CEAC5
:1092900035EC47E25EE360910D0970910E09809113
:1092A0000F09909110090F944D21AB01BC018CEA7C
:1092B0009CE00E94B65C8AE00E94CBF886C283E5FF
:1092C0000E94E9CF182F882371F00E94B2CF0F942B
:1092D0004929709325026093240221E0672B09F04D
:1092E00020E02093340C80E50E94E9CF882359F0D8
:1092F0002091240230912502232B11F00E942E652B
:109300008093340C62C2111160C20E94EB5C84ED48
:109310009CE00E94025C8091340C882319F08CEB55
:109320009CE002C088EB9CE00E94025C60912402F9
:109330007091250283EC9CE00E94C75C8FEB9CE05F
:109340000E94025C42C20E942B863FC20E9443C818
:109350003CC281E00E94AFAB0E94CFF336C2809145
:109360004E12887809F0FBC480915012867009F083
:10937000F6C425C56FEF7FEF89E40E9460ACF82E3C
:109380006FEF7FEF8AE40E9460ACE82E8AE50E94CE
:10939000E9CF182F811105C081E50E94E9CFB82ED1
:1093A00001C0B12CF7FC06C0E7FC04C0111109C0D4
:1093B000B11007C00E94E75C8EE39DE00E94025C52
:1093C00004C2F4E0FF1510F0FE1538F40E94E75CCB
:1093D0008FE19DE00E94025CF8C1CF2C0F2C000CA5
:1093E000DD080E2D0E2C000C110B0E94B2CFBB20FD
:1093F00099F025E02C9DF0012D9DF00D1124E00F3A
:10940000F11FEE0FFF1FEE0FFF1FE45AFB4E2081EE
:1094100031814281538103C020E030E0A9010F94E3
:10942000DD279B01AC0185E08C9DF0018D9DF00D49
:109430001124E00FF11FEE0FFF1FEE0FFF1FE45A84
:10944000FB4E20833183428353836E2D8F2D0E94E8
:109450004784BBC10E949FE78111B7C10DE11AE2A9
:1094600027E732E03DA32CA3CE0101965C0142E741
:10947000842E4AE2942E1C01F80165917591859124
:109480009491ACA1BDA1CD90DD90ED90FD90BDA3D8
:10949000ACA3A70196010F94DC272B013C01F1013D
:1094A000608371838283938320E030E040EA51EC53
:1094B0000F943D2A87FD0AC020E030E040EA51E4E5
:1094C000C301B2010F94E72018162CF4F401849123
:1094D00018160CF498C4D101CD90DD90ED90FD905C
:1094E0001D0120E030E040EA51ECC701B6010F94C5
:1094F0003D2A87FD0AC020E030E040EA51E4C70180
:10950000B6010F94E720181664F40E94E75C8CE71C
:109510009DE00E94025C61E08EE69DE00F942E0EBD
:1095200054C10C5F1F4FBFEF8B1A9B0AEAE209324E
:109530001E0709F0A1CF39E2E32E39E0F32E10E047
:10954000F50181919191A191B1915F01F701819311
:109550009193A193B1937F01812F0E94CFCD1F5F83
:10956000133071F70E94CFF360E08EE59DE00F9419
:109570002E0E2BC10E943BFF28C10E9402FB25C179
:1095800081E080934B140E94C26F10924B14882389
:1095900009F41BC10E94EB5C8AE99DE00E94025C19
:1095A00014C180915B1882FF10C1806280935B18A8
:1095B0000CC18AE50E9432D0882331F10E94B2CFDB
:1095C0006B017C0120E030E040EA51EC0F943D2A31
:1095D00087FD13C020E030E040EA51E4C701B60146
:1095E0000F94E72018164CF0C092D513D092D613E2
:1095F000E092D713F092D813E8C00E94E75C85EAA6
:109600009DE00E94025CE1C00E94EB5C4091D5139A
:109610005091D6136091D7137091D81382EC9DE0CE
:109620000E94B65C8AE00E94CBF8CFC00E94B7E0EF
:10963000082F87FDCAC085E50E94E9CF8823B1F1D4
:10964000E02E002E000CFF080E94B2CF4B015C01FF
:1096500020E030E0A9010F943D2A87FF04C0B7FA4B
:10966000B094B7F8B094C70123E0880F991F2A95EA
:10967000E1F79C012C5A3B4E7901D9018D929D92C4
:10968000AD92BC92139720E030E04AEF53E4C5015D
:10969000B4010F943D2A18164CF480E090E0AAEF34
:1096A000B3E4F70180839183A283B3838CE40E94A7
:1096B000E9CF882309F489C0002E000C110B0E9409
:1096C000B2CF6B017C0120E030E0A9010F943D2A6C
:1096D00087FF04C0F7FAF094F7F8F09420E030E048
:1096E0004AEF53E4C701B6010F943D2A980193E075
:1096F000220F331F9A95E1F7F901EC5AFB4E181629
:109700002CF0C482D582E682F7825FC080E090E0D0
:10971000AAEFB3E484839583A683B78356C08BE412
:109720000E9432D0882329F10E94B2CF6B017C01C4
:1097300020E030E0A9010F943D2A87FD15C020E00C
:1097400030E040E251E4C701B6010F94E72018165B
:109750005CF00E9443C8C0924C0CD0924D0CE09239
:109760004E0CF0924F0C31C083ED9DE00E94025CE4
:109770002CC00E94EB5C40914C0C50914D0C6091C0
:109780004E0C70914F0C82EF9DE00E94B65C8AE017
:109790000E94CBF81AC081E08093870210921A14BD
:1097A00060E083E50E94E96681110FC00E9481BDDF
:1097B0000CC00E9477A109C080915212882329F021
:1097C0000E948E8202C00E9477A12296FFAD22974E
:1097D000F11102C00E942CBD2CAD2093F7081EC3CE
:1097E0000E9443C83091AC183CAB80E00E94D0D5B9
:1097F0000E9422F281E0809326090E945CF588E5B0
:109800000E94E9CF182F89E50E94E9CF082F8AE549
:109810000E94E9CF101384C1181711F0012F80C1E5
:1098200001E011E091E09CA70E94106482E50E9493
:1098300032D0882361F00E94B2CF6B017C0120E01E
:1098400030E0A9010F94E720882369F106C0C12CFC
:10985000D12C30E8E32E30E4F32E111103C00023A5
:1098600009F4FCC0C092C113D092C213E092C3139A
:10987000F092C413A701960160917F02709180025B
:1098800080918102909182020F94E72087FF0BC0A4
:1098900019821A821B821C82BE016F5F7F4F81EC8E
:1098A00093E10E9424F3112309F4D3C0002309F4A7
:1098B000CDC010927B0210927C0210927D02109219
:1098C0007E02109277021092780210927902109222
:1098D0007A020E94CDF3E2E7FAE2A491A8AFE6E6AD
:1098E000FAE2C590D590E590F490EAE6FAE2859028
:1098F0009590A590B490A5019401C701B6010F946D
:109900003D2A18162CF4A7019601C501B40104C024
:10991000A5019401C701B6010F94D7282B013C0182
:10992000EDE2FAE285919591A591B4918CA39DA366
:10993000AEA3BFA3E9E2FAE285919591A591B49116
:1099400088A799A7AAA7BBA79C01AD016CA17DA17F
:109950008EA19FA10F943D2A181634F428A439A48F
:109960009AA598AB1BA505C02CA03DA0AEA1A8ABA5
:109970001FA1A3019201C301B2010F944D2120E068
:1099800030E040E85FE30F94DD270F948B2A9101CC
:1099900048A9512F0F944D2168A379A38AA39BA3B3
:1099A000E3E7FAE2149120E030E040EC5FE3C50128
:1099B000B4010F944D214B015C01612F110F770B06
:1099C000880B990B0F94EE209B01AC01C501B401EB
:1099D0000F944D2169837A838B839C8320E030E050
:1099E00040EC5FE3C701B6010F944D216B017C0190
:1099F000B8AD6B2FBB0F770B880B990B0F94EE2034
:109A00009B01AC01C701B6010F944D216C8F7D8F76
:109A10008E8F9F8FAE01405E5F4FBE016F5F7F4FA5
:109A2000CE014C960E9402F30E94F7FA10927B023C
:109A300010927C0210927D0210927E0210927702A8
:109A4000109278021092790210927A0280E00E94BD
:109A5000EFCD002319F081E00E94EFCDECA5EE23BD
:109A600009F450C080E00E9454D58091C8148370DE
:109A7000833061F060E08AEA97E00F942E0E0E9436
:109A8000EB5C8BE997E00E94025C3AC00E94CDF348
:109A900080917F0290918002A0918102B091820218
:109AA0008093C1139093C213A093C313B093C413B4
:109AB00080E090E0A6EBB2E48093B9139093BA13E0
:109AC000A093BB13B093BC1380E090E0A8E6B2E48F
:109AD0008093BD139093BE13A093BF13B093C01394
:109AE00019821A821B821C82AE014F5F5F4F6DEBA1
:109AF00073E189EB93E10E9402F382E00E94EFCDD3
:109B00000E9467AB0E94CDF38091250980932609BE
:109B10008CA90E94D0D50E9409F20E94CFF355CEA5
:109B20008CA782CE61E08EE698E00E943FD089EF5C
:109B300097E00F949C1061E08CE699E30E943FD07F
:109B40008AEE97E00E94125DB1100C94B1400C9423
:109B5000AA4080E00E94C15D0C94DD4088E50E942F
:109B6000E9CF81115F9889E50E94E9CF81118A9838
:109B70008AE50E94E9CF882329F08091080181704D
:109B80008093060185E40E94E9CF882309F41DCE65
:109B900012981BCE0E948ACFAB01BC01409357188C
:109BA000509358186093591870935A1886E695E1A7
:109BB0000E94457A0ACE61E0802F0E94C7EC6F2D8B
:109BC000802F0E9498EC6F2D70E0802F0E9403ED93
:109BD00047E0E41203C0F092230CF7CD89E0E812CD
:109BE000F4CDF092220CF1CD0E949ACF90E0853610
:109BF000910514F084E690E08093831EE6CD0E94E8
:109C0000A0C60C941844A3019201C501B4010F949D
:109C10003D2A18163CF089ED99E060E00F942E0E75
:109C20000C94384486EE99E0F8CF0E94B2CF0F949E
:109C30004929CB010E9402640E94B2CF20E030E0AB
:109C400040EA50E40F943D2A181614F40E94A0C66E
:109C50006091020970910309072E000C880B990B83
:109C60000F94EE202091FE083091FF0840910009EA
:109C7000509101090F943D2A18161CF48EE19AE0C8
:109C800002C08FE09AE060E00F942E0E812F0E94B8
:109C900006D79BCD0E94B2CF20E030E040E050ECF0
:109CA0000F94E72087FD15C00E94B2CF20E030E07E
:109CB00040E050E40F943D2A18162CF00E94B2CFD9
:109CC0006B017C010BC0C12CD12CE12C10E4F12ED6
:109CD00005C0C12CD12CE12CB0ECFB2E20919F11A2
:109CE0003091A0114091A1115091A211C701B6016C
:109CF0000F944D210F944929CB010F94FA0280E56E
:109D00000E94E9CF882329F00E942E65882309F458
:109D10005CCDA70196016091D5137091D613809107
:109D2000D7139091D8130F94DD276093D5137093B8
:109D3000D6138093D7139093D8130E94EB5C409175
:109D4000D5135091D6136091D7137091D8138DE726
:109D50009CE00E94B65C8AE00E94CBF836CD88E495
:109D60000E94E9CF882321F00E942E658093F50898
:109D700082E50E94E9CF082F83E50E94E9CF182FE2
:109D8000011102C0882351F01092F8080E9461F678
:109D9000112321F00E942E658093260284E40E9404
:109DA000E9CF882309F411CD0E94B2CF60937302EA
:109DB00070937402809375029093760206CD0E9490
:109DC000EB5C8EE09DE00E94025C80912602811196
:109DD00017C087EE9CE00E94025C8AE00E94CBF8EC
:109DE00040917302509174026091750270917602F5
:109DF0008EEE9CE00E94B65C8AE00E94CBF8E5CC37
:109E00008BEE9CE0E8CFF7FAF094F7F8F094D101EC
:109E1000CD92DD92ED92FC9213975DCBCF5BDF4F3D
:109E20000FB6F894DEBF0FBECDBFDF91CF911F916B
:109E30000F91FF90EF90DF90CF90BF90AF909F90E9
:109E40008F907F906F905F904F903F902F900895EC
:109E5000CF92DF92EF92FF920F931F93CF93DF93F6
:109E60006C017A018B01C0E0D0E0CE15DF0581F0F6
:109E7000D8016D918D01D601ED91FC910190F08199
:109E8000E02DC6011995892B11F02196EECF7E01A8
:109E9000C701DF91CF911F910F91FF90EF90DF905D
:109EA000CF900895089580E090E00895FC01538DCF
:109EB000448D252F30E0842F90E0821B930B5417A4
:109EC00010F0CF96089501970895FC01918D828D31
:109ED000981761F0828DDF01A80FB11D5D968C91FE
:109EE000928D9F5F9F73928F90E008958FEF9FEF09
:109EF0000895FC01918D828D981731F0828DE80FC5
:109F0000F11D858D90E008958FEF9FEF0895FC017E
:109F1000918D228D892F90E0805C9F4F821B91094B
:109F20008F739927089589EC94E10E94874F21E06F
:109F3000892B09F420E0822F0895FC01848DDF0134
:109F4000A80FB11DA35ABF4F2C91848D90E00196AC
:109F50008F739927848FA689B7892C93A089B1899B
:109F60008C91837080648C93938D848D981306C03C
:109F70000288F389E02D80818F7D80830895EF92A0
:109F8000FF920F931F93CF93DF93EC0181E0888FB3
:109F90009B8D8C8D981305C0E889F989808185FD9A
:109FA00026C0F62E0B8D10E00F5F1F4F0F73112789
:109FB000E02E8C8DE8120CC00FB607FCFACFE889B2
:109FC000F989808185FFF5CFCE010E949D4FF1CFA9
:109FD0008B8DFE01E80FF11DE35AFF4FF0829FB712
:109FE000F8940B8FEA89FB89808180620AC09FB751
:109FF000F894EE89FF896083E889F989808183700C
:10A00000806480839FBF81E090E0DF91CF911F91BA
:10A010000F91FF90EF900895CF93DF93EC01888D1F
:10A020008823C9F0EA89FB89808185FD05C0A8895C
:10A03000B9898C9186FD0FC00FB607FCF5CF8081E2
:10A0400085FFF2CFA889B9898C9185FFEDCFCE012C
:10A050000E949D4FE7CFDF91CF91089580E090E07F
:10A06000892B41F080E090E0892B21F00E940000D4
:10A07000811121C080E090E0892B41F080E090E0E8
:10A08000892B21F00E940000811118C080E090E02F
:10A09000892B21F00E94934F811113C080E090E042
:10A0A000892BA1F080E090E0892B81F00E940000D4
:10A0B00081110AC008950E940000DCCF0E940000B8
:10A0C000E5CF0E940000EACF0C9400000895FC0147
:10A0D00020E03EE2DB014C91403241F0283011F4A7
:10A0E00030833196DB014C91408331962F5F6F5F57
:10A0F0007F4F2B3079F7108208950F94EF2A0F933A
:10A100001F93CF93DF938B01EA01DB016D917C916B
:10A110000E944B7BD801ED91FC9111979081888131
:10A12000992349F0893638F43196ED93FC93888170
:10A130008F5F8883EFCF893658F48FE28083F801F0
:10A140008081918101969183808388818F5F88834C
:10A15000DF91CF911F910F9108951F920F920FB62B
:10A160000F9211240BB60F922F933F934F935F934F
:10A170006F937F938F939F93AF93BF93EF93FF93CF
:10A1800089EC94E10E949D4FFF91EF91BF91AF91B7
:10A190009F918F917F916F915F914F913F912F91FF
:10A1A0000F900BBE0F900FBE0F901F9018951F922F
:10A1B0000F920FB60F9211240BB60F922F938F931D
:10A1C0009F93EF93FF93E091D914F091DA1480817B
:10A1D000E091DF14F091E01482FD12C09081809133
:10A1E000E2148F5F8F732091E314821751F0E09196
:10A1F000E214F0E0E753FB4E958F8093E21401C028
:10A200008081FF91EF919F918F912F910F900BBEC5
:10A210000F900FBE0F901F9018958BE1EFEBF5E1BB
:10A22000A4EAB5E101900D928A95E1F70895809135
:10A230005B1882FF1FC088E890E10E94025C609179
:10A240005718709158188091591890915A184AE0EF
:10A250000E94D2F88FE20E94CBF86091531870915F
:10A26000541880915518909156184AE00E94D2F8DF
:10A270000C94D0F98AE990E10C94025C1092BC0A2B
:10A2800080915B188F7D8B7F80935B180E94608D1F
:10A29000882321F086E695E10C94B17D08958091A4
:10A2A0005B1883FF03C0846080935B180895CF928E
:10A2B000DF92EF92FF920F931F93CF93DF93CDB76F
:10A2C000DEB7EDB6FEB6DC010D900020E9F79D018A
:10A2D000281B390B2C5F3F4F4DB75EB7421B530B0A
:10A2E0000FB6F8945EBF0FBE4DBF0DB71EB70F5F20
:10A2F0001F4F9F938F9384E89FE09F938F931F93AB
:10A300000F930F947F20680154E0C50ED11C0F906D
:10A310000F900F900F900F900F90F601808188237F
:10A3200049F0082E000C990B0F94F42AF601819342
:10A330006F01F3CFC8010E946FBF80E89FE00E94C9
:10A34000A1BF0FB6F894FEBE0FBEEDBEDF91CF9158
:10A350001F910F91FF90EF90DF90CF9008958F9213
:10A360009F92AF92BF92CF92DF92EF92FF92CF93E4
:10A3700080915B18877F80935B188091C21588233A
:10A3800021F08FEB95E10E94B17D1092A315109200
:10A39000A01585E380939F150E9425EE6B017C013B
:10A3A00020EDC20E27E0D21EE11CF11CA89561E051
:10A3B00080919F150E9498EC61E080919F150E940A
:10A3C000C7EC209A289A219A2398229A81E00E9429
:10A3D000E6FA85E08093A1150E94E6FACAE08FEFC5
:10A3E0000E94DAFAC150D9F7A89520E030E0A9011F
:10A3F00060E08FE995E10E94917C8093A215813005
:10A4000061F00E9425EEDC01CB018C199D09AE099B
:10A41000BF09B7FDEACF81E062C0A8952AEA31E022
:10A4200040E050E068E08FE995E10E94917C853042
:10A4300011F481E00AC0C4E00E94DFFA8093A21503
:10A44000C150D1F78A3A61F482E08093A315A895B0
:10A450008091A315823081F0812C912C540111C080
:10A460000E9425EEDC01CB018C199D09AE09BF09C4
:10A47000B7FDD4CF82E033C0812C912CA12C80E495
:10A48000B82E20E030E0A90167E38FE995E10E9452
:10A49000917CA501940169E28FE995E10E94917C8C
:10A4A0008093A215882361F00E9425EEDC01CB0188
:10A4B0008C199D09AE09BF09B7FDE3CF8AE00FC033
:10A4C0008091A315823021F520E030E0A9016AE3F4
:10A4D0008FE995E10E94917C882361F088E0809368
:10A4E000A0158FE995E10E94897C0E94EB5C82E7D0
:10A4F0009FE022C00E94DFFA807C803C19F483E058
:10A500008093A3150E94DFFA0E94DFFA0E94DFFA0F
:10A510008FE995E10E94897C1092A11581E00F944A
:10A520003A0581110CC080E00F943A05811107C0F3
:10A530000E94E75C8EE59FE00E94025C1AC061E821
:10A5400075E18FEB95E10E94DC7A811105C00E94D4
:10A55000E75C8DE49FE0F0CF80915B18886080938A
:10A560005B180E94EB5C81E49FE00E94025C0E9409
:10A5700072F6CF91FF90EF90DF90CF90BF90AF90A9
:10A580009F908F900C940D512F923F925F926F92FB
:10A590007F928F929F92AF92BF92CF92DF92EF9273
:10A5A000FF920F931F93CF93DF93CDB7DEB7C356C0
:10A5B000D1090FB6F894DEBF0FBECDBF8C016B0181
:10A5C0004A012DB63EB6512C7E0187E5E80EF11CFE
:10A5D000F6018381823008F41FC180859185A285B0
:10A5E000B3858F719927AA27BB27892B8A2B8B2BA1
:10A5F00009F012C11092BC1A4CEB5AE1BE016F5F18
:10A600007F4FC6010E94467F18160CF005C18C854D
:10A61000982F9871903129F420912A0B21502230E3
:10A6200078F42981222309F4F7C0253E89F22E32DD
:10A6300079F22091BC1A2E3259F28A7049F67CC008
:10A640006DB67EB6BE016F5F7F4FC7010E94675037
:10A650000115110521F0F8018081811163C021E00D
:10A6600081E090E0F70101900020E9F73197EE19C1
:10A67000FF09E80FF91F32968DB79EB78E1B9F0B0F
:10A680000FB6F8949EBF0FBE8DBFEDB7FEB73196E3
:10A690005F01211102C0B80102C060E976E0C50186
:10A6A0000F943B2BB701C5010F94252B60E976E091
:10A6B000C5010F94252B19A21CA221E0A701B60108
:10A6C000CE0181960E949D8181110DC080912A0B3F
:10A6D000811109C00E94EB5C8DE29FE00E94025C48
:10A6E000C7010E94D6F98BE1FE01B196DE01DC962E
:10A6F00001900D928A95E1F740E050E0BE01645C64
:10A700007F4FC5010E94C452CE01CC960E94BA7DF3
:10A71000CE0181960E94BA7D0FB6F8947EBE0FBE20
:10A720006DBE56CFF80101900020E9F73197CF01B7
:10A73000801B910B20E096CF21E0903109F020E0C2
:10A7400080915B1820FB84F980935B18903141F075
:10A750008985873409F03CCF8A858E3709F438CF54
:10A7600080912A0B813021F068F08230C1F130CF26
:10A7700080912D0B90912E0B019690932E0B809330
:10A780002D0B26CFBE016F5F7F4F8EEF9AE10E94A7
:10A7900067500115110529F48EEFA82E8AE1B82E15
:10A7A00009C05801F50181915F018823A9F30E9436
:10A7B000CBF8F8CFF50181915F01882319F00E9451
:10A7C000CBF8F8CF80E20E94CBF86D8D7E8D8F8D17
:10A7D00098A14AE00E94D2F80E94D0F9F9CEBE01B9
:10A7E0006F5F7F4F8EEF9AE10E9467508114910452
:10A7F00041F06EEF7AE1C4010F94122B892B51F4D2
:10A800000BC0852D90E020912B0B30912C0B8217E3
:10A81000930711F05394DCCE0FB6F8943EBE0FBEF2
:10A820002DBECD59DF4F0FB6F894DEBF0FBECDBFA2
:10A83000DF91CF911F910F91FF90EF90DF90CF901C
:10A84000BF90AF909F908F907F906F905F903F9060
:10A850002F900895CF93DF93CDB7DEB76B970FB6E8
:10A86000F894DEBF0FBECDBF81E080932A0B10921B
:10A870002E0B10922D0B84EA95E10E94847C8BE1D3
:10A88000E4EAF5E1DE01119601900D928A95E1F777
:10A8900040E050E0BE016F5F7F4F80E090E00E949B
:10A8A000C452CE0101960E94BA7D80912D0B9091E9
:10A8B0002E0B6B960FB6F894DEBF0FBECDBFDF91A7
:10A8C000CF9108950F931F93CF93DF93CDB7DEB74A
:10A8D0006B970FB6F894DEBF0FBECDBF8B0122E0A1
:10A8E00020932A0B90932C0B80932B0B84EA95E1F9
:10A8F0000E94847C8BE1E4EAF5E1DE01119601908F
:10A900000D928A95E1F7A801BE016F5F7F4F80E04D
:10A9100090E00E94C452CE0101960E94BA7D6B96CF
:10A920000FB6F894DEBF0FBECDBFDF91CF911F9160
:10A930000F910895DF92EF92FF920F931F93CF93A1
:10A94000DF9300D01F92CDB7DEB720915B1823FFB5
:10A950003DC1F42EE62E8C010E94608D882309F4FF
:10A9600081C0FF2009F48CC080915218882351F0D7
:10A970000E94E75C83E490E10E94025C80E090E04A
:10A980000E94125D82EC9AE09A8389838FE2809321
:10A99000C10A81E08B83F12C9BE1D92E8091511863
:10A9A000F81678F4DF9CC0011124AE014D5F5F4FB3
:10A9B000BE016F5F7F4F8D5B984E0E947F50F39476
:10A9C000EDCF8B818B3578F4AE014D5F5F4FBE01CB
:10A9D0006F5F7F4F86E695E10E947F5089819A8163
:10A9E00001979A838983E981FA811082E091521854
:10A9F00084E0E89FF0011124E354F54F809157184B
:10AA000090915818A0915918B0915A188083918349
:10AA1000A283B3830E94EB5CB8018AE290E10E94BA
:10AA2000D45C6091521889E6689FB00111246F537D
:10AA3000754F8FE190E10E94D45C4091571850917E
:10AA400058186091591870915A1889E190E10E9444
:10AA5000985C8AE00E94CBF8809152188F5F8093B7
:10AA6000521826C0FF2039F00E94EB5C89E090E18B
:10AA70000E94025C1DC01092521882E0F82E02C0A3
:10AA8000FF24F3940E94EB5C84E090E10E94025C5E
:10AA900081E0F81609F497C080EF9FE00E94025C05
:10AAA000B8018CEF9FE00E94D45C8AE00E94CBF852
:10AAB0000E943E51B801CE0103960F9412028C0100
:10AAC000009709F483C06B817C81EE2009F450C0AB
:10AAD00021E0AC0186E695E10E949D81882309F47E
:10AAE0003FC08091771590917815A0917915B0911C
:10AAF0007A158093531890935418A0935518B093D7
:10AB000056181092571810925818109259181092FF
:10AB10005A18B80182EE9FE00E94D45C409153180D
:10AB20005091541860915518709156188AED9FE015
:10AB30000E94985C8AE00E94CBF88BEC9FE00E9418
:10AB4000025CB80180E090E00E9462548091BC1ADF
:10AB5000811102C0C80102C08CEB9AE160E030C0F4
:10AB6000B80187EB9FE00E94D45C84EB9FE00FC0AC
:10AB700026E5AC0186E695E10E949D8181110AC01F
:10AB8000B80180EA9FE00E94D45C8DE99FE00E94BA
:10AB9000025C1CC080915B18816080935B18B801D7
:10ABA00080E090E00E94625410924117B8018BE857
:10ABB0009FE00E94D45C8AE00E94CBF860E0C8016C
:10ABC0000F94890E03C086EF9FE068CF0F900F901F
:10ABD0000F900F90DF91CF911F910F91FF90EF9009
:10ABE000DF900895CF92DF92EF92FF92CF936B01A7
:10ABF0007C01C42F8091B11A9091B21AA091B31A1E
:10AC0000B091B41A8C159D05AE05BF05D1F00E9418
:10AC10003E7D811102C080E018C021EB38E1B70110
:10AC2000A6018091BA1A9091BB1A0E94C07D882318
:10AC300091F3C092B11AD092B21AE092B31AF09284
:10AC4000B41A81E0C1118093B91ACF91FF90EF90AF
:10AC5000DF90CF9008954F925F926F927F928F9284
:10AC60009F92AF92BF92CF92DF92EF92FF920F939B
:10AC70001F93CF93DF93EC014230510561057105BD
:10AC800010F480E069C089859A85AB85BC85019602
:10AC9000A11DB11D84179507A607B70790F38F89EB
:10ACA000803149F4852E962EA72EBB248B899C8952
:10ACB000AD89BE890FC0803221F78B889C88AD8812
:10ACC000BE88DB01CA01E7E0B695A7959795879501
:10ACD000EA95D1F7880E991EAA1EBB1E28013901DC
:10ACE0006A017B0141E0C501B4010E94F25588234D
:10ACF00041F29F89903161F4DD24EE24FF24960116
:10AD0000220F331FF901EF54F74E5182408211C0D8
:10AD1000E894C7F8DD24EE24FF249601220F331FA8
:10AD2000220F331FF901EF54F74E408251826282A5
:10AD300073829A89923080F04D815E816F8178852F
:10AD4000840E951EA61EB71E8092B51A9092B61A52
:10AD5000A092B71AB092B81ADF91CF911F910F91BC
:10AD6000FF90EF90DF90CF90BF90AF909F908F902B
:10AD70007F906F905F904F900895CF92DF92EF9207
:10AD8000FF920F931F93CF93DF93FC0181859285F0
:10AD9000A385B4850196A11DB11D84179507A6074B
:10ADA000B70710F480E061C08789803149F4BB2780
:10ADB000A72F962F852FC388D488E588F6880FC0E3
:10ADC000803281F783899489A589B6896A017B01DC
:10ADD000C7E0F694E794D794C794CA95D1F78C0D41
:10ADE0009D1DAE1DBF1DE9016A017B018F014091D0
:10ADF000B11A5091B21A6091B31A7091B41A8417B3
:10AE00009507A607B70739F040E0BC01CD010E94C5
:10AE1000F255882339F2F8018789803179F4B70136
:10AE2000A601552766277727440F551FFA01EF54CF
:10AE3000F74E80819181A0E0B0E012C0B701A60179
:10AE40004F77552766277727440F551F440F551F07
:10AE5000FA01EF54F74E80819181A281B381BF70D6
:10AE600088839983AA83BB8381E0DF91CF911F916F
:10AE70000F91FF90EF90DF90CF9008954F925F92E7
:10AE80006F927F92AF92BF92CF92DF92EF92FF923A
:10AE90000F931F93CF93DF9300D01F92CDB7DEB7F0
:10AEA0008C0149835A836B837C835901C12CD12C3B
:10AEB0007601412C82E0582E612C712C49815A81F7
:10AEC0006B817C819E012F5F3F4FC8010E94BD5660
:10AED000882341F1D301C201F801058404C0880F21
:10AEE000991FAA1FBB1F0A94D2F7C80ED91EEA1ECB
:10AEF000FB1E49815A816B817C818789803139F4BD
:10AF000081E0483F5F4F6105710538F4D7CF81E09C
:10AF1000483F5F4F6F4F7F4088F2F501C082D1827A
:10AF2000E282F3820F900F900F900F90DF91CF91FC
:10AF30001F910F91FF90EF90DF90CF90BF90AF9057
:10AF40007F906F905F904F9008954F925F926F92B5
:10AF50007F928F929F92AF92BF92CF92DF92EF92A9
:10AF6000FF920F931F93CF93DF93EC016091EE0B51
:10AF70007091EF0B072E000C880B990B0F94EE20AD
:10AF80009B01AC01688179818A819B810F94DC27C8
:10AF90006B017C016091F00B7091F10B072E000C9E
:10AFA000880B990B0F94EE209B01AC016C817D8185
:10AFB0008E819F810F94DC274B015C012091180248
:10AFC0003091190240911A0250911B02C701B6013B
:10AFD0000F94E720882309F467C0C0921802D0922A
:10AFE0001902E0921A02F0921B022091700B30912C
:10AFF000710B4091720B5091730BC701B6010F9406
:10B000004D212B013C010F947F296B017C0120E035
:10B0100030E0A9010F94E72087FD11C020E030E067
:10B0200040E850E4C701B6010F943D2A181654F4C5
:10B03000C12CD12CC0E8EC2EC0E4FC2E03C0C12CE6
:10B04000D12C7601A7019601C301B2010F94DC2730
:10B050002B013C0120E030E0A9010F94E72087FD9F
:10B0600009C040926C0B50926D0B60926E0B709207
:10B070006F0B08C010926C0B10926D0B10926E0B40
:10B0800010926F0BC701B6010F94492960936B0BA7
:10B09000062E000C770B6F5F7F4F6430710514F044
:10B0A00064E070E060936A0B209114023091150205
:10B0B0004091160250911702C501B4010F94E72088
:10B0C000D091130210916B0B811103C0D11368C092
:10B0D00028C18092140290921502A0921602B0929A
:10B0E00017022091740B3091750B4091760B5091A3
:10B0F000770BC501B4010F944D214B015C010F94F6
:10B100007F296B017C0120E030E0A9010F94E7204A
:10B1100087FD11C020E030E040E850E4C701B601EF
:10B120000F943D2A181654F4C12CD12CB0E8EB2E04
:10B13000B0E4FB2E03C0C12CD12C7601A7019601EF
:10B14000C501B4010F94DC274B015C0120E030E025
:10B15000A9010F94E72087FD09C08092660B9092A9
:10B16000670BA092680BB092690B08C01092660B37
:10B170001092670B1092680B1092690BC701B60111
:10B180000F9449296093650B062E000C770B6F5FB7
:10B190007F4F6430710514F064E070E06093640BDD
:10B1A000C091650BD11305C0809112028C1709F470
:10B1B0006EC010931302C09312020C2E000CDD0B14
:10B1C00085E0F82E2F2D1203C0011124FC01EC0F95
:10B1D000FD1FEE0FFF1FEE0FFF1FE45AFB4E2081F5
:10B1E0003181428153812093600B3093610B4093F6
:10B1F000620B5093630B0091640B002E000C110B3B
:10B20000FC01E00FF11FEE0FFF1FEE0FFF1FE45ACE
:10B21000FB4E60817181828193810F94DC27609362
:10B220005C0B70935D0B80935E0B90935F0B209192
:10B230006A0B3F2D2303F0011124CE0FDF1FCC0F2B
:10B24000DD1FCC0FDD1FC45ADB4E288139814A81B6
:10B250005B812093580B3093590B40935A0B5093BA
:10B260005B0BE00FF11FEE0FFF1FEE0FFF1FE45A05
:10B27000FB4E60817181828193810F94DC27609302
:10B28000540B7093550B8093560B9093570B8090F3
:10B29000660B9090670BA090680BB090690B2091A3
:10B2A0005C0B30915D0B40915E0B50915F0BC501C3
:10B2B000B4010F944D212091600B3091610B4091AE
:10B2C000620B5091630B0F94DD276B017C0160933F
:10B2D000500B7093510B8093520B9093530B209112
:10B2E000540B3091550B4091560B5091570BC501A3
:10B2F000B4010F944D212091580B3091590B40917E
:10B300005A0B50915B0B0F94DD27A70196010F9408
:10B31000DC2760934C0B70934D0B80934E0B9093F6
:10B320004F0B20914C0B30914D0B40914E0B509197
:10B330004F0B60916C0B70916D0B80916E0B909127
:10B340006F0B0F944D212091500B3091510B409178
:10B35000520B5091530B0F94DD27DF91CF911F912A
:10B360000F91FF90EF90DF90CF90BF90AF909F90A4
:10B370008F907F906F905F904F900895CF92DF9263
:10B38000EF92FF926091501470915114072E000CAF
:10B39000880B990B0F94EE206B017C012DEB37E3AA
:10B3A00046E855EB0F943D2A87FD0AC02DEB37E3A5
:10B3B00046E855E3C701B6010F94E72018164CF490
:10B3C000A701960160E070E080E89FE30F94D72822
:10B3D00003C060E070E0CB016093700B7093710B61
:10B3E0008093720B9093730B60915214709153146D
:10B3F000072E000C880B990B0F94EE206B017C013B
:10B400002DEB37E346E855EB0F943D2A87FD0AC044
:10B410002DEB37E346E855E3C701B6010F94E7206B
:10B4200018164CF4A701960160E070E080E89FE3F5
:10B430000F94D72803C060E070E0CB016093740BD9
:10B440007093750B8093760B9093770BFF90EF9032
:10B45000DF90CF9008952F923F924F925F926F921C
:10B460007F928F929F92AF92BF92CF92DF92EF9294
:10B47000FF920F931F93CF93DF93CDB7DEB7609703
:10B480000FB6F894DEBF0FBECDBF8A876B87942EB0
:10B49000A22E282F30E03D872C8770E079876887BF
:10B4A00015E0129FC001139F900D11249F878E8776
:10B4B000FB01E80FF91FEE0FFF1FEE0FFF1FE45A0D
:10B4C000FB4E60817181828193819B01AC010F945D
:10B4D000CF2A882309F44EC14A85490D2B852A0DB0
:10B4E000149FB0011124E885F985E60FF71FEE0FD0
:10B4F000FF1FEE0FFF1FE45AFB4ED080E180F28069
:10B500000381490D149FA0011124E885F985E40FFA
:10B51000F51FEE0FFF1FEE0FFF1FE45AFB4E1081C9
:10B52000918082807380822F90E0EE85FF85E80F06
:10B53000F91FEE0FFF1FEE0FFF1FE45AFB4E608056
:10B5400051803280338139832A0D30E0EE85FF85CA
:10B55000E20FF31FEE0FFF1FEE0FFF1FE45AFB4E2B
:10B56000FF87EE87F081FA83EE85FF85F181FB830B
:10B57000EE85FF85F281FC83EE85FF85F381FD83F7
:10B58000FB01E80FF91FEE0FFF1FEE0FFF1FE45A3C
:10B59000FB4E60816E83B18072817F8383818E8751
:10B5A000FA01E20FF31FEE0FFF1FEE0FFF1FE45A29
:10B5B000FB4E4080A1809281988B2380212F392DD2
:10B5C000482D572D612F792D882D972D0F94CF2A37
:10B5D000882321F010E0912C812C712C2D2D3E2DF3
:10B5E0004F2D502F6D2D7E2D8F2D902F0F94CF2A04
:10B5F000882321F0D12EE92CF82C072D2A813B81BC
:10B600004C815D816A817B818C819D810F94CF2AE1
:10B61000882321F01A821B821C821D82262D352D43
:10B62000432D5981662D752D832D99810F94CF2A35
:10B63000882329F06A805B803C80ED81E983242D9A
:10B640003A2D4889522D642D7A2D8889922D0F9498
:10B65000CF2A882321F0412CA12C188A212C2E815D
:10B660003B2D4F815E856E817B2D8F819E850F9452
:10B67000CF2A882329F04E82BA2CF889FF832E86A0
:10B680002D2D3E2D4F2D502F6D2D7E2D8F2D902F3A
:10B690000F94DD27212F392D482D572D0F94DC27AE
:10B6A0006B017C01262D352D432D5981662D752D7D
:10B6B000832D99810F94DD272A813B814C815D8107
:10B6C0000F94DC279B01AC01C701B6010F94DD2765
:10B6D0003B014C012E813B2D4F815E856E817B2D80
:10B6E0008F819E850F94DD27242D3A2D4889522D78
:10B6F0000F94DC279B01AC01C401B3010F94DD273B
:10B7000020E030E040E450E40F94D7289B01AC01E6
:10B7100085E06C857D85869FF001879FF00D112463
:10B7200088859985E80FF91FEE0FFF1FEE0FFF1FA9
:10B73000E45AFB4E20833183428353836B858A8591
:10B7400060960FB6F894DEBF0FBECDBFDF91CF91EC
:10B750001F910F91FF90EF90DF90CF90BF90AF902F
:10B760009F908F907F906F905F904F903F902F9021
:10B770000C94478460960FB6F894DEBF0FBECDBF21
:10B78000DF91CF911F910F91FF90EF90DF90CF90BD
:10B79000BF90AF909F908F907F906F905F904F90F1
:10B7A0003F902F900895CF92DF92EF92FF926B011E
:10B7B0007C0183E3C816D104E104F10470F082E354
:10B7C000C81AD108E108F10862E370E080E090E077
:10B7D0000E94EBED0F94A007ECCFC701B6010E94C9
:10B7E000EBEDFF90EF90DF90CF900D94A007CF93FB
:10B7F000C82FCC2329F080E20E94CBF8C150F9CFAA
:10B80000CF910895CF93DF93FC018491EF012196AE
:10B81000882321F00E94CBF8FE01F7CFDF91CF9172
:10B8200008958F929F92AF92BF92CF92DF92EF9244
:10B83000FF920F931F93CF93DF938FE292E10E94C9
:10B84000025CC12CD12C760186E00E94F75BC70117
:10B85000B6010E943FF98FEFC81AD80AE80AF80A21
:10B8600095E0C916D104E104F10471F78AE00E9461
:10B87000CBF80CE514E1C12CD12C760180E20E94BA
:10B88000CBF8C701B6010E943FF9C0E0D0E080E2EA
:10B890000E94CBF8F801EC0FFD1F80809180A28000
:10B8A000B380A5019401C501B4010F94CF2A811181
:10B8B00012C020E030E0A901C501B4010F943D2A77
:10B8C00087FD03C08BE20E94CBF843E0C501B401C1
:10B8D0000E945BF909C0B12C80E20E94CBF8B394BE
:10B8E0008DE396E0B912F9CF6496C436D10579F6A6
:10B8F0008AE00E94CBF88FEFC81AD80AE80AF80A43
:10B900000C5F1F4F95E0C916D104E104F10409F062
:10B91000B5CF8AE0DF91CF911F910F91FF90EF900B
:10B92000DF90CF90BF90AF909F908F900C94CBF80A
:10B93000CF92DF92EF92FF926A017B010E94025C3C
:10B940004AE0C701B601FF90EF90DF90CF900C94D2
:10B95000D2F8CF93DF93EB010E94025CBE0180E03E
:10B9600090E04AE0DF91CF910C94D2F8CF92DF9231
:10B97000EF92FF926A017B010E94025C42E0C701E4
:10B98000B601FF90EF90DF90CF900C945BF9CF93CE
:10B99000DF93EB010E94025CBE01DD0F880B990B67
:10B9A000DF91CF910C943FF90F931F93CF93DF93C7
:10B9B0008B010E94025CE8018991882319F00E94A2
:10B9C000CBF8FACFDF91CF911F910F91089588E2C4
:10B9D00092E10C94025C82E292E10C94025C0E947F
:10B9E00086DE0E9404C780911E14882319F080E02F
:10B9F0000E9467E780918702882399F00E94E75CA4
:10BA00008BEA91E10E94025C60E081EA91E10F948F
:10BA10002E0E6EE571E080E090E00E94D35B109204
:10BA200087020895CF93DF93CDB7DEB7A8970FB6FF
:10BA3000F894DEBF0FBECDBF8C010E9486DE0E944F
:10BA4000E75C81E891E10E94025C0115110511F4A7
:10BA500008E711E18091BC0880FD75C0816080938A
:10BA6000BC0882E996E00E94D6F9882483948AE58E
:10BA7000982E9092E0168092DF168FE090E09093DF
:10BA8000E2168093E11697E0A92EA092D31622E841
:10BA9000B22EB092D61634E8C32ED12CE12CF12C64
:10BAA000C092D716D092D816E092D916F092DA1634
:10BAB0000F94B6009092E0168092DF1688E590E031
:10BAC0009093E2168093E116A092D316B092D61608
:10BAD000C092D716D092D816E092D916F092DA1604
:10BAE0000F94B60063E070E080E090E00E942C8448
:10BAF0008AE289838A838B838C83DE011596F80121
:10BB0000CE0101969D01281B390B449131964423A7
:10BB100011F04D93F7CFFC01E20FF31F2AE2AF01C2
:10BB2000481B590B4832510511F02193F8CF40E6DC
:10BB300050E160E070E00F9465006AE070E080E042
:10BB400090E00E942C8461E08FE691E10E943FD05A
:10BB500089EE93E030E6019729F0232F2A95000023
:10BB6000E9F7F9CFF89489EE93E038EE019729F0E0
:10BB7000232F2A950000E9F7F9CF0E9486DEA895C9
:10BB8000FECF2F923F924F925F926F927F928F9251
:10BB90009F92AF92BF92CF92DF92EF92FF920F935C
:10BBA0001F93CF93DF93CDB7DEB727970FB6F894E7
:10BBB000DEBF0FBECDBF8A830E942C1D0E9425EEE2
:10BBC0006B017C0180910102882359F18091F70873
:10BBD000882339F140912F0B5091300B6091310B3C
:10BBE0007091320B97018601041B150B260B370B46
:10BBF00037FD2AC0833079F03CF4813094F00E9404
:10BC0000EB5C8AED90E10BC0843059F40E94EB5C50
:10BC10008BEA90E104C00E94EB5C83EC90E10E940F
:10BC2000025C2091010230E0A8EEB3E00F9491276E
:10BC3000C60ED71EE81EF91EC0922F0BD092300BF5
:10BC4000E092310BF092320B80912602882319F199
:10BC50008091F80881111FC080915B1882FD08C097
:10BC600080916713813021F08091BC0A882399F07C
:10BC7000F8946499C7C36091DC117091DD118091D3
:10BC8000DE119091DF11789420E030E0A9010F944B
:10BC9000E72087FD44C38091BA0A843020F40E94D3
:10BCA000DBBD0E946E8D0E9425EE6B017C014091F0
:10BCB000F1085091F2086091F3087091F408411571
:10BCC00051056105710529F18091C0149091C1144D
:10BCD000A091C214B091C314840F951FA61FB71F63
:10BCE000A7019601281B390B4A0B5B0B57FD11C0AE
:10BCF0000E94E75C6091040C7091050C85E391E172
:10BD00000E94D45C8AE00E94CBF880E090E00E9420
:10BD1000125D4091640250916502609166027091DB
:10BD20006702411551056105710509F44EC09091F6
:10BD30004D1680914E16981759F00E9425EE60938B
:10BD4000C0147093C1148093C2149093C3143DC067
:10BD50008091BC0A811137C00A81011134C08091E1
:10BD6000C0149091C114A091C214B091C314840F57
:10BD7000951FA61FB71FA7019601281B390B4A0B59
:10BD80005B0B57FD20C08091430B81111EC081E0E9
:10BD90008093430B5F9A8091C8148E7F8093C81460
:10BDA0008A9A8091C8148D7F8093C814809108016D
:10BDB00080958170809306018091C8148B7F809359
:10BDC000C814129A02C01092430B80913F0B9091BD
:10BDD000400BA091410BB091420BB701A601481B4B
:10BDE000590B6A0B7B0B77FDCBC190914D1680915F
:10BDF0004E1660915D0220915E02981317C08091EB
:10BE0000220C869FB0011124660F672F661F770BE7
:10BE1000719569836091230C629FB0011124660FB4
:10BE2000672F661F770B71956A8329C080914E1624
:10BE300053E5859FC0011124805B934FFC01EF5AAD
:10BE4000FF4F3081369FB0011124660F672F661FA8
:10BE5000770B7195698331966081269FB00111241B
:10BE6000660F672F661F770B71956A8380914E1658
:10BE700090914D16981719F08F5F8F70F9CF098147
:10BE8000002349F10E9425EE0091370B1091380BE9
:10BE90002091390B30913A0BDC01CB0101151105D2
:10BEA0002105310579F48C599F4FAF4FBF4F8093D7
:10BEB000370B9093380BA093390BB0933A0B1FEFCD
:10BEC000198311C0801B910BA20BB30BB7FF0BC0E2
:10BED0000FEF098308C01092370B1092380B1092A5
:10BEE000390B10923A0B1981612F70E089E00E94A2
:10BEF00003ED0A81002349F10E9425EE00913B0BDE
:10BF000010913C0B20913D0B30913E0BDC01CB019D
:10BF1000011511052105310579F48C599F4FAF4F5B
:10BF2000BF4F80933B0B90933C0BA0933D0BB09382
:10BF30003E0B1FEF1A8311C0801B910BA20BB30B9A
:10BF4000B7FF0BC00FEF0A8308C010923B0B109293
:10BF50003C0B10923D0B10923E0B1A81612F70E04A
:10BF600087E00E9403ED80919313882309F4FBC0BE
:10BF70002090550230905602009157020F83109185
:10BF800058021E8360913D0C70913E0C6E5F7F4F96
:10BF9000072E000C880B990B0F94EE209101A8013D
:10BFA0000F94E72087FDDFC000914E1609831A82A7
:10BFB0001B821C821D8280914D161981811709F404
:10BFC00060C0812F90E023E5289FF001299FF00DAC
:10BFD0001124E05BF34F458956896789708D452BA5
:10BFE000462B472B81F4418D528D638D748D452BEB
:10BFF000462B472B41F4458D568D678D70A1452BFF
:10C00000462B472BC9F133E5389F8001399F100D2E
:10C010001124005B134FF801618172818381948147
:10C020000F948B2A4B015C01F80161A172A183A1DD
:10C0300094A10F94EC202B013C01F80165A176A19D
:10C0400087A190A50F94EC209B01AC01C301B20124
:10C050000F94D728A50194010F944D215B018C0109
:10C060002A813B814C815D810F943D2A181624F46E
:10C07000AA82BB820C831D8389818F5F8F70898325
:10C080009ACF2091590230915A0240915B0250910F
:10C090005C026A817B818C819D810F944D2191018D
:10C0A0004F815E810F94DD275B018C01609051020E
:10C0B0007090520280905302909054029B01AC0108
:10C0C000B1018F819E810F943D2A18167CF0930157
:10C0D000A401B501C8010F943D2A181624F41301D8
:10C0E0008F829E8203C015010F831E838090330BC5
:10C0F0009090340BA090350BB090360B91014F818E
:10C100005E81C501B4010F943D2A1816D4F420E0D5
:10C1100037ED43EA5CE3B1018F819E810F944D219D
:10C120002B013C0128E431EE4AE75FE3C501B4018D
:10C130000F944D21A30192010F94DD271B018F83E2
:10C140009E83C101AF81BE818093330B9093340BEA
:10C15000A093350BB093360BB101CD010F94492953
:10C16000CB010E9475DEF4E6CF0ED11CE11CF11C60
:10C17000C0923F0BD092400BE092410BF092420BE9
:10C180000F94A00780916713813009F06EC00E9460
:10C1900025EE6B017C018091480B9091490BA09199
:10C1A0004A0BB0914B0B97018601081B190B2A0B08
:10C1B0003B0B37FD3AC08090681390906913A090B4
:10C1C0006A13B0906B130F94DE0C60936813709336
:10C1D000691380936A1390936B130091190910915E
:10C1E0001A0920911B0930911C09081919092A09FB
:10C1F0003B09DC01CB01800F911FA21FB31F80936D
:10C20000190990931A09A0931B09B0931C09D7012F
:10C21000C601805F984DAF4FBF4F8093480B9093FE
:10C22000490BA0934A0BB0934B0B8091440B909118
:10C23000450BA091460BB091470BA7019601281B17
:10C24000390B4A0B5B0B57FD10C030E8C30E3EEEB6
:10C25000D31EE11CF11CC092440BD092450BE0921E
:10C26000460BF092470B0E94DEC68091EC088823B3
:10C2700091F00E9425EE0091E8081091E9082091C4
:10C28000EA083091EB08DC01CB01801B910BA20B7B
:10C29000B30BB7FFC8C00E9425EE6B017C01209153
:10C2A000E708222309F4DDC08091E3089091E408B7
:10C2B000A091E508B091E608B701A601481B590B0B
:10C2C0006A0B7B0B77FDCDC030E0A8EEB3E00F9496
:10C2D0009127C60ED71EE81EF91EC092E308D09221
:10C2E000E408E092E508F092E60827960FB6F89485
:10C2F000DEBF0FBECDBFDF91CF911F910F91FF9099
:10C30000EF90DF90CF90BF90AF909F908F907F90F5
:10C310006F905F904F903F902F900C94175111E0C9
:10C320001093F8088091BC0A811169C08DE996E0EC
:10C330000E94D6F984E08093C20882E08093BD0811
:10C3400081E09AE59093E0168093DF168EE490E00A
:10C350009093E2168093E11687E08093D31682E8EB
:10C360008093D61684E890E0A0E0B0E08093D716E2
:10C370009093D816A093D916B093DA160F94B600FE
:10C3800010936C130E9463D040E064E271E183EC8F
:10C390009CE20E946FD080E30E94CBF88AE00E946A
:10C3A000CBF80E9457D08091F50860E018271983D8
:10C3B000112319F083EA9BE20DC082E191E10E9412
:10C3C0003FD080E30E94CBF88AE00E94CBF860E087
:10C3D0008CEE90E10E943FD080E091E10E94025CEF
:10C3E00080E30E94CBF88AE00E94CBF80981002309
:10C3F00031F082EF90E190933709809336090E94E3
:10C4000043C849CC8091730290917402A091750247
:10C41000B09176028093DC119093DD11A093DE1130
:10C42000B093DF1128CC0E9425EE6B017C01209196
:10C43000EC0830E0A8EEB3E00F949127C60ED71EAB
:10C44000E81EF91EC092E808D092E908E092EA08D6
:10C45000F092EB0880E00E9494D68AE00E94CBF82C
:10C460001ACF27960FB6F894DEBF0FBECDBFDF916F
:10C47000CF911F910F91FF90EF90DF90CF90BF90E1
:10C48000AF909F908F907F906F905F904F903F9074
:10C490002F900895CF92DF92EF92FF92C0906C029E
:10C4A000D0906D02E0906E02F0906F02FC018081EE
:10C4B0009181A281B38180936C0290936D02A093CD
:10C4C0006E02B0936F020E943AEFC0926C02D0925B
:10C4D0006D02E0926E02F0926F02FF90EF90DF909B
:10C4E000CF9008952F923F924F925F926F927F92DA
:10C4F0008F929F92AF92BF92CF92DF92EF92FF9274
:10C500000F931F93CF93DF93CDB7DEB76F970FB61F
:10C51000F894DEBF0FBECDBF9C8F8B8F7E8F6D8F4B
:10C52000212C312C2FEF28873FEF3F834FEF488B93
:10C530005FE4598B83EC8A8B97E49B8B21E030E09E
:10C5400040E050E0022C04C0220F331F441F551F4F
:10C550000A94D2F72F8B388F498F5A8F48EB5BE0C4
:10C560005B874A8700E010E02F8EAA85BB858D91FE
:10C570009D91BB87AA87A0E0B0E02F89388D498DB7
:10C580005A8D82239323A423B523892B8A2B8B2BAB
:10C5900009F0ECC08091501490915114289EB00184
:10C5A000299E700D389E700D11248091EE0B909194
:10C5B000EF0B680F791F072E000C880B990B0F9457
:10C5C000EE206C877D878E879F8780915214909193
:10C5D0005314089FB001099F700D189F700D11240E
:10C5E0008091F00B9091F10B680F791F072E000CD2
:10C5F000880B990B0F94EE206B017C012C853D85F7
:10C600004E855F85AB8DBC8D6D917D918D919C919B
:10C610000F94DC272B013C01A7019601ED8DFE8DC7
:10C6200060817181828193810F94DC274B015C01D1
:10C63000A3019201C301B2010F944D212B013C01D2
:10C64000A5019401C501B4010F944D219B01AC01DA
:10C65000C301B2010F94DD270F948B2A4B015C01BB
:10C660002C853D854E855F856091DC0B7091DD0BDF
:10C670008091DE0B9091DF0B0F94DC272B013C01A6
:10C68000A70196016091D80B7091D90B8091DA0BBC
:10C690009091DB0B0F94DC276B017C01A3019201CD
:10C6A000C301B2010F944D212B013C01A70196015A
:10C6B000C701B6010F944D219B01AC01C301B2012A
:10C6C0000F94DD270F948B2A20E030E040E751E4FF
:10C6D0000F94D728A50194010F94DD276B017C01ED
:10C6E0008090E00B9090E10BA090E20BB090E30BF8
:10C6F00020E030E040E85FE3C501B4010F943D2A3B
:10C700001816FCF4C501B4010F9449294B015C01D2
:10C7100016161706180619063CF40F942A1CA501D4
:10C7200094010F945F2703C060E070E0CB010F9489
:10C73000EE209B01AC01B601C7010F94DD276B0110
:10C740007C01288939894A895B89B601C7010F9420
:10C75000E72087FF0BC0FF8DF8870F83C986DC8A2F
:10C76000ED8AFE8AC88AD98AEA8AFB8A0F5F1F4F40
:10C770000530110509F0F9CE2FEF221A320A35E003
:10C780002316310409F0DACE4F81E42FF0E0EE0FEA
:10C79000FF1FE854F44F81E090E0088402C0880F46
:10C7A000991F0A94E2F720813181822B932B918388
:10C7B000808389859C89AD89BE898B839C83AD8369
:10C7C000BE83482F5C816D817E8128853F8180E01A
:10C7D00090E06F960FB6F894DEBF0FBECDBFDF912D
:10C7E000CF911F910F91FF90EF90DF90CF90BF906E
:10C7F000AF909F908F907F906F905F904F903F9001
:10C800002F9008958C3891051CF02CE880E002C030
:10C81000282F892F20930209809303090C94D7DDD8
:10C8200080E1E7E7F2E0A9EBB3E101900D928A9590
:10C83000E1F708952F923F924F925F926F927F920D
:10C840008F929F92AF92BF92CF92DF92EF92FF9220
:10C850000F931F93CF93DF9300D01F921F92CDB7FA
:10C86000DEB77C018B016A011901809077029090FC
:10C870007802A0907902B0907A02A5019401FC019F
:10C8800060817181828193810F94E720F1E0FD83C3
:10C89000811112C020917B0230917C0240917D0277
:10C8A00050917E02F80160817181828193810F94A1
:10C8B000E720811101C01D82F60140805180628015
:10C8C000738020911C0230911D0240911E025091F4
:10C8D0001F02C301B2010F94E720882309F455C059
:10C8E00040921C0250921D0260921E0270921F0222
:10C8F00020E030E040E05FE36091AF117091B01153
:10C900008091B1119091B2110F944D2169837A8376
:10C910008B839C838092B9139092BA13A092BB131D
:10C92000B092BC1380917B0290917C02A0917D0219
:10C93000B0917E028093BD139093BE13A093BF135A
:10C94000B093C013F60180819181A281B38180935D
:10C95000C1139093C213A093C313B093C4138091D7
:10C96000830290918402A0918502B0918602809307
:10C97000C5139093C613A093C713B093C813CE01E9
:10C9800001960E944A620E941064FD81F1110FC05D
:10C9900020E030E040EC5FE36091B3117091B4119E
:10C9A0008091B5119091B6110F94D72804C060E022
:10C9B00070E080EA91E469837A838B839C83F7013A
:10C9C00080819181A281B3818093B9139093BA132E
:10C9D000A093BB13B093BC13F80180819181A28115
:10C9E000B3818093BD139093BE13A093BF13B093F4
:10C9F000C013F10120813181428153816091C513BF
:10CA00007091C6138091C7139091C8130F94DD27BE
:10CA10006093C5137093C6138093C7139093C81384
:10CA2000CE0101960E944A620E9410640F900F90FE
:10CA30000F900F900F90DF91CF911F910F91FF906A
:10CA4000EF90DF90CF90BF90AF909F908F907F90AE
:10CA50006F905F904F903F902F9008958091321289
:10CA600090913312892B39F00E949ACF91E0811175
:10CA700003C090E001C091E0892F08952F923F926A
:10CA80004F925F926F927F928F929F92AF92BF92DE
:10CA9000CF92DF92EF92FF920F931F93CF93DF938A
:10CAA000CDB7DEB762970FB6F894DEBF0FBECDBF2D
:10CAB00083E50E94E9CF882349F00E942E65182F54
:10CAC000811106C080E00E94D0D502C01091AC1840
:10CAD0008091770290917802A0917902B0917A02C8
:10CAE00089839A83AB83BC8380917B0290917C0283
:10CAF000A0917D02B0917E028D839E83AF83B88723
:10CB000080917F0290918002A0918102B091820277
:10CB100089879A87AB87BC8786E50E94E9CF682E14
:10CB20008091501490915114892B09F4B1C083E481
:10CB30000E94E9CF882309F4B6C00E94B2CF1B013E
:10CB40002C01712C812C68EC962E72ECA72EB12C46
:10CB5000C12C28EC2F8732E4388B85E08D879D85AA
:10CB600091509D879F3FD9F1E5E0EE8735E0399FF1
:10CB7000900111243A8B298B3E8531503E873F3FEF
:10CB800071F3E989FA89E30FF11DEE0FFF1FEE0F34
:10CB9000FF1FE45AFB4ED080E180F28003812B2DF1
:10CBA0003C2D4F8558896D2D7E2D8F2D902F0F9404
:10CBB000E72087FF04C0BD2CCE2CFF86088B2D2DCF
:10CBC0003E2D4F2D502F672D782D892D9A2D0F94A6
:10CBD000E72087FFD1CF7D2C4701A02ECDCF272D79
:10CBE000382D492D5A2D6B2D7C2D8F8598890F94CA
:10CBF000DD2720E030E040E05FE30F944D21A2010B
:10CC000091010F94DD271B012C012DEB37E346E842
:10CC100055EB0F943D2A87FD0AC02DEB37E346E81C
:10CC200055E3C201B1010F94E7201816E4F580E046
:10CC30000E94D0D505E045E0C42E0150A0F135E0BA
:10CC4000D32EC09E50011124DA949FEFD916A9F378
:10CC50007501ED0CF11CC701880F991F880F991FF2
:10CC6000FC01E45AFB4E7F01A201910160817181B8
:10CC7000828193810F94DC279B01AC01F7016083D3
:10CC80007183828393836D2D802F0E944784DCCF34
:10CC9000111102C0662089F00E94EB5C80EE94E1E5
:10CCA0000E94025C16C0662041F080915014909161
:10CCB0005114892B11F00E94115C8AE50E94E9CF82
:10CCC000882321F00E94B2CF0F94A606812F0E94E4
:10CCD000D0D5112351F08091AC18811106C00E946B
:10CCE000E75C81EC94E10E94025C0E94EB5C83EBC8
:10CCF00094E10E94025C8091AC18811103C087EE20
:10CD00009CE002C08BEE9CE00E94025C8AE00E94E4
:10CD1000CBF80E94EB5C86EA94E10E94025CC09032
:10CD2000AD18D090AE18E090AF18F090B01820E099
:10CD300030E0A901C701B6010F943D2A181644F44A
:10CD400042E0C701B6010E945BF90E94D0F904C01D
:10CD500081EA94E10E94025C4CE050E067E772E0F7
:10CD6000CE0101960F94FC2A892BD1F062960FB662
:10CD7000F894DEBF0FBECDBFDF91CF911F910F9111
:10CD8000FF90EF90DF90CF90BF90AF909F908F90EB
:10CD90007F906F905F904F903F902F900C94CFF3C7
:10CDA00062960FB6F894DEBF0FBECDBFDF91CF9174
:10CDB0001F910F91FF90EF90DF90CF90BF90AF90B9
:10CDC0009F908F907F906F905F904F903F902F90AB
:10CDD0000895CF93DF93C82FD62F0E9432D0882397
:10CDE00021F0DF91CF910C942E658C2F0E94E9CF1A
:10CDF000811101C08D2FDF91CF9108952F923F9225
:10CE00004F925F926F927F928F929F92AF92BF925A
:10CE1000CF92DF92EF92FF920F931F93CF93DF9306
:10CE2000CDB7DEB7C355D1090FB6F894DEBF0FBE3C
:10CE3000CDBF80E994E10E94025C0E949FE78111CE
:10CE40000C94A86F84E50E9432D0882329F00E94B8
:10CE5000AECF81110E948E8280E090E0A0E8BFE317
:10CE60008093B1139093B213A093B313B093B41300
:10CE70008093B5139093B613A093B713B093B813E0
:10CE80008DEC9CECACE4BEE38093AD139093AE13B9
:10CE9000A093AF13B093B01380E090E0A0E2B1E4B0
:10CEA0008093E90B9093EA0BA093EB0BB093EC0B00
:10CEB0008CE390E09093E80B8093E70B8DEC90E08F
:10CEC0009093E60B8093E50B1092E40B4AE959E945
:10CED00069E97EE38FE40E9414866BAF7CAF8DAF6F
:10CEE0009EAF60E083E40E94E96660968FAF609732
:10CEF00060E08BE40E94E96661968FAF619782E4FF
:10CF00000E9432D08823C9F00E94B2CF0F944929E1
:10CF10007093E80B6093E70B6115710571F068522F
:10CF200071096536710548F06CE870E082E694E1BD
:10CF30000E94C75C8DE594E1AEC18CE40E9432D0C2
:10CF4000882301F10E94B2CF6B017C016093AD1385
:10CF50007093AE138093AF139093B01320E030E042
:10CF6000A9010F943D2A87FD0AC020E030E040E08F
:10CF700050E4C701B6010F94E72018161CF485E3AE
:10CF800094E189C181E50E94E9CF882351F1809124
:10CF9000321290913312892B09F10E94B2CF6B01AA
:10CFA0007C016093B5137093B6138093B71390937D
:10CFB000B8132DEC3CEC4CE45DE30F943D2A87FD67
:10CFC0000AC020E030E040E751E4C701B6010F9409
:10CFD000E720181634F484E094E15DC189ED93E113
:10CFE0005AC183E50E9432D08823C9F00E94B2CF93
:10CFF0004B015C012DEC3CEC4CEC5DE30F943D2AC5
:10D0000087FD0AC020E030E040E050E4C501B401F3
:10D010000F94E720181654F482EB93E13CC17DECA9
:10D02000872E7CEC972EA92C7EE3B72E80E50E94FC
:10D03000E9CF882371F18091321290913312892BBC
:10D0400019F48AE793E127C18091E40B8F5F809305
:10D05000E40B0E94B2CF6B017C016093E90B7093EB
:10D06000EA0B8093EB0B9093EC0B20E030E0A901EE
:10D070000F943D2A87FD0AC020E030E048EC51E4DF
:10D08000C701B6010F94E72018161CF482E593E15E
:10D0900002C186E40E9432D08823C9F00E94B2CF38
:10D0A0006B017C0120E030E040E85FE30F943D2A13
:10D0B00087FD0AC020E030E040E850E4C701B60137
:10D0C0000F94E72018164CF489E293E1E4C0C12CD8
:10D0D000D12C60EEE62E6FE3F62EA7019601C70174
:10D0E000B6010F944D219B01AC0160E070E084E437
:10D0F00090E40F94D7282091B1133091B21340914E
:10D10000B3135091B4130F944D212B013C01A50191
:10D110009401C501B4010F944D21A70196010F940C
:10D120004D212CEE31E548EB5DE30F94D7289B01B0
:10D13000AC01C301B2010F944D216093B113709300
:10D14000B2138093B3139093B41388E40E9432D047
:10D15000882381F00E94B2CF0F9449297093E60B87
:10D160006093E50B655A71096838710518F08BEF0B
:10D1700092E191C085E50E94E9CF8823F1F00E94F9
:10D1800025EE611571058105910511F00F94781C4C
:10D190008091321290913312892B19F00E94B2CFF4
:10D1A00004C060E070E088E492E46093E00B709368
:10D1B000E10B8093E20B9093E30B82E50E94E9CFB1
:10D1C000811103C087EC92E166C080913212909188
:10D1D0003312892B61F00E94AECF2F969FAF8EAF96
:10D1E0002F97181619064CF083E992E154C02AE1F2
:10D1F00030E02F963FAF2EAF2F9788E50E9432D0B8
:10D20000882369F00E94B2CF2091C9133091CA13CC
:10D210004091CB135091CC130F94DC2708C0609140
:10D220007702709178028091790290917A026093EE
:10D23000DC0B7093DD0B8093DE0B9093DF0B89E5A5
:10D240000E9432D0882379F00E94B2CF2091CD1372
:10D250003091CE134091CF135091D0130F94DC270F
:10D26000AB01BC0108C040917B0250917C026091EF
:10D270007D0270917E024093D80B5093D90B60933E
:10D28000DA0B7093DB0B8CED9BE00E94DFAA81111F
:10D2900005C089E692E10E94025C5AC684E40E94BD
:10D2A000E9CF91E089270E94D0D520E030E040EA24
:10D2B00050E460917F027091800280918102909190
:10D2C00082020F94E72087FF1CC0198A1A8A1B8AE2
:10D2D0001C8A80E090E0A0EAB0E489839A83AB8363
:10D2E000BC83BE016F5E7F4FCE0101960E9424F386
:10D2F00080E1E9EBF3E1A7E7B2E001900D928A95B6
:10D30000E1F73091521362963FAF62971092521339
:10D310000E9401CB88E492E10E94025C8091E70BBD
:10D320009091E80B8A3191056CF48091E50B909116
:10D33000E60B0E9475DE61E080E00E9484D88111D6
:10D3400009C059C50E94026481E00E9406D781117C
:10D35000ECCF51C510928302109284021092850284
:10D360001092860283E892E00E9454C88091E40BF8
:10D370008823B1F10E9410642091C5133091C61327
:10D380004091C7135091C8136091E90B7091EA0B5B
:10D390008091EB0B9091EC0B0F94DD276093C513FC
:10D3A0007093C6138093C7139093C81320E030E0A6
:10D3B00040E751E46091B3117091B4118091B511BF
:10D3C0009091B6110F94D72869837A838B839C83BD
:10D3D000CE0101960E944A620E9410640E9479EA7E
:10D3E00080E2E8EBFBE0DF01282F1D922A95E9F7A8
:10D3F000E8E9FBE0DF01282F1D922A95E9F7E8E72D
:10D40000FBE0DF011D928A95E9F70E94106480918C
:10D41000AD139091AE13A091AF13B091B013809360
:10D42000C1139093C213A093C313B093C413198272
:10D430001A821B821C829E012F5F3F4F41EC53E1F9
:10D440006DEB73E189EB93E10E941A649E01255C08
:10D450003F4F41EC53E16DEB73E189EB93E10E94A7
:10D460001A646096BFAD6097BB2329F06BE772E04A
:10D4700087E792E004C068ED7BE08CED9BE00E94C2
:10D480007262298F3A8F4B8F5C8F6D8F7E8F3FAF8B
:10D490002D962FAF2D972D96EFAD2D97E7FD94C4C8
:10D4A000FFADF7FD91C420915014309151144E2FCF
:10D4B0004203B001439F700D11248091EE0B9091B7
:10D4C000EF0B680F791F072E000C880B990B0F9438
:10D4D000EE202B013C01CB01D3018FAB98AFA9AF5C
:10D4E000BAAF20915214309153144FAD4203B001A2
:10D4F000439F700D11248091F00B9091F10B680FF8
:10D50000791F072E000C880B990B0F94EE20162F15
:10D51000072FF82EE92E462F572F682F792FCE018F
:10D52000C7960E94DFAA882309F452C420E030E0A5
:10D5300040EA50E4B201C3010F94DD27D62E272E16
:10D54000382EC92E862F922DA32DBC2D8BAB9CABD4
:10D55000ADABBEAB812F902FAF2DBE2D8FA798AB5B
:10D56000A9ABBAAB2D968FAD2D9781114AC09FAD57
:10D5700091111FC020E030E040EA50E4612F702F8D
:10D580008F2D9E2D0F94DD2721966FAF2197239627
:10D590007FAF239725968FAF259727969FAF279725
:10D5A000AFADD42C252C362CC72CAA2309F4C6C029
:10D5B00023C0C201D3018BAB9CABADABBEAB20E0B3
:10D5C00030E040EA50E4612F702F8F2D9E2D0F9494
:10D5D000DC276FA778AB89AB9AABBFADB43054F200
:10D5E00021961FAF219723960FAF23972596FFAE65
:10D5F00025972796EFAE2797EFADE4300CF489C05E
:10D600009DC02D96FFAD2D97F4300CF453C02FAD77
:10D6100024305CF020E030E040EA50E4B201C30185
:10D620000F94DC27362F272F03C0342D252DC3015F
:10D63000432F522FBC014BAB5CAB6DAB7EAB3FAD10
:10D6400031117DC420E030E040EA50E4B201C30172
:10D650000F94DC27D62E272E382EC92E20E030E05E
:10D6600040EA50E4612F702F8F2D9E2D0F94DD27FF
:10D670006FA778AB89AB9AAB4FAD442309F452C086
:10D6800020E030E040EA50E4612F702F8F2D9E2D76
:10D690000F94DC2721966FAF219723967FAF2397B6
:10D6A00025968FAF259727969FAF27978FAD84300C
:10D6B00084F144C09FAD91110FC020E030E040E202
:10D6C00051E46D2D722D832D9C2D0F94DC27D62EC9
:10D6D000272E382EC92E11C0AFADA430C4F120E0E2
:10D6E00030E040E251E46D2D722D832D9C2D0F947E
:10D6F000DC276BAB7CAB8DAB9EAB21961FAF21972C
:10D7000023960FAF23972596FFAE25972796EFAE6A
:10D71000279752ED852E53E5952E5BE7A52E51E414
:10D72000B52E29C021961FAF219723960FAF2397BF
:10D730002596FFAE25972796EFAE279742ED842ECC
:10D7400043E5942E4BEFA42E40E4B42E14C0219652
:10D750001FAF219723960FAF23972596FFAE2597EE
:10D760002796EFAE279732ED832E33E5932E3BEFCE
:10D77000A32E31E4B32E8BA99CA9ADA9BEA92C96EA
:10D780008CAF9DAFAEAFBFAF2C979C01AD01B20186
:10D79000C3010F94DC27698B7A8B8B8B9C8B4FA4F6
:10D7A00058A869A87AA8A3019201612F702F8F2D24
:10D7B0009E2D0F94DC276D8B7E8B8F8B988F2C96F4
:10D7C0002CAD3DAD4EAD5FAD2C9760917702709161
:10D7D00078028091790290917A020F94DC272C963E
:10D7E0006CAF7DAF8EAF9FAF2C97A301920160917C
:10D7F0007B0270917C0280917D0290917E020F9459
:10D80000DC272B013C018D2D922DA32DBC2D89836E
:10D810009A83AB83BC8321968FAD219723969FADCE
:10D8200023972596AFAD25972796BFAD27978D8374
:10D830009E83AF83B8878091AD139091AE13A09172
:10D84000AF13B091B01389879A87AB87BC872DEC53
:10D850003CEC4CEC5CE3C501B4010F944D212091EC
:10D86000B1133091B2134091B3135091B4130F948C
:10D870004D21209183023091840240918502509184
:10D8800086020F94DD276D877E878F87988B2C9675
:10D890002CAD3DAD4EAD5FAD2C97CA01B9010F94D3
:10D8A0004D216B017C01A3019201C301B2010F94D0
:10D8B0004D219B01AC01C701B6010F94DD2720E08B
:10D8C00030E040E050E40F943D2A18160CF047C0B9
:10D8D0000E9479EA1BA21CA21DA21EA220E030E039
:10D8E00040E05FE360917F0270918002809181024D
:10D8F000909182020F94DD276F8F78A389A39AA35A
:10D900009E012D5D3F4FAE01415E5F4F6BE772E0C0
:10D9100087E792E00E941A641BA21CA21DA21EA20D
:10D9200020E030E040E05FE36091AD137091AE1312
:10D930008091AF139091B0130F94DD276F8F78A370
:10D9400089A39AA39E012D5D3F4FAE01415E5F4FBB
:10D95000BE01615D7F4FCE01C3960E941A641F8E87
:10D9600018A219A21AA29E01215E3F4F4DEA53E16F
:10D97000BE01615D7F4FCE01C3960E941A640E9472
:10D98000A5EA40906C0250906D0260906E0270901B
:10D990006F02E090AB11F090AC110091AD111091BD
:10D9A000AE11A090A711B090A811C090A911D0906D
:10D9B000AA119501A601B701C8010F943D2A1816B6
:10D9C00014F47501860120E030E040E251E4B70133
:10D9D000C8010F94D72860936C0270936D028093F6
:10D9E0006E0290936F0240E0BE016F5E7F4FCE01EA
:10D9F00001960E94E7C140926C0250926D026092C3
:10DA00006E0270926F020E94106422242394312CC3
:10DA1000D10111972896BFAFAEAF2897812C912CDA
:10DA20005401839427960FAC279704C0880C991C47
:10DA3000AA1CBB1C0A94D2F7412C512C32014394EE
:10DA4000022C04C0440C551C661C771C0A94D2F7A7
:10DA5000482859286A287B28E1E0F0E027960FAC97
:10DA6000279702C0EE0FFF1F0A94E2F72A96FFAF36
:10DA7000EEAF2A9728E73BE026963FAF2EAF2697DA
:10DA800088EB9BE024969FAF8EAF2497A8E9BBE07C
:10DA90002296BFAFAEAF2297C12CD12C2496EEAD0B
:10DAA000FFAD24976496FFAFEEAF649780819181BC
:10DAB000A0E0B0E084219521A621B7218415950529
:10DAC000A605B70509F099C02296AEADBFAD229765
:10DAD0008D919C91A0E0B0E088219921AA21BB21E1
:10DAE000892B8A2B8B2B09F088C00091EE0B1091AB
:10DAF000EF0BE0905014F090511428962EAD3FADEE
:10DB000028972E9DB0012F9D700D3E9D700D112404
:10DB1000600F711F6E5F7F4F072E000C880B990BF3
:10DB20000F94EE206BA77CA78DA79EA72E9CB0011B
:10DB30002F9C700D3E9C700D1124600F711F625060
:10DB40007109072E000C880B990B0F94EE206BA324
:10DB50007CA38DA39EA347E651E061E070E0CE0177
:10DB60008B960F9423078091521490915314C89E62
:10DB7000B001C99E700DD89E700D11248091F00BDC
:10DB80009091F10B680F791F161617060CF09BC1C8
:10DB9000683631E0730714F067E671E0072E000C79
:10DBA000880B990B0F94EE206F8F78A389A39AA30B
:10DBB0006FA378A789A79AA747E651E061E070E0D4
:10DBC000CE0183960F9423074FA158A569A57AA586
:10DBD000CE018B960E94DFAA81117AC12296AEAD4A
:10DBE000BFAD22978D919C9111972A96EEADFFAD16
:10DBF0002A978E2B9F2B8D939C9324962EAD3FAD11
:10DC000024972E5F3F4F24963FAF2EAF2497649604
:10DC1000AEADBFAD64978D919C91A0E0B0E088213E
:10DC20009921AA21BB21892B8A2B8B2B09F4A9C00E
:10DC3000F90180819181A0E0B0E088219921AA2199
:10DC4000BB21892B8A2B8B2B09F49BC02696EEAD2A
:10DC5000FFAD269780819181A0E0B0E088219921D5
:10DC6000AA21BB21892B8A2B8B2B09F08AC000911A
:10DC7000F00B1091F10BE0905214F0905314CE9CE5
:10DC8000B001CF9C700DDE9C700D1124600F711FD0
:10DC90006E5F7F4F072E000C880B990B0F94EE20C0
:10DCA0006FA378A789A79AA7C60101968E9DB00198
:10DCB0008F9D700D9E9D700D1124600F711F62501D
:10DCC0007109072E000C880B990B0F94EE206F8FB3
:10DCD00078A389A39AA38091501490915114289607
:10DCE0002EAD3FAD2897289FB001299F700D389F1A
:10DCF000700D11248091EE0B9091EF0B680F791F3E
:10DD0000161617060CF0FDC0683631E0730714F0E4
:10DD100067E671E0072E000C880B990B0F94EE203C
:10DD20006BA37CA38DA39EA36BA77CA78DA79EA7A7
:10DD300047E651E061E070E0CE0187960F9423073B
:10DD400047E651E061E070E0CE014F960F94230763
:10DD50004FA158A569A57AA5CE018B960E94DFAA8E
:10DD60008111D4C02696AEADBFAD26978D919C9102
:10DD700011972A96EEADFFAD2A978E2B9F2B8D9390
:10DD80009C93FFEFCF1ADF0A26962EAD3FAD269764
:10DD90002E5F3F4F26963FAF2EAF269722968EAD31
:10DDA0009FAD2297029622969FAF8EAF229795E065
:10DDB000C916D10409F072CEAFEF2A1A3A0AB6E0BA
:10DDC0002B16310409F024CE8091551280935612FF
:10DDD0002F96EEADFFAD2F9731972F96FFAFEEAF99
:10DDE0002F97EF2B41F02D96FFAD2D97F7FD03C038
:10DDF0002FAD27FF36CB6FEF8DE592E10F942E0EFE
:10DE00000E9479EA80E090E0A0EAB0E48093C11338
:10DE10009093C213A093C313B093C41319821A82B0
:10DE20001B821C829E012F5F3F4F41EC53E16DEB43
:10DE300073E189EB93E10E941A648091DC0B90916D
:10DE4000DD0BA091DE0BB091DF0B8093B9139093A3
:10DE5000BA13A093BB13B093BC138091D80B9091CD
:10DE6000D90BA091DA0BB091DB0B8093BD1390938B
:10DE7000BE13A093BF13B093C01319821A821B82E2
:10DE80001C829E012F5F3F4F41EC53E16DEB73E12C
:10DE900089EB93E10E941A6462963FAD62973093DA
:10DEA00052130E9401CB61964FAD6197411150C052
:10DEB00010920309109202090E94D7DD80E090E0E1
:10DEC0000E9475DE45C060E070E080E89FE36CCEA4
:10DED0004F8D58A169A17AA1CE0183960E94DFAA35
:10DEE000882309F47BCE9E01215E3F4FAE014D5D3C
:10DEF0005F4FBE01695D7F4FCE018B960E94D5EAD0
:10DF00006DCE60E070E080E89FE30ACF4F8D58A1AE
:10DF100069A17AA1CE0183960E94DFAA882309F421
:10DF200021CF9E01215E3F4FAE014D5D5F4FBE018F
:10DF3000695D7F4FCE018B960E94D5EA13CFFFAD6E
:10DF4000D42C252C362CC72CF4300CF099CB86CB56
:10DF5000CD5ADF4F0FB6F894DEBF0FBECDBFDF91B5
:10DF6000CF911F910F91FF90EF90DF90CF90BF90D6
:10DF7000AF909F908F907F906F905F904F903F9069
:10DF80002F9008952F923F924F925F926F927F92BF
:10DF90008F929F92AF92BF92CF92DF92EF92FF92B9
:10DFA0000F931F93CF93DF93CDB7DEB7CE59D1092F
:10DFB0000FB6F894DEBF0FBECDBF2DB63EB6CB5622
:10DFC000DF4F19821882C559D04084E690E0C956C7
:10DFD000DF4F99838883C759D04001E09E012B56BB
:10DFE0003F4F44E050E0BE016F567F4FCE0189564F
:10DFF0009F4F0E943AF89E012B563F4F42E050E05F
:10E00000BE0167567F4FCE0189569F4F0E943AF856
:10E0100043E050E0BE016F567F4F85E893E00F94D8
:10E02000422B892B19F1CC56DF4F8881C459D0403F
:10E03000882359F08FE3CF56DF4F8883C159D040F2
:10E04000CE56DF4F1882C259D0400E94EB5CBE0111
:10E050006F567F4F89EA95E10E94D45C8BE995E188
:10E060000E94025C81E08093FE0BDFC5C357DF4F47
:10E07000188219821A821B82CD58D040CB56DF4FAE
:10E0800019821882C559D04001E09E012B563F4F9E
:10E0900041E050E0BE0164567F4FCE0189569F4F4C
:10E0A0000E943AF84DB65EB680E1E5EFF2E0DE019F
:10E0B000A358BF4F01900D928A95E1F780E1E5E00A
:10E0C000F3E0DE01A359BF4F01900D928A95E1F76D
:10E0D00080E1E5E1F3E09E012F5F3F4F7901D90137
:10E0E00001900D928A95E1F7C456DF4F4881CC59D3
:10E0F000D04050E04D5F5F4F440F551F440F551FF8
:10E100008DB79EB7841B950B0FB6F8949EBF0FBEBC
:10E110008DBFADB7BEB711965D0100914B1411E0F4
:10E1200001272C563F4FBD01CE0189569F4F0E94BB
:10E130003AF800914B1401279E012B563F4F44E0C3
:10E1400050E063E971E1CE0189569F4F0E943AF891
:10E15000C456DF4FC880CC59D040D12CB3E0CB0E91
:10E16000D11CCC0CDD1CCC0CDD1CEDB7FEB7EC19C2
:10E17000FD090FB6F894FEBF0FBEEDBF2DB73EB739
:10E180002F5F3F4F49014DB75EB74C195D090FB680
:10E19000F8945EBF0FBE4DBF8DB79EB701963C0190
:10E1A00000914B1401279E012B563F4FA601B4014D
:10E1B000CE0189569F4F0E943AF800914B140127D7
:10E1C0009E012B563F4FA601B301CE0189569F4FAA
:10E1D0000E943AF800914B14002309F44EC011E05C
:10E1E00001279E012B563F4F44E050E067EB71E161
:10E1F000CE0189569F4F0E943AF800914B14012797
:10E200009E012B563F4F44E050E06BEB71E1CE0195
:10E2100089569F4F0E943AF800914B1401279E01A6
:10E220002B563F4F44E050E06FEB71E1CE01895631
:10E230009F4F0E943AF800914B1401279E012B56E4
:10E240003F4F44E050E063EC71E1CE0189569F4FAF
:10E250000E943AF800914B1401279E012B563F4F24
:10E2600044E050E067EC71E1CE0189569F4F0E9477
:10E270003AF815E0DD24D39489C0C456DF4F2881D5
:10E28000CC59D04030E02E5F3F4FE3E8F1E1C35678
:10E29000DF4FB982A882CD59D04080E090E0B7012D
:10E2A000281739073CF0C356DF4FA881B981CD59F3
:10E2B000D04012C0AC018430910510F043E050E032
:10E2C000440F551F440F551FBDE7CB2ED12CCC0E4C
:10E2D000DD1E4C0D5D1DDA01AD90BD90CD90DC9042
:10E2E000A192B192C192D1922817390714F0D401AA
:10E2F00012C0AC018430910510F043E050E0440FAF
:10E30000551F440F551F1DE6C12ED12CCC0EDD1E0E
:10E310004C0D5D1DDA01AD90BD90CD90DC90A08AD2
:10E32000B18AC28AD38A2817390714F0D3010DC0E5
:10E33000AC018430910510F043E050E0440F551FCC
:10E34000440F551F460F571FDA01AD90BD90CD9079
:10E35000DC90A0A2B1A2C2A2D3A20196B4E06B0E3F
:10E36000711C44E0840E911CC356DF4FA881B98113
:10E37000CD59D0401496C356DF4FB983A883CD59E9
:10E38000D0408430910509F08BCF29CF11500091F6
:10E390004B14112379F00D259E012B563F4F44E07D
:10E3A00050E0BE0163577F4FCE0189569F4F0E94B8
:10E3B0003AF8ECCF11E001279E012B563F4F44E085
:10E3C00050E066E07CE0CE0189569F4F0E943AF80B
:10E3D0000FB6F8945EBE0FBE4DBE00914B140127E0
:10E3E0009E012B563F4F4CE050E069E279E0CE01B0
:10E3F00089569F4F0E943AF800914B1401279E01C5
:10E400002B563F4F41E050E066E272E0CE01895664
:10E410009F4F0E943AF800914B1401279E012B5602
:10E420003F4F44E050E0BE016F5F7F4FCE01895601
:10E430009F4F0E943AF800914B1401110CC0898142
:10E440009A81AB81BC818093730290937402A093F4
:10E450007502B093760211E001279E012B563F4FC3
:10E4600044E050E06CE474E1CE0189569F4F0E9475
:10E470003AF800914B1401279E012B563F4F44E080
:10E4800050E0BE0163577F4FCE0189569F4F0E94D7
:10E490003AF801E09E012B563F4F41E050E0BE01AB
:10E4A00063597F4FCE0189569F4F0E943AF89E01D3
:10E4B0002B563F4F41E050E0BE016F5F7F4FCE01D2
:10E4C00089569F4F0E943AF8AE96AFACAE978981BD
:10E4D000A89E50011124C12CD12C00914B14CA14B8
:10E4E000DB0491F001279E012B563F4F44E050E0A2
:10E4F000BE0163577F4FCE0189569F4F0E943AF865
:10E50000BFEFCB1ADB0AE9CF81E008279E012B562B
:10E510003F4F44E050E065ED73E1CE0189569F4FD7
:10E520000E943AF81AE0DD24D394115089F000914A
:10E530004B140D259E012B563F4F44E050E0BE0189
:10E5400063577F4FCE0189569F4F0E943AF8EDCF17
:10E5500001E09E012B563F4F41E050E0BE01655661
:10E560007F4FCE0189569F4F0E943AF89E012B564D
:10E570003F4F41E050E0BE0163587F4FCE018956C6
:10E580009F4F0E943AF8C556DF4F8881CB59D04043
:10E5900000914B148530C9F5EE968FADEE9785301E
:10E5A000A1F5011103C080E00E94D0D500914B1469
:10E5B00011E001279E012B563F4F44E050E060E5FB
:10E5C00074E1CE0189569F4F0E943AF800914B1496
:10E5D00001279E012B563F4F44E050E06EEE7BE05A
:10E5E000CE0189569F4F0E943AF800914B140127A3
:10E5F0009E012B563F4F44E650E06CE574E1CE019E
:10E6000089569F4F0E943AF843C011E001279E01AE
:10E610002B563F4F44E050E0BE0163597F4FCE017F
:10E6200089569F4F0E943AF800914B1401279E0192
:10E630002B563F4F44E050E0BE016F5F7F4FCE014D
:10E6400089569F4F0E943AF8C556DF4FA880CB5994
:10E65000D040EE968FADEE97A89E50011124C12CAC
:10E66000D12CAC14BD04A1F000914B1401279E01E4
:10E670002B563F4F44E050E0BE0163577F4FCE0121
:10E6800089569F4F0E943AF8EFEFCE1ADE0AE9CF83
:10E6900000914B1411E001279E012B563F4F41E0A2
:10E6A00050E0BE0163597F4FCE0189569F4F0E94B3
:10E6B0003AF800914B1401279E012B563F4F41E041
:10E6C00050E0B701CE0189569F4F0E943AF8009161
:10E6D0004B1401279E012B563F4F44E050E0B701F9
:10E6E000CE0189569F4F0E943AF800914B140127A2
:10E6F0009E012B563F4F41E050E06DEE7BE0CE0196
:10E7000089569F4F0E943AF800914B1401279E01B1
:10E710002B563F4F44E050E0BE0163597F4FCE017E
:10E7200089569F4F0E943AF800914B1401279E0191
:10E730002B563F4F44E050E0B701CE0189569F4F22
:10E740000E943AF800914B1401279E012B563F4F2F
:10E7500042E050E0BE0163587F4FCE0189569F4F83
:10E760000E943AF800914B1401279E012B563F4F0F
:10E7700040E150E0B701CE0189569F4F0E943AF820
:10E7800000914B1401112EC089809A80AB80BC800F
:10E7900020E030E84BE355E4C501B4010F94E720D5
:10E7A000882301F18092400C9092410CA092420C7F
:10E7B000B092430C8D819E81AF81B8858093440CCB
:10E7C0009093450CA093460CB093470C89859A858D
:10E7D000AB85BC858093480C9093490CA0934A0C60
:10E7E000B0934B0C11E001279E012B563F4F42E0A6
:10E7F00050E0BE016F5F7F4FCE0189569F4F0E9450
:10E800003AF800914B1401279E012B563F4F4CE0E4
:10E8100050E0BE016F5F7F4FCE0189569F4F0E942F
:10E820003AF800914B14011115C020E030E84BE399
:10E8300055E469817A818B819C810F94E72088233C
:10E8400049F08CE0FE013196A5E0B9E001900D920F
:10E850008A95E1F711E001279E012B563F4F42E0D8
:10E8600050E0B701CE0189569F4F0E943AF80091BF
:10E870004B1401279E012B563F4F41E050E0B7015A
:10E88000CE0189569F4F0E943AF800914B14012700
:10E890009E012B563F4F40E250E0B701CE01895612
:10E8A0009F4F0E943AF800914B1401279E012B566E
:10E8B0003F4F41E050E0BE0163597F4FCE01895682
:10E8C0009F4F0E943AF800914B1401279E012B564E
:10E8D0003F4F45E050E0B701CE0189569F4F0E945F
:10E8E0003AF800914B1401110FC0898180935213A3
:10E8F0008A819B81AC81BD8180935713909358137B
:10E90000A0935913B0935A1311E001279E012B567F
:10E910003F4F4AE150E0B701CE0189569F4F0E9418
:10E920003AF800914B1401279E012B563F4F44E3C8
:10E9300050E0B701CE0189569F4F0E943AF80091EE
:10E940004B1401279E012B563F4F46E050E0B70184
:10E95000CE0189569F4F0E943AF800914B1401272F
:10E960009E012B563F4F4DE050E0B701CE01895636
:10E970009F4F0E943AF800914B1401279E012B569D
:10E980003F4F44E050E0B701CE0189569F4F0E94AF
:10E990003AF800914B1401110CC089819A81AB8126
:10E9A000BC8180934C0C90934D0CA0934E0CB09373
:10E9B0004F0C11E001279E012B563F4F4CE050E0D9
:10E9C000B701CE0189569F4F0E943AF800914B142F
:10E9D00001279E012B563F4F4CE650E0B701CE0178
:10E9E00089569F4F0E943AF819821A821B821C8214
:10E9F0001D821E821F82188619861A861B861C8617
:10EA000000914B1401279E012B563F4F4CE050E0E4
:10EA1000B701CE0189569F4F0E943AF800914B14DE
:10EA200001279E012B563F4F48E050E064E574E11A
:10EA3000CE0189569F4F0E943AF800914B1401274E
:10EA40009E012B563F4F44E050E0B701CE0189565E
:10EA50009F4F0E943AF800914B1401279E012B56BC
:10EA60003F4F44E050E0BE016B5F7F4FCE018956BF
:10EA70009F4F0E943AF800914B1401279E012B569C
:10EA80003F4F44E050E0BE01675F7F4FCE018956A3
:10EA90009F4F0E943AF800914B1401279E012B567C
:10EAA0003F4F41E050E0BE0163587F4FCE01895691
:10EAB0009F4F0E943AF800914B1401279E012B565C
:10EAC0003F4F44E050E0BE0163597F4FCE0189566D
:10EAD0009F4F0E943AF880E3D7011D928A95E9F78B
:10EAE00000914B1401279E012B563F4F40E350E00D
:10EAF000B701CE0189569F4F0E943AF880914B147E
:10EB0000811104C082EB96E00E94D6F9C956DF4F0E
:10EB100088819981C759D0408632934041F00E9444
:10EB2000E75C81E195E10E94025C81E001C080E048
:10EB30008093FE0B8823C1F00E94EB5CC956DF4F27
:10EB400068817981C759D0406456710983E995E19C
:10EB50000E94C75C62EC72E08BE895E10E94A95CC0
:10EB60008AE00E94CBF857C0CB56DF4F288139810D
:10EB7000C559D040C756DF4F88819981C959D040C7
:10EB800028173907E1F081E08093FE0B0E94E75CD3
:10EB9000C756DF4F68817981C959D0408BE695E12E
:10EBA0000E94A95CCB56DF4F68817981C559D0405E
:10EBB00086E695E10E94A95C86E595E12AC08091F0
:10EBC0004B14811128C00E94EB5C05E813E0F801AA
:10EBD00081918F01882319F00E94CBF8F8CFC95694
:10EBE000DF4F68817981C759D0406456710989E344
:10EBF00095E10E94C75CCB56DF4F48815981C559CA
:10EC0000D04060E070E08CE295E10E94985C89E27F
:10EC100095E10E94025C80914B14811106C08091A5
:10EC2000FE0B811102C00F94000C80914B148111D6
:10EC300002C00E9437FC9091FE0B81E089270FB63D
:10EC4000F8943EBE0FBE2DBEC256DF4F0FB6F894ED
:10EC5000DEBF0FBECDBFDF91CF911F910F91FF900F
:10EC6000EF90DF90CF90BF90AF909F908F907F906C
:10EC70006F905F904F903F902F900895CF92DF92CA
:10EC8000EF92FF920F931F93CF93DF93CDB7DEB731
:10EC9000CE5AD1090FB6F894DEBF0FBECDBFCF5507
:10ECA000DF4F188219821A821B82C15AD04080918C
:10ECB000F9069091FA06A091FB06B091FC06CB559F
:10ECC000DF4F88839983AA83BB83C55AD040C75539
:10ECD000DF4F19821882C95AD04084E690E0C555AA
:10ECE000DF4F99838883CB5AD0401092FE0B9E0150
:10ECF00027553F4F44E050E0BE016B557F4FCE019A
:10ED000085559F4F0E9477F8C555DF4F88819981BF
:10ED1000CB5AD0400296C555DF4F99838883CB5A92
:10ED2000D040C755DF4F19821882C95AD04081E0C0
:10ED3000C255DF4F8883CE5AD0409E0127553F4FA2
:10ED400041E050E0BE0162557F4FCE0185559F4F97
:10ED50000E9477F89E0127553F4F48E450E063E852
:10ED600071E1CE0185559F4F0E9477F88E010F5FAC
:10ED70001F4F80E1F80111928A95E9F780E090E059
:10ED8000A0EAB0E489839A83AB83BC839E012755B4
:10ED90003F4F40E150E0B801CE0185559F4F0E94A2
:10EDA00077F89E0127553F4F44E050E066E07CE055
:10EDB000CE0185559F4F0E9477F89E0127553F4F02
:10EDC0004CE050E069E279E0CE0185559F4F0E940A
:10EDD00077F89E0127553F4F41E050E066E272E030
:10EDE000CE0185559F4F0E9477F89E0127553F4FD2
:10EDF00044E050E063E772E0CE0185559F4F0E94EA
:10EE000077F88091AD189091AE18A091AF18B0919D
:10EE1000B01889839A83AB83BC839E0127553F4FEB
:10EE200044E050E0B801CE0185559F4F0E9477F82D
:10EE3000CF55DF4F188219821A821B82C15AD040E7
:10EE40007E01FDE6EF0EF11C83E0F70180838983EC
:10EE50009E0127553F4F44E050E0BE016F557F4F64
:10EE6000CE0185559F4F0E9477F89E0127553F4F51
:10EE700041E050E0B701CE0185559F4F0E9477F8E1
:10EE80009E0127553F4F41E050E0B801CE01855526
:10EE90009F4F0E9477F82AE0D22EDA949E012755E0
:10EEA0003F4F44E050E0DD2049F0BE016F557F4FF9
:10EEB000CE0185559F4F0E9477F8EFCF65ED73E146
:10EEC000CE0185559F4F0E9477F8CF55DF4F1882AE
:10EED00019821A821B82C15AD0409AE0D92EDA9444
:10EEE000DD2071F09E0127553F4F44E050E0BE0108
:10EEF0006F557F4FCE0185559F4F0E9477F8EFCF1A
:10EF000085E0F701808389839E0127553F4F41E0CB
:10EF100050E0B701CE0185559F4F0E9477F89E01C2
:10EF200027553F4F41E050E0B801CE0185559F4F36
:10EF30000E9477F89E0127553F4F44E050E060E57E
:10EF400074E1CE0185559F4F0E9477F89E012755A9
:10EF50003F4F44E050E06EEE7BE0CE0185559F4F81
:10EF60000E9477F89E0127553F4F44E650E06CE53C
:10EF700074E1CE0185559F4F0E9477F8F70110820A
:10EF80008FEF89839E0127553F4F41E050E0B70145
:10EF9000CE0185559F4F0E9477F89E0127553F4F20
:10EFA00041E050E0B801CE0185559F4F0E9477F8AF
:10EFB0009E0127553F4F44E050E061E873E0CE01E9
:10EFC00085559F4F0E9477F89E0127553F4F41E09E
:10EFD00050E06DEE7BE0CE0185559F4F0E9477F8A3
:10EFE0008091250390912603A0912703B0912803D7
:10EFF000F70180839183A283B38380912903909149
:10F000002A03A0912B03B0912C0389839A83AB83AD
:10F01000BC83C356DF4F1882CD59D040C256DF4F54
:10F020001882CE59D0409E0127553F4F44E050E012
:10F03000B701CE0185559F4F0E9477F89E01275555
:10F040003F4F44E050E0B801CE0185559F4F0E94EC
:10F0500077F89E0127553F4F42E050E0BE016356CE
:10F060007F4FCE0185559F4F0E9477F880E1F801D0
:10F0700011928A95E9F780E090E0A0E8BFE38D87E0
:10F080009E87AF87B88B8091400C9091410CA091E6
:10F09000420CB091430C89839A83AB83BC838091EB
:10F0A000440C9091450CA091460CB091470C8D8377
:10F0B0009E83AF83B8878091480C9091490CA091B2
:10F0C0004A0CB0914B0C89879A87AB87BC879E010D
:10F0D00027553F4F40E150E0B801CE0185559F4F85
:10F0E0000E9477F884E190E09A8389839E012755F6
:10F0F0003F4F42E050E0B801CE0185559F4F0E943E
:10F1000077F89E0127553F4F4CE050E065E079E0ED
:10F11000CE0185559F4F0E9477F880E290E09A8358
:10F1200089839E0127553F4F42E050E0B801CE0150
:10F1300085559F4F0E9477F881E089839E0127556E
:10F140003F4F41E050E0B801CE0185559F4F0E94EE
:10F1500077F880E2EDE2F3E0D80101900D928A9514
:10F16000E1F79E0127553F4F40E250E0B801CE0144
:10F1700085559F4F0E9477F8F70110829E01275511
:10F180003F4F41E050E0B701CE0185559F4F0E94AF
:10F1900077F89E0127553F4F41E050E062E573E16B
:10F1A000CE0185559F4F0E9477F89E0127553F4F0E
:10F1B00044E050E067E573E1CE0185559F4F0E9422
:10F1C00077F88AE1F80111928A95E9F79E012755AF
:10F1D0003F4F4AE150E0B801CE0185559F4F0E9454
:10F1E00077F884E3EDE4F3E0D80101900D928A957D
:10F1F000E1F79E0127553F4F44E350E0B801CE01AF
:10F2000085559F4F0E9477F81A8219821C821B82B3
:10F210001E821D829E0127553F4F46E050E0B801F7
:10F22000CE0185559F4F0E9477F88DE0F80111922D
:10F230008A95E9F79E0127553F4F4DE050E0B80110
:10F24000CE0185559F4F0E9477F89E0127553F4F6D
:10F2500044E050E06CE47CE0CE0185559F4F0E9475
:10F2600077F88CE0D82EF8018D2D11928A95E9F768
:10F270009E0127553F4F4CE050E0B801CE01855527
:10F280009F4F0E9477F88CE6F80111928A95E9F772
:10F290009E0127553F4F4CE650E0B801CE01855501
:10F2A0009F4F0E9477F89E0127553F4F4CE050E05A
:10F2B00062EF7BE0CE0185559F4F0E9477F89E015B
:10F2C00027553F4F48E050E064E574E1CE01855595
:10F2D0009F4F0E9477F8F7011192DA94E9F7C3552E
:10F2E000DF4F1882CD5AD04080E090E0A0E4B0E437
:10F2F000C356DF4F88839983AA83BB83CD59D040FF
:10F300009E0127553F4F44E050E0B701CE0185559F
:10F310009F4F0E9477F89E0127553F4F44E050E0F1
:10F32000B7016C5F7F4FCE0185559F4F0E9477F8E4
:10F330009E0127553F4F44E050E0B701685F7F4F83
:10F34000CE0185559F4F0E9477F89E0127553F4F6C
:10F3500041E050E0BE0163557F4FCE0185559F4F80
:10F360000E9477F89E0127553F4F44E050E0BE01D0
:10F3700063567F4FCE0185559F4F0E9477F880E3FB
:10F38000F70111928A95E9F785EC96E00E94D6F98B
:10F390009E0127553F4F40E350E0B701CE01855510
:10F3A0009F4F0E9477F81091FE0B111156C0C55562
:10F3B000DF4FC880D980CB5AD040F4E6CF1AD108AD
:10F3C000C755DF4F88819981C95AD040F701918391
:10F3D000808384E690E0C555DF4F99838883CB5ABC
:10F3E000D0409E0127553F4F44E050E065E873E070
:10F3F000CE0185559F4F0E9477F89E0127553F4FBC
:10F4000042E050E0B701CE0185559F4F0E9477F84A
:10F410000E94EB5CB6018FEF94E10E94A95CF701BA
:10F420004081518160E070E082EF94E10E94985C3D
:10F430008FEE94E10E94025CF2ECCF16F2E0DF0660
:10F4400039F00E94E75C81E195E10E94025C11E0E5
:10F450008091FE0B182B1093FE0B1091FE0B89ED83
:10F4600096E00E94D6F981E08127C255DF4F0FB6A2
:10F47000F894DEBF0FBECDBFDF91CF911F910F91EA
:10F48000FF90EF90DF90CF9008958F929F92AF9270
:10F49000BF92CF92DF92EF92FF920F931F93CF9381
:10F4A000DF93EC018B81811102C080E078C0098973
:10F4B0001A892B893C890417150726073707A8F3F3
:10F4C0006A017B01823029F4C886D986EA86FB86E8
:10F4D0000DC0C114D104E104F10451F41886198659
:10F4E0001A861B861C821D821E821F8281E057C0E5
:10F4F00088849984AA84BB84E98DFA8D258530E0BF
:10F50000275F3F4FB501A4014150510961097109BD
:10F51000022E04C076956795579547950A94D2F7C1
:10F52000D701C6010197A109B10904C0B695A795F5
:10F53000979587952A95D2F784179507A607B70759
:10F5400020F089288A288B2871F44D895E896F897B
:10F55000788D4C835D836E837F834C015D018E01CA
:10F560000C5F1F4F16C0841B950BA60BB70BF5CF76
:10F570004C815D816E817F819801898D9A8D0E9479
:10F58000BD5691E0891A9108A108B108882309F4B1
:10F590008CCF81149104A104B10451F795CFDF9170
:10F5A000CF911F910F91FF90EF90DF90CF90BF9080
:10F5B000AF909F908F9008950F931F93CF93DF93F9
:10F5C000FC012381222311F080E044C08B01EC0177
:10F5D000FB018789803139F18032B1F783E08B8379
:10F5E000F801428D538D648D758D4D8B5E8B6F8BC5
:10F5F000788F9E012F5E3F4FC8010E943E5788239F
:10F6000019F31A8F098F81E08983188619861A8663
:10F610001B861C821D821E821F82188A1C861D86E4
:10F620001E861F8617C082E08B831D8A1E8A1F8A52
:10F63000188EFB01808D918DA0E0B0E025E0880F51
:10F64000991FAA1FBB1F2A95D1F7898B9A8BAB8B69
:10F65000BC8BD7CFDF91CF911F910F910895CF939E
:10F66000DF93EC0141E0611101C040E06C857D85D4
:10F670008E859F850E94F255882341F0888920E27B
:10F68000829FC00111248F54974E02C080E090E009
:10F69000DF91CF910895CF93DF93EB01FC0123819C
:10F6A000211102C080E028C02250223020F48FE2D5
:10F6B0008883198220C060E00E942F7B009791F31D
:10F6C000FC0190E080E02EE23081303269F0883039
:10F6D00029F4DE01A90FB11D2C939F5FDE01A90F54
:10F6E000B11D30813C939F5F8F5F31968B3061F706
:10F6F000C90FD11D188281E0DF91CF9108953F920B
:10F700004F925F926F927F928F929F92AF92BF9231
:10F71000CF92DF92EF92FF920F931F93CF93DF93DD
:10F72000CDB7DEB72C970FB6F894DEBF0FBECDBFB6
:10F730005C01DC0159968D909C905A97F40181856B
:10F740009285A385B4859C01AD012F5F3F4F4F4F3C
:10F750005F4F29873A874B875C87D5011496CD90F8
:10F76000DD90ED90FC901797C114D104E104F104F1
:10F7700039F0BFEFCB1ADB0AEB0AFB0A312C07C0CA
:10F78000F401C080D180E280F380332433942601D9
:10F7900037011D821E821F821886F40181859285A1
:10F7A000A385B4852D813E814F815885281739075F
:10F7B0004A075B0708F064C089859A85AB85BC85DC
:10F7C0008C159D05AE05BF0550F482E0C82ED12CE6
:10F7D000E12CF12C92E0492E512C612C712C9E01D0
:10F7E0002F5F3F4FB701A601C4010E94BD56882379
:10F7F00009F446C089819A81AB81BC81892B8A2B0F
:10F800008B2B41F0260137019FEF491A590A690AEB
:10F81000790A05C0C414D504E604F70491F02D81DB
:10F820003E814F8158852F5F3F4F4F4F5F4F2D8354
:10F830003E834F8358873FEFC31AD30AE30AF30A84
:10F84000ACCF0FEF1FEF2FEF3FE0B301A201C401D8
:10F850000E942B56F82E882399F0D50114964D91CD
:10F860005D916D917C911797411551056105710569
:10F8700049F093018201C4010E942B56811102C0FC
:10F88000F12C29C0D50114964D925D926D927C9217
:10F890001797332051F0D301C2010196A11DB11D6C
:10F8A000F40180839183A283B383F50185899689CE
:10F8B000A789B08D892B8A2B8B2B69F4D50155969E
:10F8C0004D925D926D927C92589711968C91119702
:10F8D000806811968C938F2D2C960FB6F894DEBF0E
:10F8E0000FBECDBFDF91CF911F910F91FF90EF9091
:10F8F000DF90CF90BF90AF909F908F907F906F9050
:10F900005F904F903F90089540E050E0BA010C9412
:10F91000457A61E0FC0180810E9498EC8FEF0C94A5
:10F92000DAFAEF92FF921F93CF93DF9300D01F92EA
:10F93000CDB7DEB77C01162F29833A834B835C83D6
:10F94000FC0182810E94E6FA60E0F70180810E945A
:10F9500098EC0F945C01812F80640E94DAFA8C810C
:10F960000E94DAFA8B810E94DAFA8A810E94DAFA1E
:10F9700089810E94DAFA112311F087E801C085E934
:10F980000E94DAFA1C3011F40E94DFFA10E00E94A3
:10F99000DFFAF701838387FF04C01F3F11F01F5F69
:10F9A000F6CF0F900F900F900F90DF91CF911F9196
:10F9B000FF90EF9008950F931F93CF93DF93EC0187
:10F9C00089018C81833039F089E0440F551F661F0F
:10F9D000771F8A95D1F79A01AB0168E1CE010E94A9
:10F9E000917C811128C08EEF8EBDF801C8019E5F09
:10F9F0000DB407FEFDCF20812EBD0DB407FEFDCF57
:10FA000021812EBD32968E179F0791F70DB407FE08
:10FA1000FDCF8FEF0E94DAFA8FEF0E94DAFA0E9490
:10FA2000DFFA8B838F71853041F083E18983CE01CA
:10FA30000E94897C19C086E016C00F945C0188235F
:10FA400079F020E030E0A9016DE0CE010E94917CC8
:10FA5000811108C00E94DFFA811104C011E005C0C5
:10FA600087E101C086E1898310E0CE010E94897C94
:10FA7000812FDF91CF911F910F910895CF938091A6
:10FA8000B91A8823B9F14091B11A5091B21A609114
:10FA9000B31A7091B41A21EB38E18091BA1A90919F
:10FAA000BB1A0E94DB7CC82F811102C0C0E023C0BA
:10FAB0004091B51A5091B61A6091B71A7091B81A60
:10FAC000411551056105710591F021EB38E18091F7
:10FAD000BA1A9091BB1A0E94DB7C882339F31092EA
:10FAE000B51A1092B61A1092B71A1092B81A10924C
:10FAF000B91A01C0C1E08C2FCF910895CF93DF9345
:10FB0000EC018B81882339F1898187FF20C061E076
:10FB1000CE010E942F7BFC01892BE9F08081853E7C
:10FB2000D1F08B81823040F489899A89AB89BC8974
:10FB3000848F958FA68FB78F8D899E89AF89B88D59
:10FB4000938F828FB58BA48B89818F778983DF9187
:10FB5000CF910C943E7D81E0888380E0DF91CF914E
:10FB60000895CF93DF93EC010E947E7D1B82DF918D
:10FB7000CF910895FC01238121110C94B17D08954A
:10FB8000CF92DF92EF92FF920F931F93CF93DF9369
:10FB9000EC0189018C81833039F089E0440F551FD5
:10FBA000661F771F8A95D1F79A01AB0161E1CE01FB
:10FBB0000E94917C882339F084E08983CE010E94E1
:10FBC000897C80E03EC00E9425EE6B017C012CE226
:10FBD000C20E21E0D21EE11CF11C0E94DFFA8B83D1
:10FBE0008F3F61F40E9425EEDC01CB018C199D0949
:10FBF000AE09BF09B7FDF1CF81E11DC08E3FD1F441
:10FC00008FEF8EBDF801D801A150BE4F0DB407FE95
:10FC1000FDCF9EB591938EBDEA17FB07B9F70DB4E2
:10FC200007FEFDCF8EB58C930E94DFFA0E94DFFAAB
:10FC300011E003C08FE0898310E0CE010E94897C2F
:10FC4000812FDF91CF911F910F91FF90EF90DF9067
:10FC5000CF9008952F923F924F925F926F927F9232
:10FC60008F929F92AF92BF92CF92DF92EF92FF92CC
:10FC70000F931F93CF93DF9300D01F92CDB7DEB7C2
:10FC80009C838B834B015A01DC0113968C9181116B
:10FC900003C08FEF9FEFE3C0EB81FC81818180FF88
:10FCA000F8CFEB81FC8181899289A389B489408551
:10FCB000518562857385841B950BA60BB70BA50137
:10FCC00060E070E084179507A607B70708F45C01A9
:10FCD00075018B819C8104969A838983612C42E013
:10FCE000742EE114F10409F48BC0AB81BC81189629
:10FCF0004D915D916D917C911B976A01B1E0DB2282
:10FD0000EB81FC812381818D928D1A012B0139E0D9
:10FD100056944794379427943A95D1F7223061F45A
:10FD2000FC01828D938DA48DB58DBC01CD01620D3A
:10FD3000731D841D951D4AC0DC0114961C91115041
:10FD40001221C114D10401F511111EC0452B462BFF
:10FD5000472B59F4EB81FC8185899689A789B08D61
:10FD600084839583A683B7830FC0AB81BC8114962F
:10FD70004D915D916D917C91179729813A810E94F7
:10FD8000BD56882309F485CFEB81FC81218D328D0E
:10FD900084819581A681B7810297A109B109F901F2
:10FDA000058404C0880F991FAA1FBB1F0A94D2F7AD
:10FDB0004685578560897189840F951FA61FB71FD7
:10FDC000BC01CD01610F711D811D911D93012C1985
:10FDD0003D0987012E153F0508F489010115F2E060
:10FDE0001F0779F52091B11A3091B21A4091B31AD8
:10FDF0005091B41A621773078407950719F421C04C
:10FE0000C5012DC09401AB01BC018091BA1A90913B
:10FE1000BB1A0E94C07D882309F43BCF800E911E3F
:10FE2000EB81FC8180859185A285B385800F911F30
:10FE3000A11DB11D80879187A287B387E01AF10ABF
:10FE400050CF40E00E94F255882309F422CFB6013A
:10FE50006F54774EA801C4010F94092BDFCF0F9088
:10FE60000F900F900F90DF91CF911F910F91FF9006
:10FE7000EF90DF90CF90BF90AF909F908F907F904A
:10FE80006F905F904F903F902F900895DF92EF9288
:10FE9000FF920F931F93CF93DF938C01EB017A01B5
:10FEA0008DE0D82E40E250E0BE01C8010E942A7EBB
:10FEB0008032910539F021E0892B09F420E0822F6E
:10FEC000819544C028812223C9F1253E11F02E32AC
:10FED00031F4E114F10431F3F7011082E3CFE114BE
:10FEE000F10441F13B853F733F3021F54A8D5B8D35
:10FEF000452B01F52F713FEF320F3530D8F430E04C
:10FF000021503109D29EC001D39E900D1124D701FA
:10FF1000A80FB91FFE0120E0AD01253088F4318122
:10FF20003D932F5F32962D30C1F7288126FF02C006
:10FF3000FA0115862B8523FDB5CF08C080E006C0E9
:10FF40002B3010F43481ECCF3681EACFDF91CF91A2
:10FF50001F910F91FF90EF90DF9008954F925F9265
:10FF60006F927F929F92AF92BF92CF92DF92EF9269
:10FF7000FF920F931F93CF93DF931F92CDB7DEB7FE
:10FF80008C017B015A01C22EDB0159968D919C9107
:10FF90005A97F801928F818FCB010E94847C912C1B
:10FFA000F70180859185A285B3854189528963894E
:10FFB000748984179507A607B70708F060C025E085
:10FFC000B695A795979587952A95D1F7F82FFF7045
:10FFD000DF2ED70113968C91823008F460C041E087
:10FFE00050E0BE016F5F7F4FC7010E942A7E0197DC
:10FFF00019F4898190E002C08FEF9FEF019609F418
:020000021000EC
:100000004EC0F70180859185A285B3854F96A11DCD
:10001000B11D80879187A287B387F0E2DF9EB00190
:1000200011246F54774E61157105C9F1DB018C9174
:10003000882319F0853EC1F46CC191100EC08091E7
:10004000B11A9091B21AA091B31AB091B41AF801F2
:1000500084879587A687B787D08ADB018C91882310
:1000600061F0992493949CCF4BE050E0C5010F942C
:10007000FC2A892B09F094CF14C0992493948C2DD9
:100080008274823461F4992009F48BC0F801D0881D
:1000900061E0C8010E942F7B009709F00DC180E04C
:1000A0003BC1C7FCFCCFF0E2DF9EA00111249A0106
:1000B0002F54374ED9011B968C91817121F08C2DD4
:1000C000827109F06AC08091B11A9091B21AA09120
:1000D000B31AB091B41AF80184879587A687B787B9
:1000E000D08ACA018F54974E7C01DC0154964D9101
:1000F0005C91559760E070E0DA0199278827858B3D
:10010000968BA78BB08FF701428D538D60E070E026
:10011000482B592B6A2B7B2BD80155964D935D9319
:100120006D937C935897F9018385887161F4F70189
:10013000848D958DA68DB78DF801818B928BA38BC5
:10014000B48B81E010C0803141F598012F5E3F4FA4
:10015000D80159968D919C915A970E943E578823B9
:10016000E1F084E0F80183838C2D8F70D801119623
:100170008C931197F80114821582168217821896B3
:100180001D921D921D921C921B97C4FEB5C0C80102
:100190000F9480018111B0C082CFD80113961C92B8
:1001A0007ECFD70113968C911397823009F477CFC5
:1001B00051968D919D910D90BC91A02D803E9F4FA9
:1001C000AF41B10508F06BCFC7010E947F7B882348
:1001D00009F465CF0E943E7D882309F460CFD701E2
:1001E00059962D913C915A9714968D919D910D9011
:1001F000BC91A02D0297A109B109F901058404C0A1
:10020000880F991FAA1FBB1F0A94D2F746845784F0
:1002100060887188480E591E6A1E7B1E81E080939B
:10022000B91A4092B11A5092B21A6092B31A7092EF
:10023000B41A80E092E0E1EBF8E1DF019C011D924D
:1002400021503040E1F7DD24D394D7015996ED9148
:10025000FC915A978481D81698F421EB38E1B301C8
:10026000A2014D0D511D611D711D8091BA1A909111
:10027000BB1A0E94DB7C882309F411CFD394E5CF0D
:1002800080E092E0A0E0B0E0058404C0880F991FF0
:10029000AA1FBB1F0A94D2F7F701418952896389CB
:1002A0007489840F951FA61FB71F818B928BA38B18
:1002B000B48B81EB98E1D12C20E2DC011D922A95D0
:1002C000E9F72BE0F501DC0101900D922A95E1F7A9
:1002D00021E238E2FC01318B208B40E058E0578767
:1002E0004687338B228B318F208F578B468B0E9412
:1002F0003E7D8111D8CED3CEC5FE09C0F80141891B
:10030000528963897489C8010E94457A05C081E0D9
:1003100003C09110A6CE93CE0F90DF91CF911F9185
:100320000F91FF90EF90DF90CF90BF90AF909F9094
:100330007F906F905F904F9008952F923F924F92D1
:100340005F926F927F928F929F92AF92BF92CF9265
:10035000DF92EF92FF920F931F93CF93DF93CDB76E
:10036000DEB7C254D1090FB6F894DEBF0FBECDBFC1
:100370004C015B016A01322E19821C821C8E1F8E79
:100380006115710511F410E0A6C0FC018381811193
:10039000FACFFA0180818F3209F09BC0F501838189
:1003A0008250823010F485010CC0F501618D728D90
:1003B000CE014C960E94DC7A882329F38E01045EDC
:1003C0001F4FC6016C010196F60120812F32D1F337
:1003D000CE0101967C013C012E019CE1490E511C8D
:1003E0002396EFAE23972F2C9BE09150E7E3F0E0AC
:1003F000EC0FFD1FE90FF11D80E280839111F5CF15
:10040000960147E0D9018D91882369F18F3259F126
:100410008E3239F44A3009F4B6CF98E04AE09D01B3
:10042000F1CFECEDF5E12491222321F031968213F6
:10043000FACFA9CF491708F4A6CF813208F4A3CF89
:100440008F3709F4A0CF21E0290FE7E3F0E0EC0FAC
:10045000FD1FE90FF11D9FE9980F9A3108F48052B2
:100460008083922FDCCF8FA9803209F48CCF690171
:10047000F90180812F5F3F4F8F32C9F38823F9F054
:1004800021E0AE01495C5F4FB801C7010E94AE7F19
:10049000882309F478CF0A151B0519F0C8010E94BA
:1004A000B17D6E147F0441F023969FAD2397822D7A
:1004B0008701E92EF82E98CF942D852DF9CF232D85
:1004C000AE01495C5F4FB801C4010E94AE7F182F96
:1004D00002C08B017DCFCE014C960E94BA7DCE0129
:1004E00001960E94BA7D812FCE5BDF4F0FB6F89444
:1004F000DEBF0FBECDBFDF91CF911F910F91FF9057
:10050000EF90DF90CF90BF90AF909F908F907F90B3
:100510006F905F904F903F902F900895CF93C82F8A
:100520000E94EB5C84E50E94CBF86C2F70E080E0C9
:1005300090E00E943FF980E20E94CBF88AEC95E1BE
:10054000CF910C94025C8091090180FD06C08091DE
:100550005B1883FB882780F9089580E008950F9346
:100560001F93CF93DF938B01D82FC92F4630C1F44F
:100570001092891310928A1310928B1310928C137D
:1005800010928D130E94D7DD20E030E04CE053E460
:10059000B8018D2F9C2F0F94E72087FD0FC01DC041
:1005A0000F941D0F20E030E046E953E4B8018D2F91
:1005B0009C2F0F94E72087FD20C02EC020E030E064
:1005C000A901B8018D2F9C2F0F943D2A18164CF0CD
:1005D00000E010E0D0E0C0E004C000E010E0DCE0AB
:1005E000C3E4B8018D2F9C2F0F944929CB01DF91D3
:1005F000CF911F910F910C94026420E030E0A9018B
:10060000B8018D2F9C2F0F943D2A18164CF000E056
:1006100010E0D0E0C0E004C000E010E0D6E9C3E4A0
:10062000B8018D2F9C2F0F944929CB01DF91CF91D9
:100630001F910F910C9475DE9091C814977081E012
:10064000973009F080E0089580914D1690914E16F4
:10065000891B8F7069F48091BA0A811109C081E009
:100660002091360930913709232B19F480E0089541
:1006700081E008953F924F925F926F927F928F92A6
:100680009F92AF92BF92CF92DF92EF92FF920F9321
:100690001F93CF93DF93CDB7DEB762970FB6F89471
:1006A000DEBF0FBECDBF2B013C01342E24E0429FA4
:1006B000C00111249A8B898BFC01E958FD4FC08041
:1006C000D180E280F38020E030E04AE754E4C701C3
:1006D000B6010F94DC274B015C0120E030E04AE7D3
:1006E00054E4C701B6010F94DD277B018C01809192
:1006F00070028823D1F181E0381639F13816A0F064
:1007000092E0391232C08090430290904402A0904F
:100710004502B0904602E0904702F09048020091F6
:10072000490210914A0221C0809033029090340215
:10073000A0903502B0903602E0903702F090380277
:100740000091390210913A0210C080903B029090C3
:100750003C02A0903D02B0903E02E0903F02F0903B
:100760004002009141021091420280E1E9E8F3E089
:10077000DE01119601900D928A95E1F7E1E0F0E03B
:10078000EC0FFD1F89899A89E80FF91F20E030E0FE
:1007900040E752E460817181828193810F94D72870
:1007A00060936C0270936D0280936E0290936F025F
:1007B0008091BC0881FF0E9410649201A301B701DF
:1007C000C8010F943D2A181614F472018301970191
:1007D000A801B401C5010F94E72087FD02C0740190
:1007E0008501E989FA89E754FC4EC701D801808365
:1007F0009183A283B3838091BC0882608093BC08FC
:1008000062960FB6F894DEBF0FBECDBFDF91CF91D9
:100810001F910F91FF90EF90DF90CF90BF90AF901E
:100820009F908F907F906F905F904F903F90089532
:100830002091BC0890E0880F991F880F991FFC0138
:1008400021FF03C0E754FC4E02C0E958FD4F608110
:1008500071818281938108952091BC0820FF14C08A
:1008600020E83EE3629FA001639F500D729F500DF0
:100870001124CA019695879596958795009731F032
:100880008A950000E9F708950C94D35B08959F9230
:10089000AF92BF92CF92DF92EF92FF920F931F938E
:1008A000CF93DF938091C608833009F50E941C83A3
:1008B0008823E9F06091020970910309072E000C6A
:1008C000880B990B0F94EE2020E030E040E85FE3C6
:1008D0000F94DC272091FE083091FF084091000919
:1008E000509101090F94E72018160CF062C0D0E077
:1008F000FF24F39400E010E0EE24E39445E0D42ECE
:10090000C0E0CC24C39455E0B52E65E0A62E72E875
:10091000972EFC24DC16D1F18D2F90E04897A4F59A
:10092000DF5FF801BC9EE00DF11D1124EE0FFF1FEB
:10093000EE0FFF1FE45AFB4E20E030E04AE754E49C
:1009400060817181828193810F944D210F94492997
:100950007093E0166093DF16A092D3169092D6168D
:100960008D2F90E08158974F880F991F092E000C0A
:10097000AA0BBB0B8093D7169093D816A093D916C9
:10098000B093DA160F94B600CE0DC4CF0F5F1F4F91
:100990000530110579F1F11006C0EE24EA94DD244A
:1009A000DA94C4E0B6CFEE24E39435E0D32EC0E071
:1009B000B0CF81E09AE59093E0168093DF1680E453
:1009C00090E09093E2168093E11687E08093D3162F
:1009D00082E88093D61684E890E0A0E0B0E08093AF
:1009E000D7169093D816A093D916B093DA160F9411
:1009F000B6007DCFDF91CF911F910F91FF90EF90C7
:100A0000DF90CF90BF90AF909F900895AF92BF922C
:100A1000CF92DF92EF92FF920F931F93CF93DF93CA
:100A2000EC0188EEC82E80E2D82EE12CF12C02E8F1
:100A3000A12C90E2B92E15E00093D616C092D716DD
:100A4000D092D816E092D916F092DA16B092E0164B
:100A5000A092DF161093D3160F94B6008FEFC81A2A
:100A6000D80AE80AF80A80E1C81681E2D806E1044B
:100A7000F10411F748EE50E260E070E0CE01DF9142
:100A8000CF911F910F91FF90EF90DF90CF90BF908B
:100A9000AF900D94650084E08093C20882E080935B
:100AA000BD0881E09AE59093E0168093DF168EE40E
:100AB00090E09093E2168093E11687E08093D3163E
:100AC00082E88093D61684E890E0A0E0B0E08093BE
:100AD000D7169093D816A093D916B093DA160F9420
:100AE000B6008DEF96E00C94D6F987E197E00E946E
:100AF000D6F98091C608833009F443C00F946D0E77
:100B00008FE297E00E94D6F98BE397E00E94D6F936
:100B100040E060E070E0CB010F94D40E41E060E073
:100B200070E0CB010F94D40E81E08093020210920A
:100B3000C10821E030E03093C5082093C4088093B9
:100B4000000281E09AE59093E0168093DF168DE233
:100B500090E09093E2168093E11687E08093D3169D
:100B600082E88093D61684E890E0A0E0B0E080931D
:100B7000D7169093D816A093D916B093DA160D9481
:100B8000B6000895CF938BE497E00E94D6F9809148
:100B9000C608873009F446C083E08093C20881E02C
:100BA0008093000280E190E09093E0168093DF163E
:100BB00085E08093D316C2E8C093D61684E190E115
:100BC000A0E0B0E08093D7169093D816A093D916E2
:100BD000B093DA160F94B60061E070E080E090E028
:100BE0000E942C8481E09AE59093E0168093DF16B2
:100BF00085E390E09093E2168093E11687E080937E
:100C0000D316C093D61684E890E0A0E0B0E08093BD
:100C1000D7169093D816A093D916B093DA16CF9121
:100C20000D94B600CF910895CF92DF92EF92FF928C
:100C30006A017B010E9432D0882331F0FF90EF904F
:100C4000DF90CF900C94B2CFC701B601FF90EF9028
:100C5000DF90CF9008952F923F924F925F926F92C4
:100C60007F928F929F92AF92BF92CF92DF92EF923C
:100C7000FF920F931F93CF93DF93CDB7DEB7CD5481
:100C8000D1090FB6F894DEBF0FBECDBF60E070E0B3
:100C900085E40E9460AC182F81E0810F823018F04B
:100CA00085E498E154C065E070E083E40E9460ACA4
:100CB00089A760E085E50E94E9662C968FAF2C97A6
:100CC00017FF05C040E050E06CE872E404C040E06B
:100CD00050E066E173E483E50E9414860F9449298D
:100CE000072E000C880B990B0F94EE206D837E83EA
:100CF0008F832E969FAF2E970E9425EE2B013C01ED
:100D00001F3F09F409C5E12E012E000CFF08F70171
:100D100083E0EE0FFF1F8A95E1F7E75FFD4F6681E5
:100D200077816F507109072E000C880B990B0F9477
:100D3000EE209B01AC016D817E818F812E969FAD4F
:100D40002E970F943D2A1816ECF48AE198E1C35BC4
:100D5000DF4F0FB6F894DEBF0FBECDBFDF91CF914E
:100D60001F910F91FF90EF90DF90CF90BF90AF90C9
:100D70009F908F907F906F905F904F903F902F90BB
:100D80000C94025C86E098E10E94025C0E9486DE80
:100D900087E18E9DF0018F9DF00D1124EB5CF34FE8
:100DA0008FE7828722E330E0A8EEB3E00F9491272B
:100DB0006BA77CA78DA79EA79B01AC01240D351DB9
:100DC000461D571D28AF39AF4AAF5BAF81E0809316
:100DD000110210925F021F3F11F58BEA9AEAAAEA0C
:100DE000BEE38CAF9DAFAEAFBFAF2DEC3CEC4CE49F
:100DF0005EE324962CAF3DAF4EAF5FAF24972596B0
:100E00001FAE25974EE457E127965FAF4EAF279769
:100E100088E197E129969FAF8EAF299721C020E006
:100E200030E040E05EE32CAF3DAF4EAF5FAF8AE90C
:100E300099E9A9E1BFE324968CAF9DAFAEAFBFAFF8
:100E4000249725961FAF2597ACE3B7E12796BFAF50
:100E5000AEAF2797E5E0F7E12996FFAFEEAF299710
:100E600049A25AA26BA27CA24FA658AA69AA7AAA42
:100E70002FE730E040E050E0288739874A875B87DA
:100E8000188A198A1A8A1B8A1C861D861E861F8646
:100E9000C12CD12C76011E8A30E43F8B4CE1488F67
:100EA00056E4598F1A8E1B8E1C8E1D8E1BAACCAA3F
:100EB000DDAAEEAAFFAAFFE78F2E912CA12CB12C60
:100EC0001DA21EA21FA218A681E088A31D8A1C8A4B
:100ED000212C312C00E02D961FAE2D97A7E11A0290
:100EE000C00111248B5C934FFC013A962B96FFAF07
:100EF000EEAF2B979C012C5F3F4F3F8F2E8F49A564
:100F0000042E000C550B5AA749A780911102882383
:100F100009F454C20E9425EE69837A838B839C83F3
:100F200080919413882309F4BAC00E94EBDF1F3F1D
:100F300061F42090FE083090FF0800910009509164
:100F400001092D965FAF2D970EC0AE8DBF8D2C90F1
:100F500011963C90119712960C9112971396BC9192
:100F60002D96BFAF2D972A8D3B8D4C8D5D8DB10198
:100F7000802F2D969FAD2D970F943D2A18163CF487
:100F80002A8E3B8E0C8F2D96EFAD2D97ED8F2E89EF
:100F90003F89488D598DB101802F2D969FAD2D979A
:100FA0000F94E72087FF07C02E8A3F8A088F2D966F
:100FB000FFAD2D97F98F28A1222309F44DC091018F
:100FC000402F2D965FAD2D976D817E818F812E965E
:100FD0009FAD2E970F94E72087FF61C049815A810A
:100FE0006B817C814419550966097709DB01CA01C7
:100FF00088589341A109B109B7FD51C088859985E9
:10100000AA85BB8588199909AA09BB09B595A79531
:10101000979587951F3F19F48093040905C02B9677
:10102000EEADFFAD2B9780834DA35EA36FA378A792
:10103000FD81FA8F2E812B8F3F813C8F2E964FADF5
:101040002E974D8F89819A81AB81BC8189A39AA308
:10105000ABA3BCA318A223C09101402F2D965FAD76
:101060002D976D817E818F812E969FAD2E970F9447
:101070003D2A1816A4F489819A81AB81BC8129A1EB
:101080003AA14BA15CA1821B930BA40BB50BAC0145
:10109000BD01485853416109710977FFAEC120E095
:1010A00030E040EA51E46D817E818F812E969FADC4
:1010B0002E970F94DD279101402F2D965FAD2D9730
:1010C0000F94E72087FF03C080E797E1B9C08981CB
:1010D0009A81AB81BC812FA538A949A95AA9821B45
:1010E000930BA40BB50BB7FD90C025968FAD25973C
:1010F0000E9494D68AE00E94CBF889819A81AB81C4
:10110000BC818053984FAF4FBF4F8FA798ABA9AB0F
:10111000BAAB9BA9911159C02CA93DA94EA95FA9B1
:10112000B101802F2D969FAD2D970F943D2A181653
:10113000BCF520E030E040E050E4B101802F2D9676
:101140009FAD2D970F94DD276CAB7DAB8EAB9FAB26
:101150002BA53CA54DA55EA589819A81AB81BC815B
:10116000280F391F4A1F5B1F28AF39AF4AAF5BAF4B
:1011700020E030E040EC50E46D817E818F812E963E
:101180009FAD2E970F94DC279101402F2D965FADD8
:101190002D970F94E720881F8827881F8BAB35C0B9
:1011A00089819A81AB81BC8128AD39AD4AAD5BADF7
:1011B000821B930BA40BB50BB7FD27C027964EAD32
:1011C0005FAD279761E677E11DC020E030E040EA9F
:1011D00051E46D817E818F812E969FAD2E970F9465
:1011E000DC279B01AC01B101802F2D969FAD2D977F
:1011F0000F94E72087FF09C029964EAD5FAD299770
:101200006CE277E1812F0F94660789819A81AB8127
:10121000BC81880F991FAA1FBB1F29A13AA14BA10E
:101220005CA1821B930BA40BB50B84199509A6092D
:10123000B70981389F44A241B10528F087EE96E1B5
:101240000E94025CBBC049A55AA58C899D8948179C
:1012500059070CF0B0C003970CF4ADC08AE896E1D2
:101260000E94025C1F3F29F4AAE7B6E1BA83A98372
:1012700004C0E9E7F6E1FA83E98388E696E10E9493
:10128000025C89819A810E94025CB701A60186E80E
:1012900096E10E94B65C8AE00E94CBF888E696E16F
:1012A0000E94025C89819A810E94025C4C855D8566
:1012B0006E857F8582E896E10E94B65C8AE00E9496
:1012C000CBF888E696E10E94025C89819A810E94AF
:1012D000025C488959896A897B898EE796E10E9478
:1012E000B65C8AE00E94CBF82C96FFAD2C97FF23CA
:1012F00009F466C01F3F69F5C0920509D09206093E
:10130000E0920709F09208092CEA35EC47E25EE327
:101310006C857D858E859F850F944D21609309098D
:1013200070930A0980930B0990930C092CEA35EC11
:1013300047E25EE3688979898A899B890F94D72877
:1013400060930D0970930E0980930F099093100913
:1013500037C047E11402900111242B5C334F3A83CC
:101360002983D9011B96CD92DD92ED92FC921E97B6
:101370002CEA35EC47E25EE36C857D858E859F85A2
:101380000F944D21E981FA816787708B818B928B55
:101390002CEA35EC47E25EE3688979898A899B8982
:1013A0000F94D728A981BA8153966D937D938D931D
:1013B0009C93569705C00E942C1DA7CD0E9486DEE7
:1013C00081E080935F02C35BDF4F0FB6F894DEBF0E
:1013D0000FBECDBFDF91CF911F910F91FF90EF9086
:1013E000DF90CF90BF90AF909F908F907F906F9045
:1013F0005F904F903F902F9008954C895D89452BC9
:1014000009F451C14DA05EA06FA078A4480E591EEA
:101410006A1E7B1E2DA13EA14FA158A5281B390B8A
:101420004A0B5B0BC501B4010F942D27A301920158
:101430000F945F2788849984AA84BB84820E931EAC
:10144000A41EB51E54E185169104A104B1040CF14B
:101450008CEE88169104A104B1043CF490E889163E
:101460009104A104B10434F422C06BEE862E912CB9
:10147000A12CB12C88869986AA86BB862EEF30E0F7
:1014800040E050E0281939094A095B0949015A012D
:1014900012C084E190E0A0E0B0E088879987AA8735
:1014A000BB8754E1852E912CA12CB12C04C08886D9
:1014B0009986AA86BB868EEF97E10E94025C6885BA
:1014C00079858A859B850E943FF989EF97E10E9483
:1014D000025CC501B4010E943FF94E895F89688DA5
:1014E000798D82EF97E10E94B65C4A8D5B8D6C8DA1
:1014F0007D8D8BEE97E10E94B65CAC89BD89139718
:101500000CF4D1C0C501B4010F94EE2020E030E00E
:1015100040E850E40F944D216B017C012E893F89F6
:10152000488D598D6A8D7B8D8C8D9D8D0F94DC2718
:101530002BED3FE049E450E40F944D2120E030E0F2
:1015400040E05FE30F944D219B01AC01C701B60160
:101550000F94D7286B017C01C301B2010F94EE20D8
:101560002FE632E143E85AE30F944D212B013C0171
:10157000B701A60185EE97E10E94B65CB301A20116
:101580008FED97E10E94B65C1F3F09F044C02DEC3F
:101590003CEC4CE45EE3C701B6010F944D216B01B6
:1015A0007C019B01AC010F94DD27A30192010F94F4
:1015B000D7286C877D878E879F87A7019601C301F7
:1015C000B2010F944D2120E030E040E450E40F944C
:1015D000D728688B798B8A8B9B8B8FEC97E10E9445
:1015E000025CB701A60189EC97E10E94B65C4C85CC
:1015F0005D856E857F8583EC97E10E94B65C4889A6
:1016000059896A897B898DEB97E10E94B65C8AE0F3
:101610000E94CBF84AC024962CAD3DAD4EAD5FADD7
:101620002497C701B6010F944D216B017C019B01EA
:10163000AC01C301B2010F944D212CAD3DAD4EADB7
:101640005FAD0F944D21688B798B8A8B9B8BA701A3
:101650009601C701B6010F94DD27A30192010F94F3
:10166000D7286C877D878E879F878DEA97E10E94B8
:10167000025CB701A60187EA97E10E94B65C4C853F
:101680005D856E857F8581EA97E10E94B65C488919
:1016900059896A897B898BE997E10E94B65C8AE067
:1016A0000E94CBF811C01F3F79F488859985AA85DF
:1016B000BB85880D991DAA1DBB1DB595A79597954E
:1016C00087958093040911C088859985AA85BB8573
:1016D000880D991DAA1DBB1DB595A7959795879552
:1016E0002B96EEADFFAD2B9780832C893D892F5F24
:1016F0003F4F3D8B2C8B3D813E8B4E814F8B5F81CD
:10170000588F2E968FAD2E97898F49805A806B8087
:101710007C8091E098A3C3CC20E030E047E053E424
:101720006D817E818F812E969FAD2E970F943D2ADD
:1017300018160CF40ACB86E098E10E94025C0E9425
:1017400086DE8FE78093040924EB30E02DCB2F92C7
:101750003F924F925F926F927F928F929F92AF9241
:10176000BF92CF92DF92EF92FF920F931F93CF938E
:10177000DF93EB01FC0180809180A280B380C501E2
:10178000B40120E831E541E050E00F943D27C90164
:101790006DE671E00F94AC276B017C01C501B401CB
:1017A00020E13EE040E050E00F943D27CA01B9013E
:1017B00028E130E040E050E00F943D27362E272E00
:1017C000062F172F8CE3482E512C612C712CC5014C
:1017D000B401A30192010F943D27B62EA72ECA0192
:1017E000B901A30192010F943D27CB01C114D1048B
:1017F000D9F0AF92BF927F936F932F923F92FF9257
:10180000EF92DF92CF9284E596E19F938F93DF93DF
:10181000CF930F947F208DB79EB70E960FB6F89496
:101820009EBF0FBE8DBF5CC0E114F104C9F0AF9242
:10183000BF927F936F932F923F92FF92EF9284E437
:1018400096E19F938F93DF93CF930F947F20EDB713
:10185000FEB73C960FB6F894FEBF0FBEEDBF40C07A
:10186000012BB9F0AF92BF927F936F932F923F926B
:1018700088E396E19F938F93DF93CF930F947F201C
:101880008DB79EB70A960FB6F8949EBF0FBE8DBF58
:1018900027C0892BA9F0AF92BF927F936F9380E30B
:1018A00096E19F938F93DF93CF930F947F20EDB7B3
:1018B000FEB738960FB6F894FEBF0FBEEDBF10C04E
:1018C000AF92BF928CE296E19F938F93DF93CF9379
:1018D0000F947F200F900F900F900F900F900F900C
:1018E000DF91CF911F910F91FF90EF90DF90CF90FC
:1018F000BF90AF909F908F907F906F905F904F9030
:101900003F902F9008958F929F92AF92BF92CF9267
:10191000DF92EF92FF920F931F93CF93DF93CDB798
:10192000DEB7E6970FB6F894DEBF0FBECDBF0091CD
:10193000FF0B1091000C82E080932A0BF8010190BC
:101940000020E9F731975F01A01AB10AF801CF0131
:10195000801B910B8A159B0534F480818F3209F42A
:1019600010823196F4CF8BE1EFEBF5E1DE015C966E
:1019700001900D928A95E1F7E12CF12CEA14FB0419
:101980000CF084C0F801EE0DFF1D8081811103C0B1
:101990008FEFE81AF80A6801CE0CDF1CF60180818F
:1019A000882309F473C0FFEFEF1AFF0AF801EE0D68
:1019B000FF1D7F01E01AF10A81918111FACFCE015A
:1019C0004C960E94847C8BE1FE017C96DE01119690
:1019D00001900D928A95E1F7A601BE016F5F7F4FDE
:1019E00080E090E00E94C452CE0101960E94BA7D30
:1019F0008FE20E94CBF88091BC1A811103C083E66C
:101A000097E002C08CEB9AE14C01F40181914F0107
:101A1000882319F00E94CBF8F8CF80915B1884FFDF
:101A200035C019821C8221E0A601BE01645E7F4F91
:101A3000CE0101960E949D81811116C08AE00E940C
:101A4000CBF80E94EB5C88E196E10E94025CF60113
:101A500081916F01882319F00E94CBF8F8CFCE0155
:101A600001960E94BA7D12C0CE014C960E94B17DB3
:101A70008BE1FE013196DE015C9601900D928A9514
:101A8000E1F7CE0101960E94BA7D78CF8AE00E94EC
:101A9000CBF8CE014C960E94BA7DE6960FB6F8942C
:101AA000DEBF0FBECDBFDF91CF911F910F91FF9091
:101AB000EF90DF90CF90BF90AF909F908F90089560
:101AC00090915B1893FB882780F993FF06C081E013
:101AD00090916915911101C080E008954F925F9235
:101AE0006F927F92AF92BF92CF92DF92EF92FF926E
:101AF0000F931F93CF93DF931F92CDB7DEB78091E3
:101B00005B1882FF1CC18091BA0A811102C0109239
:101B1000020CEE24E39440915718509158186091AC
:101B2000591870915A188091531890915418A09197
:101B30005518B0915618481759076A077B0708F4DB
:101B4000E12C00E010E0DD24D39480E6C82E94E67A
:101B5000B92E29E6A22E8091BA0A843008F0EFC08F
:101B6000E110EDC08091020C8111E9C080916E15E9
:101B700090916F15A0917015B091711580935718C1
:101B800090935818A0935918B0935A1841E050E018
:101B9000BE016F5F7F4F86E695E10E942A7E019726
:101BA00019F4898190E002C08FEF9FEFF82E4090EA
:101BB0005718509058186090591870905A184091C2
:101BC0005318509154186091551870915618EE247E
:101BD000E394441655066606770608F4E12C44168D
:101BE000550666067706B0F4019609F461C08AE0EE
:101BF000F81609F46EC02DE0F21609F46AC083E20B
:101C0000F81619F02AE3F2127CC08091010C8111C0
